:100000000000032035B8010019B80100D1B7010084
:10001000D1B70100D1B70100D1B70100D1B70100BC
:10002000D1B70100D1B70100D1B7010019B8010063
:1000300019B80100D1B70100CDE8010045EB01007E
:1000400019B8010019B8010019B8010019B8010068
:1000500019B8010019B8010019B8010019B8010058
:1000600019B8010019B8010019B8010019B8010048
:1000700019B8010019B8010019B8010019B8010038
:1000800019B8010019B8010019B8010019B8010028
:1000900019B8010019B8010019B8010019B8010018
:1000A000398501009586010019B8010019B80100D1
:1000B00019B8010019B8010019B8010019FF0100B1
:1000C00019B801007500020019B80100D101020041
:1000D00019B801000103020019B8010019B80100A4
:1000E00019B8010019B8010019B8010019B80100C8
:1000F00019B8010019B8010019B8010019B80100B8
:1001000019B8010019B8010019B8010019B80100A7
:1001100019B80100F1C3010019B8010019B80100B4
:1001200019B8010019B8010019B8010019B8010087
:1001300019B8010019B8010019B8010019B8010077
:1001400019E6010019B801003104020019B80100D4
:1001500019B8010019B8010019B8010019B8010057
:1001600019B8010019B80100F187010019B80100A0
:1001700019B8010019B8010019B8010019B8010037
:1001800019B8010019B8010019B8010019B8010027
:1001900019B8010019B801006105020019B8010081
:1001A00019B8010019B8010019B8010019B8010007
:1001B00019B8010019B8010019B8010019B80100F7
:1001C00019B8010019B8010019B8010019B80100E7
:1001D000FFFFFFFFFFFFFFFFFFFFFFFFFFFFFFFF2F
:10040000FFFFFFFFFFFFFFFFFFFFFFFFDEF9FFFF23
:1004100010B5054C237833B9044B13B10448AFF33E
:1004200000800123237010BD00F0002000000000B8
:100430005C720200084B10B51BB108490848AFF3C5
:1004400000800848036803B910BD074B002BFBD0A0
:10045000BDE81040184700BF0000000004F0002075
:100460005C72020034EC002000000000704700BF06
:1004700010B54FF4097104461EF0CAFD204610BDA8
:1004800070B54FF06A522DED028B064645F21813F7
:1004900008EE902A40F6DB72C0F202034FF61A050E
:1004A00040F6DA70C4F24902C2F20005C3F64920F0
:1004B00008EE102A336000240FE007EE904AF8EEB1
:1004C000E77A77EE807A67EEA87A67EE887A27EE89
:1004D000800A20F079FB10EE100A23F037FB41EC84
:1004E000100B20F0D9F900230022CCF2900351EC3C
:1004F000100B23F07FFB41EC100B20F0E1F951ECE5
:10050000100B23F04FFE0134B4F5806FB6EE000AF5
:1005100025F8020FD1D14FF06A534FF21A0508EEB9
:10052000103AC2F20005002407EE904AF8EEE77A8E
:10053000013467EE887A17EE900A23F007FB9FEDEF
:10054000140B41EC110B20F03FFC002351EC100B7D
:100550000022C3F6F07323F099F900230022C4F2BD
:10056000B00323F047FB23F03DFE23F0EFFA41EC0C
:10057000100B20F0A5F951EC100B23F013FEB4F58D
:10058000806F25F8020FCFD1BDEC028B304670BDD5
:100590000000000000000040704700BF10B54FF49D
:1005A000097104461EF034FD204610BD2DE9F04FC0
:1005B0004DF6BC66C2F200060A9D0B989DF830709D
:1005C000B6F800C045F23014C0F20204C5EB000AD0
:1005D000002F18BF0C466FEA0C0B0AF1200A4DF6EB
:1005E000BC294DF6BC48043A271FA1F1040E0FFAAE
:1005F0008BFB4FEAAA1AC2F20009C2F200080026D9
:1006000027E0B4F5007F02D08CB3C943C9B239F8F2
:1006100011104CEA010101EBC00080B20BEA0004AA
:10062000E143C9B2241238F8111001F58061490084
:10063000E14010EA0C0F18BFC94357F8044F09985E
:1006400009B2013604EB8131402E03444EF8041FF9
:1006500010D052F8041F1944891301F44074554412
:10066000B4F5807FC9B2A8B2CBD1C943C9B239F8B9
:100670001110D0E7BDE8F08F2DE9F04F4DF6BC65C5
:10068000C2F2000509982E880A9D9DF82C7045F24B
:100690003014C0F20204C0EB050E002F14BF0F4649
:1006A00027466FEA06090EF1200E4DF6BC284DF6DE
:1006B000BC4C3C1F0D1F0FFA89F9FC374FEAAE1EE8
:1006C000C2F20008C2F2000C2AE0BBF5007F04D0A1
:1006D000BBF1000F30D0C943C9B238F81110314313
:1006E00001EBCA0A1FFA8AFA09EA0A0B6FEA0B0140
:1006F000C9B24FEA2B2B3CF8111001F5806149007B
:100700001AEA060F21FA0BF154F804AF18BFC943D7
:1007100009B20AEB8131BC421A4445F8041F0ED0DD
:10072000911301F4407B7044BBF5807F1FFA80FA7F
:10073000C9B2CAD1C943C9B238F81110D0E7BDE86F
:10074000F08F00BF2DE9F04F4DF6BC6083B0C2F2D0
:1007500000000D9EB0F800C00C9C9DF840A00F9FBB
:100760000E980E9D019345F2301EC0F2020EC4EBAE
:10077000060B6FEA0C06BAF1000F14BF8A46F24668
:1007800033B20BF1200B4DF6BC294DF6BC48AAF153
:10079000040600686D680093A1F1040E0AF1FC0ADA
:1007A0004FEAAB1B0137C2F20009C2F2000829E090
:1007B000B0F5007F02D098B3DB43DBB239F81330D9
:1007C0004CEA030303EBC101009B89B203EA010079
:1007D000C343DBB2001238F8133003F580635B00CB
:1007E000C34011EA0C0F18BFDB4356F8041F0198F1
:1007F0001BB29B031944564502444EF8041F284679
:1008000011D01D4643193B4113449B1303F4407020
:100810005C44B0F5807FDBB2A1B2C9D1DB43DBB26F
:1008200039F81330CEE70E9A1560536003B0BDE877
:10083000F08F00BF2DE9F04F46F2A84403EB4303CD
:10084000C0F2020404EBC3050646144689460FCDE8
:1008500091B00AAF0FC795E80300002387E80300B3
:10086000012704F160088DF8247007978DF8253072
:100870008DF826300AAD48E00AF1FF3101EB011195
:1008800006EB0111133121F00F0194E80140C0146F
:10089000C0F500706060BEF1000F3FD0BEF5FE7F76
:1008A0003EDA10AFBA441AF81CCCBCF1000F04D0E9
:1008B00012F1000C18BF4FF0010CC3F301123AB152
:1008C00010AF07EB020B1BF81CBCBBF1000F34D1BF
:1008D00003F0C003C02B02D11B9B0F2B41DDA3688B
:1008E000E2680190CDF808C0CDF800E03046FFF78F
:1008F000C3FE9DF81C300AF81C3CE368A26803EBB9
:100900008213E3601034A04514D055F8043B13F073
:10091000030A03F00402AFD14946B6E740F2FF1ED6
:10092000B0F5FE7FBDDB002AE7D110AB9A440AF890
:100930001C2CE2E711B0BDE8F08F013A02EB021285
:10094000E368CDF80CC006EB02120290CDF804E08B
:10095000A0680090133222F00F023046FFF726FE07
:10096000C7E71F46E268A36803971A9F0190CDF876
:1009700010C00297CDF800E03046FFF7E3FEB8E77D
:1009800000207047704700BF704700BF704700BF2E
:10099000704700BF704700BF10B504461DF0BEFD94
:1009A000204610BD10B5044624F0EAF80146204662
:1009B000BDE810401DF0A8BA10B5044624F0E0F8D8
:1009C000014620461DF0A0FA04464EF24020C2F235
:1009D00000001EF0ADF9204410BD00BF45F2C82054
:1009E00008B51621C0F202001DF08EFA41F2C05087
:1009F000C2F201004FF20F6119F0DAFD45F2E0207A
:100A00001421C0F202001DF07FFA4FF20F601CF0BB
:100A1000F1FB45F2F820C0F202000F211DF074FA3C
:100A20004EF24020C2F20000BDE808401EF080B93E
:100A300045F2083008B51521C0F202001DF064FA35
:100A400041F67863C2F20103FA21986C03681B68CF
:100A5000984745F220300F21C0F202001DF054FAF1
:100A60004FF60F201CF0C6FB45F2F820C0F2020042
:100A70000F211DF049FA4EF24020C2F20000BDE8FD
:100A800008401EF055B900BF45F2303008B51821B6
:100A9000C0F202001DF038FA41F67863C2F2010399
:100AA000FB21986C03681B68984745F220300F21A2
:100AB000C0F202001DF028FA4FF60F301CF09AFB2E
:100AC00045F2F820C0F202000F211DF01DFA4EF28F
:100AD0004020C2F20000BDE808401EF029B900BF66
:100AE00045F24C3008B51421C0F202001DF00CFA9A
:100AF00041F67863C2F20103FC21986C03681B681D
:100B0000984745F220300F21C0F202001DF0FCF999
:100B10004FF60F401CF06EFB45F2F820C0F20200C9
:100B20000F211DF0F1F94EF24020C2F20000BDE8A5
:100B300008401EF0FDB800BF45F2643008B51D2125
:100B4000C0F202001DF0E0F941F67863C2F2010341
:100B5000FE21986C03681B68984745F220300F21EE
:100B6000C0F202001DF0D0F94FF60F601CF042FBFE
:100B700045F2F820C0F202000F211DF0C5F94EF237
:100B80004020C2F20000BDE808401EF0D1B800BF0E
:100B900038B545F284304EF2402541F29054102190
:100BA000C2F20104C2F20005C0F202001DF0ACF96D
:100BB00028461EF0BDF820680EF056FF20680EF0A3
:100BC0005FFE20680EF070FE45F298301B21C0F2E7
:100BD00002001DF099F941F67863C2F20103FF218A
:100BE000986C03681B68984745F220300F21C0F2CB
:100BF00002001DF089F94FF60F701CF0FBFA45F268
:100C0000F820C0F202000F211DF07EF92846BDE851
:100C100038401EF08DB800BF10B50446240445F2DC
:100C2000B43004F4FE041521C0F2020044F473440D
:100C30001DF06AF944F0020441F2C0502146C2F2AC
:100C4000010019F0B5FC45F2E0201421C0F20200C9
:100C50001DF05AF920461CF0CDFA45F2F820C0F2FA
:100C600002000F211DF050F94EF24020C2F20000A8
:100C7000BDE810401EF05CB845F2CC3008B510213C
:100C8000C0F202001DF040F941F2C050C2F2010072
:100C90004FF60F2119F08CFC45F2E0201421C0F230
:100CA00002001DF031F94FF60F201CF0A3FA45F2B7
:100CB000F820C0F202000F211DF026F94EF240206C
:100CC000C2F20000BDE808401EF032B845F2E03044
:100CD00008B51321C0F202001DF016F941F2C05010
:100CE000C2F201004FF60F3119F062FC45F2E0202C
:100CF0001421C0F202001DF007F94FF60F301CF06E
:100D000079FA45F2F820C0F202000F211DF0FCF83C
:100D10004EF24020C2F20000BDE808401EF008B8C4
:100D200045F2F43008B50F21C0F202001DF0ECF8D6
:100D300041F2C050C2F201004FF60F4119F038FCE9
:100D400045F2E0201421C0F202001DF0DDF84FF65C
:100D50000F401CF04FFA45F2F820C0F202000F21BC
:100D60001DF0D2F84EF24020C2F20000BDE808406B
:100D70001DF0DEBF45F2044008B51821C0F20200A4
:100D80001DF0C2F841F2C050C2F201004FF60F61EF
:100D900019F00EFC45F2E0201421C0F202001DF013
:100DA000B3F84FF60F601CF025FA45F2F820C0F2B8
:100DB00002000F211DF0A8F84EF24020C2F2000000
:100DC000BDE808401DF0B4BF38B505464EF24024DA
:100DD00045F22040C2F200041E21C0F202001DF0C4
:100DE00093F8294600230A2220461DF0B3FF45F25E
:100DF00040400E21C0F202001DF086F84DF6C0639F
:100E0000C2F200030A22197C204600231DF0A2FF33
:100E100045F250400121C0F202001DF075F8204655
:100E20001DF086FF002038BD45F2544008B518215A
:100E3000C0F202001DF068F841F67863C2F20103C7
:100E4000FE21986C03681B68984745F220300F21FB
:100E5000C0F202001DF058F841F2C050C2F2010089
:100E60004FF60F6119F0A4FB45F2E020C0F202003A
:100E700014211DF049F84EF24020C2F20000BDE8F6
:100E800008401DF055BF00BF45F2704008B50F2166
:100E9000C0F202001DF038F841F67863C2F2010397
:100EA000FC21986C03681B68984745F220300F219D
:100EB000C0F202001DF028F841F2C050C2F2010059
:100EC0004FF60F4119F074FB45F2E020C0F202002A
:100ED00014211DF019F84EF24020C2F20000BDE8C6
:100EE00008401DF025BF00BF45F2804008B51B211A
:100EF000C0F202001DF008F841F67863C2F2010367
:100F0000F621986C0368DB6C984745F220300F217E
:100F1000C0F202001CF0F8FF4FF20F601CF06AF9FB
:100F200045F2F820C0F202000F211CF0EDFF4EF256
:100F30004020C2F20000BDE808401DF0F9BE00BF2D
:100F400045F29C4008B51021C0F202001CF0DCFF05
:100F500041F67863C2F20103FA21986C03681B68BA
:100F6000984745F220300F21C0F202001CF0CCFF60
:100F700041F2C050C2F201004FF60F2119F018FBE8
:100F800045F2E020C0F2020014211CF0BDFF4EF239
:100F90004020C2F20000BDE808401DF0C9BE00BFFD
:100FA00045F2B04008B51321C0F202001CF0ACFFBE
:100FB00041F67863C2F20103FB21986C03681B6859
:100FC000984745F220300F21C0F202001CF09CFF30
:100FD00041F2C050C2F201004FF60F3119F0E8FAA9
:100FE00045F2E020C0F2020014211CF08DFF4EF209
:100FF0004020C2F20000BDE808401DF099BE00BFCD
:1010000038B545F284304EF2402541F2905410211B
:10101000C2F20104C2F20005C0F202001CF074FF2B
:1010200028461DF085FE20680EF01EFD20680EF09B
:1010300027FC20680EF038FC45F2C4401621C0F2AF
:1010400002001CF061FF41F2C050C2F201004FF6F5
:101050000F7119F0ADFA45F2E0201421C0F2020040
:101060001CF052FF4FF60F701CF0C4F845F2F82048
:10107000C0F202000F211CF047FF2846BDE83840AF
:101080001DF056BE10B5044645F2DC401F21C0F2EB
:10109000020004F00F041CF037FF44F010044FF27C
:1010A000021343EA044441F2C0502146C2F2010057
:1010B00019F07EFA45F2E0201421C0F202001CF083
:1010C00023FF20461CF096F845F2F820C0F20200FB
:1010D0000F211CF019FF4EF24020C2F20000BDE8C3
:1010E00010401DF025BE00BF45F2FC4008B516219A
:1010F000C0F202001CF008FF41F67863C2F201035F
:10110000F621986C0368DB6C984745F220300F217C
:10111000C0F202001CF0F8FE41F2C050C2F2010021
:101120004FF20F6119F044FA45F2E020C0F20200DC
:1011300014211CF0E9FE4EF24020C2F20000BDE88E
:1011400008401DF0F5BD00BF38B545F284304EF2C1
:10115000402541F290541021C2F20104C2F2000570
:10116000C0F202001CF0D0FE28461DF0E1FD206810
:101170000EF07AFC20680EF083FB20680EF094FBE2
:1011800045F214501621C0F202001CF0BDFE41F6DB
:101190007863C2F20103FF21986C03681B689847CB
:1011A00045F220300F21C0F202001CF0ADFE41F2EA
:1011B000C050C2F201004FF60F7119F0F9F945F273
:1011C000E020C0F2020014211CF09EFE2846BDE87B
:1011D00038401DF0ADBD00BFF8B5064645F22C50B5
:1011E0000C46C0F20200122115461CF08DFE711E45
:1011F000C9B20F2915D841F67867C2F2010741F04C
:10120000A001B86C03681B689847B86C036804F0C9
:101210007F011B689847B86C036805F07F011B6865
:10122000984745F240500A21C0F202001CF06CFEC3
:101230006B1E1B02240404F4FE0403F470632343B6
:10124000310143F4504343F00D03C9B241F2C050A1
:101250001943C2F2010019F0ABF945F2E020C0F2E7
:10126000020014211CF050FE4EF24020C2F2000099
:10127000BDE8F8401DF05CBDF8B54DF6C063C2F2A4
:1012800000030E461B7C1446054623B1984202D04B
:10129000FFF79AFD38B141F29053C2F20103314693
:1012A00018680EF0B7F945F24C501221013DC0F21A
:1012B00002001CF029FEE9B20F2915D841F6786723
:1012C000C2F2010741F08001B86C03681B689847BF
:1012D000B86C036806F07F011B689847B86C036818
:1012E00004F07F011B68984745F220300F21C0F2BF
:1012F00002001CF009FE230603F0FE43310443F410
:10130000004301F4FE012D0243F008030B4341F2B8
:10131000C05005F470611943C2F2010019F048F998
:1013200045F2E020C0F2020014211CF0EDFD4EF267
:101330004020C2F20000BDE8F8401DF0F9BC00BF3B
:101340001F2970B50C46054608D84DF6C063C2F299
:10135000000318790FF070FB0BF0DAF845F26050DB
:101360000D21013DC0F202001CF0CEFDE9B20F29B3
:101370000FD841F67866C2F2010641F0C001B06CA8
:1013800003681B689847B06C036804F07F011B6812
:10139000984745F220300F21C0F202001CF0B4FD46
:1013A000230403F4FE03290243F4404343F00C03F7
:1013B00001F4706141F2C0501943C2F2010019F00A
:1013C000F7F845F2E020C0F2020014211CF09CFD69
:1013D0004EF24020C2F20000BDE870401DF0A8BCF3
:1013E000F8B54DF6C063C2F200030E461B7C1446EE
:1013F000054623B1984202D0FFF7E6FC40B141F226
:101400009053C2F201032246186831460DF0C2FE25
:1014100045F270501121013DC0F202001CF074FD34
:10142000E9B20F2915D841F67867C2F2010741F0F9
:101430009001B86C03681B689847B86C036806F0A5
:101440007F011B689847B86C036804F07F011B6834
:10145000984745F220300F21C0F202001CF054FDE5
:10146000230603F0FE43310443F4104301F4FE016C
:101470002D0243F009030B4341F2C05005F47061A3
:101480001943C2F2010019F093F845F2E020C0F2CE
:10149000020014211CF038FD4EF24020C2F2000080
:1014A000BDE8F8401DF044BCF8B541F29053C2F2DB
:1014B000010305461B6801F5005645F284500C46B1
:1014C000013D0D21C3F8C060C0F202001CF01CFDFC
:1014D000E9B20F2915D841F67867C2F2010741F049
:1014E000E001B86C03681B689847B86C036806F0A5
:1014F0007F011B689847B86C0368C6F3C6111B6868
:10150000984745F2203004F30D040F2104F50054F0
:10151000C0F202001CF0F8FC2902230403F4FE03CD
:1015200001F47061194341F46041640404F0FE4425
:1015300041F00E0141F2C0502143C2F2010019F006
:1015400037F845F2E020C0F2020014211CF0DCFC68
:101550004EF24020C2F20000BDE8F8401DF0E8BBAA
:10156000F0B54AF28C62C2F2010283B040F27063BD
:1015700011680091C2F2010300991E68126801927D
:1015800041F28855C2F2010541F25452C2F2010201
:10159000891B45F294504EF24024C2F20004019F90
:1015A000298000260C21C0F2020016701F601CF07A
:1015B000ABFC2B8820464EF6602191FBF3F11DF029
:1015C00059FB45F2A4500521C0F202001CF09CFC1E
:1015D000298820461DF04EFB45F2AC500F21C0F289
:1015E00002001CF091FC20461DF0A2FB03B0F0BDF0
:1015F00008B541F25451C2F201014AF6AB230A7810
:101600000132D2B2CAF6AA23A3FB02031B0903EBE1
:101610004303A2EBC30313F0FF0F0A7001D1FFF7DE
:101620009FFF45F2BC501021C0F202001CF06CFC80
:1016300041F2C050C2F201004FF60F0118F0B8FF9E
:1016400045F2E0201421C0F202001CF05DFC4FF6D0
:101650000F001BF0CFFD45F2F820C0F202000F2171
:101660001CF052FC4EF24020C2F20000BDE80840DF
:101670001DF05EBB08B541F25451C2F201014AF6B9
:10168000AB230A780132D2B2CAF6AA23A3FB020323
:101690001B0903EB4303A2EBC30313F0FF0F0A7014
:1016A00001D1FFF75DFF45F2D0501521C0F20200D5
:1016B0001CF02AFC41F67863C2F20103F821986C11
:1016C00003681B68984745F220300F21C0F20200E2
:1016D0001CF01AFC4FF60F001BF08CFD45F2F820B1
:1016E000C0F202000F211CF00FFC4EF24020C2F2AB
:1016F0000000BDE808401DF01BBB00BF08B541F26B
:101700005451C2F201014AF6AB230A780132D2B237
:10171000CAF6AA23A3FB02031B0903EB4303A2EBB4
:10172000C30313F0FF0F0A7001D1FFF719FF45F251
:10173000E8501021C0F202001CF0E6FB41F678638D
:10174000C2F20103F821986C03681B68984745F2C0
:1017500020300F21C0F202001CF0D6FB41F2C05035
:10176000C2F201004FF60F0118F022FF45F2E0200F
:10177000C0F2020014211CF0C7FB4EF24020C2F25E
:101780000000BDE808401DF0D3BA00BF1F2970B5A6
:101790000C46054608D84DF6C063C2F2000318791E
:1017A0000FF04AF90AF0B4FE45F2FC501221013D57
:1017B000C0F202001CF0A8FBE9B20F290FD841F6D5
:1017C0007866C2F2010641F0C001B06C03681B6884
:1017D0009847B06C036804F07F011B68984745F296
:1017E00020300F21C0F202001CF08EFB230403F412
:1017F000FE03280243F4404343F00C0300F47060FE
:1018000018431BF0F7FC45F2F820C0F202000F214C
:101810001CF07AFB4EF24020C2F20000BDE870409E
:101820001DF086BA70B5064645F210600C46C0F24F
:101830000200172115461CF067FB711EC9B20F2963
:101840002BD841F67866C2F2010641F0A001B06CD7
:1018500003681B689847B06C036804F07F011B683D
:101860009847B06C036805F07F011B68984745F204
:101870004050C0F202000A211CF046FB45F2F8205D
:10188000C0F202000F211CF03FFB4EF24020C2F2DA
:101890000000BDE870401DF04BBA45F24050C0F268
:1018A00002000A211CF030FB002EE7D1681E000266
:1018B000240404F4FE0400F47060204340F450401B
:1018C00040F00D001BF096FCD8E700BF1F2938B58B
:1018D0000C46054608D84DF6C063C2F200031879DD
:1018E0000FF0AAF80AF014FE240404F4FE04013DEB
:1018F00045F2286044F440442D020D2105F4706542
:10190000C0F2020044F00C041CF0FEFA2C4341F239
:10191000C0502146C2F2010018F04AFE45F2E02014
:101920001421C0F202001CF0EFFA20461BF062FC0A
:1019300045F2F820C0F202000F211CF0E5FA4EF249
:101940004020C2F20000BDE838401DF0F1B900BFF0
:1019500070B5064645F2386015460C46C0F20200E6
:1019600012211CF0D1FA6B1E1B02240404F4FE04A5
:1019700003F47063234343F45043340143F00D03F5
:10198000E4B21C4341F2C0502146C2F2010018F0FB
:101990000FFE45F2E020C0F2020014211CF0B4FA60
:1019A00016B920461BF026FC45F2F820C0F20200D2
:1019B0000F211CF0A9FA4EF24020C2F20000BDE84F
:1019C00070401DF0B5B900BFF8B54DF6C063C2F266
:1019D00000030E461B7C1446054623B1984202D0F4
:1019E000FFF7F2F938B141F29053C2F201033146E8
:1019F00018680DF00FFE45F24C601721013DC0F252
:101A000002001CF081FAE9B20F2915D841F6786777
:101A1000C2F2010741F08001B86C03681B68984767
:101A2000B86C036806F07F011B689847B86C0368C0
:101A300004F07F011B68984745F220300F21C0F267
:101A400002001CF061FA230603F0FE43310443F464
:101A5000004301F4FE01280243F008030B4300F4A5
:101A6000706018431BF0C6FB45F2F820C0F202007C
:101A70000F211CF049FA4EF24020C2F20000BDE8EE
:101A8000F8401DF055B900BF38B541F678650446F9
:101A9000C2F2010545F264601A21C0F202001CF096
:101AA00033FAA86C0368F3211B689847A86C036895
:101AB00004F07F01DB6C984745F220300F21C0F223
:101AC00002001CF021FA200400F4FE0040F47340F0
:101AD00040F002001BF08EFB45F2F820C0F202003D
:101AE0000F211CF011FA4EF24020C2F20000BDE8B6
:101AF00038401DF01DB900BFF8B54DF6C063C2F205
:101B000000030E461B7C1446054623B1984202D0C2
:101B1000FFF75AF940B141F29053C2F20103224655
:101B2000186831460DF036FB45F280601621013D04
:101B3000C0F202001CF0E8F9E9B20F2915D841F60D
:101B40007867C2F2010741F09001B86C03681B6826
:101B50009847B86C036806F07F011B689847B86C1B
:101B6000036804F07F011B68984745F220300F217D
:101B7000C0F202001CF0C8F9230603F0FE43310452
:101B800043F4104301F4FE01280243F009030B4320
:101B900000F4706018431BF02DFB45F2F820C0F2F2
:101BA00002000F211CF0B0F94EF24020C2F20000FA
:101BB000BDE8F8401DF0BCB838B541F6786504467C
:101BC000C2F2010545F298602421C0F202001CF027
:101BD0009BF9A86C0368F1211B689847A86C0368FF
:101BE00021461B68984745F220300F21C0F20200C1
:101BF00004F00F041CF088F944F010044FF20210B6
:101C000040EA04401BF0F6FA45F2F820C0F2020068
:101C10000F211CF079F94EF24020C2F20000BDE81D
:101C200038401DF085B800BF70B54DF6C063C2F2F4
:101C300000030E461B7C1446054623B1984202D091
:101C4000FFF7C2F840B141F29053C2F201032246BD
:101C5000186831460DF09EFA45F2C0601121C0F2BD
:101C600002001CF051F9230603F0FE43340443F450
:101C70001043013D43F0090304F4FE042D021C430C
:101C800005F470652C4341F2C0502146C2F20100B8
:101C900018F08EFC45F2E0201421C0F202001CF086
:101CA00033F920461BF0A6FA45F2F820C0F20200F4
:101CB0000F211CF029F94EF24020C2F20000BDE8CD
:101CC00070401DF035B800BF70B54DF6C063C2F26C
:101CD00000030E461B7C1446054623B1984202D0F1
:101CE000FFF772F838B141F29053C2F20103314666
:101CF00018680DF08FFC45F2D4601221C0F202008A
:101D00001CF002F9230603F0FE43340443F40043BD
:101D1000013D43F0080304F4FE042D021C4305F4C6
:101D200070652C4341F2C0502146C2F2010018F008
:101D30003FFC45F2E0201421C0F202001CF0E4F860
:101D400020461BF057FA45F2F820C0F202000F219E
:101D50001CF0DAF84EF24020C2F20000BDE87040FC
:101D60001CF0E6BF38B541F678650446C2F20105BD
:101D700045F2E8601521C0F202001CF0C5F8A86C1D
:101D80000368F3211B689847A86C036804F07F017F
:101D9000DB6C984745F220300F21C0F202001CF0A6
:101DA000B3F8210401F4FE0141F4734141F2C05043
:101DB00041F00201C2F2010018F0FAFB45F2E02006
:101DC000C0F2020014211CF09FF84EF24020C2F233
:101DD0000000BDE838401CF0ABBF00BF38B541F68D
:101DE00078650446C2F2010545F200701F21C0F279
:101DF00002001CF089F8A86C0368F1211B68984761
:101E0000A86C036821461B68984745F220300F21D3
:101E1000C0F2020004F00F041CF076F844F0100445
:101E20004FF2021141F2C05041EA0441C2F20100F6
:101E300018F0BEFB45F2E020C0F2020014211CF0B5
:101E400063F84EF24020C2F20000BDE838401CF0BA
:101E50006FBF00BF38B541F29053C2F2010301F5E4
:101E600000521B6805460C4645F22070C3F8C0209E
:101E70000D2104F30D04C0F202001CF045F804F536
:101E800000536C1E1A04240202F4FE0204F470646F
:101E9000144344F460445B0403F0FE4344F00E0436
:101EA0001C4341F2C0502146C2F2010018F080FBF1
:101EB00045F2E0201421C0F202001CF025F8204673
:101EC0001BF098F945F2F820C0F202000F211CF037
:101ED0001BF84EF24020C2F20000BDE838401CF072
:101EE00027BF00BFF8B541F29053C2F20103054687
:101EF0001B6801F5005645F230700C46013D122179
:101F0000C3F8C060C0F202001BF0FEFFE9B20F2967
:101F100015D841F67867C2F2010741F0E001B86CCC
:101F200003681B689847B86C036806F07F011B685C
:101F30009847B86C0368C6F3C6111B68984745F20A
:101F4000203004F30D040F2104F50054C0F2020008
:101F50001BF0DAFF2802230403F4FE0300F4706090
:101F6000184340F46040640404F0FE4440F00E0066
:101F700020431BF03FF945F2F820C0F202000F2188
:101F80001BF0C2FF4EF24020C2F20000BDE8F84054
:101F90001CF0CEBE4AF28853C2F2010310B4D3F84B
:101FA000C8201368506819780478507A137A04426C
:101FB00001EA03011AD0937A03F0030309B143F055
:101FC000040343F008039910082B91722AD8072BB9
:101FD00022D2032B2ED011D9042B13D0062B14D1CF
:101FE000D3685DF8044B023BD3607047937A03F0EB
:101FF00003030029E7D043F00403E4E7012B0BD0EF
:10200000022B02D1D368013BD3605DF8044B7047CB
:102010000D2BF7D00E2BF8D1D3685DF8044B0133AC
:10202000D36070470C2B05D0F2D8092BD8D00B2BDE
:10203000E8D0EAE7D3685DF8044B0233D360704719
:102040004AF28853C2F2010310B4D3F8CC201368CB
:10205000506819780478507A137A044201EA03012F
:102060001AD0937A03F0030309B143F0040343F059
:1020700008039910082B91722AD8072B22D2032B20
:102080002ED011D9042B13D0062B14D1D3685DF8B0
:10209000044B023BD3607047937A03F0030300299B
:1020A000E7D043F00403E4E7012B0BD0022B02D16D
:1020B000D368013BD3605DF8044B70470D2BF7D01C
:1020C0000E2BF8D1D3685DF8044B0133D360704711
:1020D0000C2B05D0F2D8092BD8D00B2BE8D0EAE78F
:1020E000D3685DF8044B0233D36070474AF28853DB
:1020F000C2F2010310B4D3F8D020136850681978E5
:102100000478507A137A044201EA03011AD0937AD0
:1021100003F0030309B143F0040343F008039910EB
:10212000082B91722AD8072B22D2032B2ED011D93B
:10213000042B13D0062B14D1D3685DF8044B023B5B
:10214000D3607047937A03F003030029E7D043F08C
:102150000403E4E7012B0BD0022B02D1D368013B2F
:10216000D3605DF8044B70470D2BF7D00E2BF8D1E0
:10217000D3685DF8044B0133D36070470C2B05D056
:10218000F2D8092BD8D00B2BE8D0EAE7D3685DF85A
:10219000044B0233D36070474AF28853C2F2010302
:1021A00010B4D3F8D4201368506819780478507AA2
:1021B000137A044201EA03011AD0937A03F003036D
:1021C00009B143F0040343F008039910082B9172FE
:1021D0002AD8072B22D2032B2ED011D9042B13D0AF
:1021E000062B14D1D3685DF8044B023BD3607047D3
:1021F000937A03F003030029E7D043F00403E4E7F4
:10220000012B0BD0022B02D1D368013BD3605DF8C8
:10221000044B70470D2BF7D00E2BF8D1D3685DF827
:10222000044B0133D36070470C2B05D0F2D8092B37
:10223000D8D00B2BE8D0EAE7D3685DF8044B023323
:10224000D36070474AF28853C2F2010310B4D3F846
:10225000D8201368506819780478507A137A0442A9
:1022600001EA03011AD0937A03F0030309B143F0A2
:10227000040343F008039910082B91722AD8072B06
:1022800022D2032B2ED011D9042B13D0062B14D11C
:10229000D3685DF8044B023BD3607047937A03F038
:1022A00003030029E7D043F00403E4E7012B0BD03C
:1022B000022B02D1D368013BD3605DF8044B704719
:1022C0000D2BF7D00E2BF8D1D3685DF8044B0133FA
:1022D000D36070470C2B05D0F2D8092BD8D00B2B2C
:1022E000E8D0EAE7D3685DF8044B0233D360704767
:1022F0004AF28853C2F2010310B4D3F8DC20136809
:10230000506819780478507A137A044201EA03017C
:102310001AD0937A03F0030309B143F0040343F0A6
:1023200008039910082B91722AD8072B22D2032B6D
:102330002ED011D9042B13D0062B14D1D3685DF8FD
:10234000044B023BD3607047937A03F003030029E8
:10235000E7D043F00403E4E7012B0BD0022B02D1BA
:10236000D368013BD3605DF8044B70470D2BF7D069
:102370000E2BF8D1D3685DF8044B0133D36070475E
:102380000C2B05D0F2D8092BD8D00B2BE8D0EAE7DC
:10239000D3685DF8044B0233D36070474AF2885328
:1023A000C2F2010310B4D3F8E02013685068197822
:1023B0000478507A137A044201EA03011AD0937A1E
:1023C00003F0030309B143F0040343F00803991039
:1023D000082B91722AD8072B22D2032B2ED011D989
:1023E000042B13D0062B14D1D3685DF8044B023BA9
:1023F000D3607047937A03F003030029E7D043F0DA
:102400000403E4E7012B0BD0022B02D1D368013B7C
:10241000D3605DF8044B70470D2BF7D00E2BF8D12D
:10242000D3685DF8044B0133D36070470C2B05D0A3
:10243000F2D8092BD8D00B2BE8D0EAE7D3685DF8A7
:10244000044B0233D36070474AF28853C2F201034F
:1024500010B4D3F8E4201368506819780478507ADF
:10246000137A044201EA03011AD0937A03F00303BA
:1024700009B143F0040343F008039910082B91724B
:102480002AD8072B22D2032B2ED011D9042B13D0FC
:10249000062B14D1D3685DF8044B023BD360704720
:1024A000937A03F003030029E7D043F00403E4E741
:1024B000012B0BD0022B02D1D368013BD3605DF816
:1024C000044B70470D2BF7D00E2BF8D1D3685DF875
:1024D000044B0133D36070470C2B05D0F2D8092B85
:1024E000D8D00B2BE8D0EAE7D3685DF8044B023371
:1024F000D36070474AF28853C2F2010310B4D3F894
:1025000088201368506819780478507A137A044246
:1025100001EA03011AD0937A03F0030309B143F0EF
:10252000040343F008039910082B91722AD8072B53
:1025300022D2032B2ED011D9042B13D0062B14D169
:10254000D3685DF8044B023BD3607047937A03F085
:1025500003030029E7D043F00403E4E7012B0BD089
:10256000022B02D1D368013BD3605DF8044B704766
:102570000D2BF7D00E2BF8D1D3685DF8044B013347
:10258000D36070470C2B05D0F2D8092BD8D00B2B79
:10259000E8D0EAE7D3685DF8044B0233D3607047B4
:1025A0004AF28853C2F2010310B4D3F88C201368A6
:1025B000506819780478507A137A044201EA0301CA
:1025C0001AD0937A03F0030309B143F0040343F0F4
:1025D00008039910082B91722AD8072B22D2032BBB
:1025E0002ED011D9042B13D0062B14D1D3685DF84B
:1025F000044B023BD3607047937A03F00303002936
:10260000E7D043F00403E4E7012B0BD0022B02D107
:10261000D368013BD3605DF8044B70470D2BF7D0B6
:102620000E2BF8D1D3685DF8044B0133D3607047AB
:102630000C2B05D0F2D8092BD8D00B2BE8D0EAE729
:10264000D3685DF8044B0233D36070474AF2885375
:10265000C2F2010310B4D3F89020136850681978BF
:102660000478507A137A044201EA03011AD0937A6B
:1026700003F0030309B143F0040343F00803991086
:10268000082B91722AD8072B22D2032B2ED011D9D6
:10269000042B13D0062B14D1D3685DF8044B023BF6
:1026A000D3607047937A03F003030029E7D043F027
:1026B0000403E4E7012B0BD0022B02D1D368013BCA
:1026C000D3605DF8044B70470D2BF7D00E2BF8D17B
:1026D000D3685DF8044B0133D36070470C2B05D0F1
:1026E000F2D8092BD8D00B2BE8D0EAE7D3685DF8F5
:1026F000044B0233D36070474AF28853C2F201039D
:1027000010B4D3F894201368506819780478507A7C
:10271000137A044201EA03011AD0937A03F0030307
:1027200009B143F0040343F008039910082B917298
:102730002AD8072B22D2032B2ED011D9042B13D049
:10274000062B14D1D3685DF8044B023BD36070476D
:10275000937A03F003030029E7D043F00403E4E78E
:10276000012B0BD0022B02D1D368013BD3605DF863
:10277000044B70470D2BF7D00E2BF8D1D3685DF8C2
:10278000044B0133D36070470C2B05D0F2D8092BD2
:10279000D8D00B2BE8D0EAE7D3685DF8044B0233BE
:1027A000D36070474AF28853C2F2010310B4D3F8E1
:1027B00098201368506819780478507A137A044284
:1027C00001EA03011AD0937A03F0030309B143F03D
:1027D000040343F008039910082B91722AD8072BA1
:1027E00022D2032B2ED011D9042B13D0062B14D1B7
:1027F000D3685DF8044B023BD3607047937A03F0D3
:1028000003030029E7D043F00403E4E7012B0BD0D6
:10281000022B02D1D368013BD3605DF8044B7047B3
:102820000D2BF7D00E2BF8D1D3685DF8044B013394
:10283000D36070470C2B05D0F2D8092BD8D00B2BC6
:10284000E8D0EAE7D3685DF8044B0233D360704701
:102850004AF28853C2F2010310B4D3F89C201368E3
:10286000506819780478507A137A044201EA030117
:102870001AD0937A03F0030309B143F0040343F041
:1028800008039910082B91722AD8072B22D2032B08
:102890002ED011D9042B13D0062B14D1D3685DF898
:1028A000044B023BD3607047937A03F00303002983
:1028B000E7D043F00403E4E7012B0BD0022B02D155
:1028C000D368013BD3605DF8044B70470D2BF7D004
:1028D0000E2BF8D1D3685DF8044B0133D3607047F9
:1028E0000C2B05D0F2D8092BD8D00B2BE8D0EAE777
:1028F000D3685DF8044B0233D36070474AF28853C3
:10290000C2F2010310B4D3F8A020136850681978FC
:102910000478507A137A044201EA03011AD0937AB8
:1029200003F0030309B143F0040343F008039910D3
:10293000082B91722AD8072B22D2032B2ED011D923
:10294000042B13D0062B14D1D3685DF8044B023B43
:10295000D3607047937A03F003030029E7D043F074
:102960000403E4E7012B0BD0022B02D1D368013B17
:10297000D3605DF8044B70470D2BF7D00E2BF8D1C8
:10298000D3685DF8044B0133D36070470C2B05D03E
:10299000F2D8092BD8D00B2BE8D0EAE7D3685DF842
:1029A000044B0233D36070474AF28853C2F20103EA
:1029B00010B4D3F8A4201368506819780478507ABA
:1029C000137A044201EA03011AD0937A03F0030355
:1029D00009B143F0040343F008039910082B9172E6
:1029E0002AD8072B22D2032B2ED011D9042B13D097
:1029F000062B14D1D3685DF8044B023BD3607047BB
:102A0000937A03F003030029E7D043F00403E4E7DB
:102A1000012B0BD0022B02D1D368013BD3605DF8B0
:102A2000044B70470D2BF7D00E2BF8D1D3685DF80F
:102A3000044B0133D36070470C2B05D0F2D8092B1F
:102A4000D8D00B2BE8D0EAE7D3685DF8044B02330B
:102A5000D36070474AF28853C2F2010310B4D3F82E
:102A6000A8201368506819780478507A137A0442C1
:102A700001EA03011AD0937A03F0030309B143F08A
:102A8000040343F008039910082B91722AD8072BEE
:102A900022D2032B2ED011D9042B13D0062B14D104
:102AA000D3685DF8044B023BD3607047937A03F020
:102AB00003030029E7D043F00403E4E7012B0BD024
:102AC000022B02D1D368013BD3605DF8044B704701
:102AD0000D2BF7D00E2BF8D1D3685DF8044B0133E2
:102AE000D36070470C2B05D0F2D8092BD8D00B2B14
:102AF000E8D0EAE7D3685DF8044B0233D36070474F
:102B00004AF28853C2F2010310B4D3F8AC20136820
:102B1000506819780478507A137A044201EA030164
:102B20001AD0937A03F0030309B143F0040343F08E
:102B300008039910082B91722AD8072B22D2032B55
:102B40002ED011D9042B13D0062B14D1D3685DF8E5
:102B5000044B023BD3607047937A03F003030029D0
:102B6000E7D043F00403E4E7012B0BD0022B02D1A2
:102B7000D368013BD3605DF8044B70470D2BF7D051
:102B80000E2BF8D1D3685DF8044B0133D360704746
:102B90000C2B05D0F2D8092BD8D00B2BE8D0EAE7C4
:102BA000D3685DF8044B0233D36070474AF2885310
:102BB000C2F2010310B4D3F8B0201368506819783A
:102BC0000478507A137A044201EA03011AD0937A06
:102BD00003F0030309B143F0040343F00803991021
:102BE000082B91722AD8072B22D2032B2ED011D971
:102BF000042B13D0062B14D1D3685DF8044B023B91
:102C0000D3607047937A03F003030029E7D043F0C1
:102C10000403E4E7012B0BD0022B02D1D368013B64
:102C2000D3605DF8044B70470D2BF7D00E2BF8D115
:102C3000D3685DF8044B0133D36070470C2B05D08B
:102C4000F2D8092BD8D00B2BE8D0EAE7D3685DF88F
:102C5000044B0233D36070474AF28853C2F2010337
:102C600010B4D3F8B4201368506819780478507AF7
:102C7000137A044201EA03011AD0937A03F00303A2
:102C800009B143F0040343F008039910082B917233
:102C90002AD8072B22D2032B2ED011D9042B13D0E4
:102CA000062B14D1D3685DF8044B023BD360704708
:102CB000937A03F003030029E7D043F00403E4E729
:102CC000012B0BD0022B02D1D368013BD3605DF8FE
:102CD000044B70470D2BF7D00E2BF8D1D3685DF85D
:102CE000044B0133D36070470C2B05D0F2D8092B6D
:102CF000D8D00B2BE8D0EAE7D3685DF8044B023359
:102D0000D36070474AF28853C2F2010310B4D3F87B
:102D1000B8201368506819780478507A137A0442FE
:102D200001EA03011AD0937A03F0030309B143F0D7
:102D3000040343F008039910082B91722AD8072B3B
:102D400022D2032B2ED011D9042B13D0062B14D151
:102D5000D3685DF8044B023BD3607047937A03F06D
:102D600003030029E7D043F00403E4E7012B0BD071
:102D7000022B02D1D368013BD3605DF8044B70474E
:102D80000D2BF7D00E2BF8D1D3685DF8044B01332F
:102D9000D36070470C2B05D0F2D8092BD8D00B2B61
:102DA000E8D0EAE7D3685DF8044B0233D36070479C
:102DB0004AF28853C2F2010310B4D3F8BC2013685E
:102DC000506819780478507A137A044201EA0301B2
:102DD0001AD0937A03F0030309B143F0040343F0DC
:102DE00008039910082B91722AD8072B22D2032BA3
:102DF0002ED011D9042B13D0062B14D1D3685DF833
:102E0000044B023BD3607047937A03F0030300291D
:102E1000E7D043F00403E4E7012B0BD0022B02D1EF
:102E2000D368013BD3605DF8044B70470D2BF7D09E
:102E30000E2BF8D1D3685DF8044B0133D360704793
:102E40000C2B05D0F2D8092BD8D00B2BE8D0EAE711
:102E5000D3685DF8044B0233D36070474AF288535D
:102E6000C2F2010310B4D3F8C02013685068197877
:102E70000478507A137A044201EA03011AD0937A53
:102E800003F0030309B143F0040343F0080399106E
:102E9000082B91722AD8072B22D2032B2ED011D9BE
:102EA000042B13D0062B14D1D3685DF8044B023BDE
:102EB000D3607047937A03F003030029E7D043F00F
:102EC0000403E4E7012B0BD0022B02D1D368013BB2
:102ED000D3605DF8044B70470D2BF7D00E2BF8D163
:102EE000D3685DF8044B0133D36070470C2B05D0D9
:102EF000F2D8092BD8D00B2BE8D0EAE7D3685DF8DD
:102F0000044B0233D36070474AF28853C2F2010384
:102F100010B4D3F8C4201368506819780478507A34
:102F2000137A044201EA03011AD0937A03F00303EF
:102F300009B143F0040343F008039910082B917280
:102F40002AD8072B22D2032B2ED011D9042B13D031
:102F5000062B14D1D3685DF8044B023BD360704755
:102F6000937A03F003030029E7D043F00403E4E776
:102F7000012B0BD0022B02D1D368013BD3605DF84B
:102F8000044B70470D2BF7D00E2BF8D1D3685DF8AA
:102F9000044B0133D36070470C2B05D0F2D8092BBA
:102FA000D8D00B2BE8D0EAE7D3685DF8044B0233A6
:102FB000D36070474AF28853C2F2010310B49A6892
:102FC0001368506819780478507A137A044201EA39
:102FD00003011AD0937A03F0030309B143F0040309
:102FE00043F008039910082B91722AD8072B22D29C
:102FF000032B2ED011D9042B13D0062B14D1D36858
:103000005DF8044B023BD3607047937A03F00303EF
:103010000029E7D043F00403E4E7012B0BD0022B97
:1030200002D1D368013BD3605DF8044B70470D2B90
:10303000F7D00E2BF8D1D3685DF8044B0133D36081
:1030400070470C2B05D0F2D8092BD8D00B2BE8D029
:10305000EAE7D3685DF8044B0233D360704700BFE2
:103060004AF28853C2F2010310B4DA681368506858
:1030700019780478507A137A044201EA03011AD0CD
:10308000937A03F0030309B143F0040343F0080308
:103090009910082B91722AD8072B22D2032B2ED0FD
:1030A00011D9042B13D0062B14D1D3685DF8044B2F
:1030B000023BD3607047937A03F003030029E7D003
:1030C00043F00403E4E7012B0BD0022B02D1D368B9
:1030D000013BD3605DF8044B70470D2BF7D00E2BEE
:1030E000F8D1D3685DF8044B0133D36070470C2BE3
:1030F00005D0F2D8092BD8D00B2BE8D0EAE7D3685B
:103100005DF8044B0233D360704700BF4AF2885326
:10311000C2F2010310B41A69136850681978047870
:10312000507A137A044201EA03011AD0937A03F029
:10313000030309B143F0040343F008039910082B7B
:1031400091722AD8072B22D2032B2ED011D9042B0F
:1031500013D0062B14D1D3685DF8044B023BD36027
:103160007047937A03F003030029E7D043F0040388
:10317000E4E7012B0BD0022B02D1D368013BD360D3
:103180005DF8044B70470D2BF7D00E2BF8D1D368A8
:103190005DF8044B0133D36070470C2B05D0F2D897
:1031A000092BD8D00B2BE8D0EAE7D3685DF8044BA5
:1031B0000233D360704700BF4AF28853C2F2010362
:1031C00010B45A691368506819780478507A137AE1
:1031D000044201EA03011AD0937A03F0030309B110
:1031E00043F0040343F008039910082B91722AD886
:1031F000072B22D2032B2ED011D9042B13D0062B50
:1032000014D1D3685DF8044B023BD3607047937AC6
:1032100003F003030029E7D043F00403E4E7012BA4
:103220000BD0022B02D1D368013BD3605DF8044B75
:1032300070470D2BF7D00E2BF8D1D3685DF8044BF7
:103240000133D36070470C2B05D0F2D8092BD8D0AE
:103250000B2BE8D0EAE7D3685DF8044B0233D36068
:10326000704700BF4AF28853C2F2010310B49A6952
:103270001368506819780478507A137A044201EA86
:1032800003011AD0937A03F0030309B143F0040356
:1032900043F008039910082B91722AD8072B22D2E9
:1032A000032B2ED011D9042B13D0062B14D1D368A5
:1032B0005DF8044B023BD3607047937A03F003033D
:1032C0000029E7D043F00403E4E7012B0BD0022BE5
:1032D00002D1D368013BD3605DF8044B70470D2BDE
:1032E000F7D00E2BF8D1D3685DF8044B0133D360CF
:1032F00070470C2B05D0F2D8092BD8D00B2BE8D077
:10330000EAE7D3685DF8044B0233D360704700BF2F
:103310004AF28853C2F2010310B4DA6913685068A4
:1033200019780478507A137A044201EA03011AD01A
:10333000937A03F0030309B143F0040343F0080355
:103340009910082B91722AD8072B22D2032B2ED04A
:1033500011D9042B13D0062B14D1D3685DF8044B7C
:10336000023BD3607047937A03F003030029E7D050
:1033700043F00403E4E7012B0BD0022B02D1D36806
:10338000013BD3605DF8044B70470D2BF7D00E2B3B
:10339000F8D1D3685DF8044B0133D36070470C2B30
:1033A00005D0F2D8092BD8D00B2BE8D0EAE7D368A8
:1033B0005DF8044B0233D360704700BF4AF2885374
:1033C000C2F2010310B41A6A1368506819780478BD
:1033D000507A137A044201EA03011AD0937A03F077
:1033E000030309B143F0040343F008039910082BC9
:1033F00091722AD8072B22D2032B2ED011D9042B5D
:1034000013D0062B14D1D3685DF8044B023BD36074
:103410007047937A03F003030029E7D043F00403D5
:10342000E4E7012B0BD0022B02D1D368013BD36020
:103430005DF8044B70470D2BF7D00E2BF8D1D368F5
:103440005DF8044B0133D36070470C2B05D0F2D8E4
:10345000092BD8D00B2BE8D0EAE7D3685DF8044BF2
:103460000233D360704700BF4AF28853C2F20103AF
:1034700010B45A6A1368506819780478507A137A2D
:10348000044201EA03011AD0937A03F0030309B15D
:1034900043F0040343F008039910082B91722AD8D3
:1034A000072B22D2032B2ED011D9042B13D0062B9D
:1034B00014D1D3685DF8044B023BD3607047937A14
:1034C00003F003030029E7D043F00403E4E7012BF2
:1034D0000BD0022B02D1D368013BD3605DF8044BC3
:1034E00070470D2BF7D00E2BF8D1D3685DF8044B45
:1034F0000133D36070470C2B05D0F2D8092BD8D0FC
:103500000B2BE8D0EAE7D3685DF8044B0233D360B5
:10351000704700BF4AF28853C2F2010310B49A6A9E
:103520001368506819780478507A137A044201EAD3
:1035300003011AD0937A03F0030309B143F00403A3
:1035400043F008039910082B91722AD8072B22D236
:10355000032B2ED011D9042B13D0062B14D1D368F2
:103560005DF8044B023BD3607047937A03F003038A
:103570000029E7D043F00403E4E7012B0BD0022B32
:1035800002D1D368013BD3605DF8044B70470D2B2B
:10359000F7D00E2BF8D1D3685DF8044B0133D3601C
:1035A00070470C2B05D0F2D8092BD8D00B2BE8D0C4
:1035B000EAE7D3685DF8044B0233D360704700BF7D
:1035C0004AF28853C2F2010310B4DA6A13685068F1
:1035D00019780478507A137A044201EA03011AD068
:1035E000937A03F0030309B143F0040343F00803A3
:1035F0009910082B91722AD8072B22D2032B2ED098
:1036000011D9042B13D0062B14D1D3685DF8044BC9
:10361000023BD3607047937A03F003030029E7D09D
:1036200043F00403E4E7012B0BD0022B02D1D36853
:10363000013BD3605DF8044B70470D2BF7D00E2B88
:10364000F8D1D3685DF8044B0133D36070470C2B7D
:1036500005D0F2D8092BD8D00B2BE8D0EAE7D368F5
:103660005DF8044B0233D360704700BF4AF28853C1
:10367000C2F2010310B41A6B136850681978047809
:10368000507A137A044201EA03011AD0937A03F0C4
:10369000030309B143F0040343F008039910082B16
:1036A00091722AD8072B22D2032B2ED011D9042BAA
:1036B00013D0062B14D1D3685DF8044B023BD360C2
:1036C0007047937A03F003030029E7D043F0040323
:1036D000E4E7012B0BD0022B02D1D368013BD3606E
:1036E0005DF8044B70470D2BF7D00E2BF8D1D36843
:1036F0005DF8044B0133D36070470C2B05D0F2D832
:10370000092BD8D00B2BE8D0EAE7D3685DF8044B3F
:103710000233D360704700BF4AF28853C2F20103FC
:1037200010B45A6B1368506819780478507A137A79
:10373000044201EA03011AD0937A03F0030309B1AA
:1037400043F0040343F008039910082B91722AD820
:10375000072B22D2032B2ED011D9042B13D0062BEA
:1037600014D1D3685DF8044B023BD3607047937A61
:1037700003F003030029E7D043F00403E4E7012B3F
:103780000BD0022B02D1D368013BD3605DF8044B10
:1037900070470D2BF7D00E2BF8D1D3685DF8044B92
:1037A0000133D36070470C2B05D0F2D8092BD8D049
:1037B0000B2BE8D0EAE7D3685DF8044B0233D36003
:1037C000704700BF4AF28853C2F2010310B49A6BEB
:1037D0001368506819780478507A137A044201EA21
:1037E00003011AD0937A03F0030309B143F00403F1
:1037F00043F008039910082B91722AD8072B22D284
:10380000032B2ED011D9042B13D0062B14D1D3683F
:103810005DF8044B023BD3607047937A03F00303D7
:103820000029E7D043F00403E4E7012B0BD0022B7F
:1038300002D1D368013BD3605DF8044B70470D2B78
:10384000F7D00E2BF8D1D3685DF8044B0133D36069
:1038500070470C2B05D0F2D8092BD8D00B2BE8D011
:10386000EAE7D3685DF8044B0233D360704700BFCA
:103870004AF28853C2F2010310B4DA6B136850683D
:1038800019780478507A137A044201EA03011AD0B5
:10389000937A03F0030309B143F0040343F00803F0
:1038A0009910082B91722AD8072B22D2032B2ED0E5
:1038B00011D9042B13D0062B14D1D3685DF8044B17
:1038C000023BD3607047937A03F003030029E7D0EB
:1038D00043F00403E4E7012B0BD0022B02D1D368A1
:1038E000013BD3605DF8044B70470D2BF7D00E2BD6
:1038F000F8D1D3685DF8044B0133D36070470C2BCB
:1039000005D0F2D8092BD8D00B2BE8D0EAE7D36842
:103910005DF8044B0233D360704700BF4AF288530E
:10392000C2F2010310B41A6C136850681978047855
:10393000507A137A044201EA03011AD0937A03F011
:10394000030309B143F0040343F008039910082B63
:1039500091722AD8072B22D2032B2ED011D9042BF7
:1039600013D0062B14D1D3685DF8044B023BD3600F
:103970007047937A03F003030029E7D043F0040370
:10398000E4E7012B0BD0022B02D1D368013BD360BB
:103990005DF8044B70470D2BF7D00E2BF8D1D36890
:1039A0005DF8044B0133D36070470C2B05D0F2D87F
:1039B000092BD8D00B2BE8D0EAE7D3685DF8044B8D
:1039C0000233D360704700BF4AF28853C2F201034A
:1039D00010B45A6C1368506819780478507A137AC6
:1039E000044201EA03011AD0937A03F0030309B1F8
:1039F00043F0040343F008039910082B91722AD86E
:103A0000072B22D2032B2ED011D9042B13D0062B37
:103A100014D1D3685DF8044B023BD3607047937AAE
:103A200003F003030029E7D043F00403E4E7012B8C
:103A30000BD0022B02D1D368013BD3605DF8044B5D
:103A400070470D2BF7D00E2BF8D1D3685DF8044BDF
:103A50000133D36070470C2B05D0F2D8092BD8D096
:103A60000B2BE8D0EAE7D3685DF8044B0233D36050
:103A7000704700BF4AF28853C2F2010310B49A6C37
:103A80001368506819780478507A137A044201EA6E
:103A900003011AD0937A03F0030309B143F004033E
:103AA00043F008039910082B91722AD8072B22D2D1
:103AB000032B2ED011D9042B13D0062B14D1D3688D
:103AC0005DF8044B023BD3607047937A03F0030325
:103AD0000029E7D043F00403E4E7012B0BD0022BCD
:103AE00002D1D368013BD3605DF8044B70470D2BC6
:103AF000F7D00E2BF8D1D3685DF8044B0133D360B7
:103B000070470C2B05D0F2D8092BD8D00B2BE8D05E
:103B1000EAE7D3685DF8044B0233D360704700BF17
:103B20004AF28853C2F2010310B4DA6C1368506889
:103B300019780478507A137A044201EA03011AD002
:103B4000937A03F0030309B143F0040343F008033D
:103B50009910082B91722AD8072B22D2032B2ED032
:103B600011D9042B13D0062B14D1D3685DF8044B64
:103B7000023BD3607047937A03F003030029E7D038
:103B800043F00403E4E7012B0BD0022B02D1D368EE
:103B9000013BD3605DF8044B70470D2BF7D00E2B23
:103BA000F8D1D3685DF8044B0133D36070470C2B18
:103BB00005D0F2D8092BD8D00B2BE8D0EAE7D36890
:103BC0005DF8044B0233D360704700BF4AF288535C
:103BD000C2F2010310B41A6D1368506819780478A2
:103BE000507A137A044201EA03011AD0937A03F05F
:103BF000030309B143F0040343F008039910082BB1
:103C000091722AD8072B22D2032B2ED011D9042B44
:103C100013D0062B14D1D3685DF8044B023BD3605C
:103C20007047937A03F003030029E7D043F00403BD
:103C3000E4E7012B0BD0022B02D1D368013BD36008
:103C40005DF8044B70470D2BF7D00E2BF8D1D368DD
:103C50005DF8044B0133D36070470C2B05D0F2D8CC
:103C6000092BD8D00B2BE8D0EAE7D3685DF8044BDA
:103C70000233D360704700BF4AF28853C2F2010397
:103C800010B45A6D1368506819780478507A137A12
:103C9000044201EA03011AD0937A03F0030309B145
:103CA00043F0040343F008039910082B91722AD8BB
:103CB000072B22D2032B2ED011D9042B13D0062B85
:103CC00014D1D3685DF8044B023BD3607047937AFC
:103CD00003F003030029E7D043F00403E4E7012BDA
:103CE0000BD0022B02D1D368013BD3605DF8044BAB
:103CF00070470D2BF7D00E2BF8D1D3685DF8044B2D
:103D00000133D36070470C2B05D0F2D8092BD8D0E3
:103D10000B2BE8D0EAE7D3685DF8044B0233D3609D
:103D2000704700BF4AF28853C2F2010310B49A6D83
:103D30001368506819780478507A137A044201EABB
:103D400003011AD0937A03F0030309B143F004038B
:103D500043F008039910082B91722AD8072B22D21E
:103D6000032B2ED011D9042B13D0062B14D1D368DA
:103D70005DF8044B023BD3607047937A03F0030372
:103D80000029E7D043F00403E4E7012B0BD0022B1A
:103D900002D1D368013BD3605DF8044B70470D2B13
:103DA000F7D00E2BF8D1D3685DF8044B0133D36004
:103DB00070470C2B05D0F2D8092BD8D00B2BE8D0AC
:103DC000EAE7D3685DF8044B0233D360704700BF65
:103DD0004AF28853C2F2010310B4DA6D13685068D6
:103DE00019780478507A137A044201EA03011AD050
:103DF000937A03F0030309B143F0040343F008038B
:103E00009910082B91722AD8072B22D2032B2ED07F
:103E100011D9042B13D0062B14D1D3685DF8044BB1
:103E2000023BD3607047937A03F003030029E7D085
:103E300043F00403E4E7012B0BD0022B02D1D3683B
:103E4000013BD3605DF8044B70470D2BF7D00E2B70
:103E5000F8D1D3685DF8044B0133D36070470C2B65
:103E600005D0F2D8092BD8D00B2BE8D0EAE7D368DD
:103E70005DF8044B0233D360704700BF4AF28853A9
:103E8000C2F2010310B41A6E1368506819780478EE
:103E9000507A137A044201EA03011AD0937A03F0AC
:103EA000030309B143F0040343F008039910082BFE
:103EB00091722AD8072B22D2032B2ED011D9042B92
:103EC00013D0062B14D1D3685DF8044B023BD360AA
:103ED0007047937A03F003030029E7D043F004030B
:103EE000E4E7012B0BD0022B02D1D368013BD36056
:103EF0005DF8044B70470D2BF7D00E2BF8D1D3682B
:103F00005DF8044B0133D36070470C2B05D0F2D819
:103F1000092BD8D00B2BE8D0EAE7D3685DF8044B27
:103F20000233D360704700BF4AF28853C2F20103E4
:103F300010B45A6E1368506819780478507A137A5E
:103F4000044201EA03011AD0937A03F0030309B192
:103F500043F0040343F008039910082B91722AD808
:103F6000072B22D2032B2ED011D9042B13D0062BD2
:103F700014D1D3685DF8044B023BD3607047937A49
:103F800003F003030029E7D043F00403E4E7012B27
:103F90000BD0022B02D1D368013BD3605DF8044BF8
:103FA00070470D2BF7D00E2BF8D1D3685DF8044B7A
:103FB0000133D36070470C2B05D0F2D8092BD8D031
:103FC0000B2BE8D0EAE7D3685DF8044B0233D360EB
:103FD000704700BF4AF28853C2F2010310B49A6ED0
:103FE0001368506819780478507A137A044201EA09
:103FF00003011AD0937A03F0030309B143F00403D9
:1040000043F008039910082B91722AD8072B22D26B
:10401000032B2ED011D9042B13D0062B14D1D36827
:104020005DF8044B023BD3607047937A03F00303BF
:104030000029E7D043F00403E4E7012B0BD0022B67
:1040400002D1D368013BD3605DF8044B70470D2B60
:10405000F7D00E2BF8D1D3685DF8044B0133D36051
:1040600070470C2B05D0F2D8092BD8D00B2BE8D0F9
:10407000EAE7D3685DF8044B0233D360704700BFB2
:104080004AF28853C2F2010310B4DA6E1368506822
:1040900019780478507A137A044201EA03011AD09D
:1040A000937A03F0030309B143F0040343F00803D8
:1040B0009910082B91722AD8072B22D2032B2ED0CD
:1040C00011D9042B13D0062B14D1D3685DF8044BFF
:1040D000023BD3607047937A03F003030029E7D0D3
:1040E00043F00403E4E7012B0BD0022B02D1D36889
:1040F000013BD3605DF8044B70470D2BF7D00E2BBE
:10410000F8D1D3685DF8044B0133D36070470C2BB2
:1041100005D0F2D8092BD8D00B2BE8D0EAE7D3682A
:104120005DF8044B0233D360704700BF4AF28853F6
:10413000C2F2010310B41A6F13685068197804783A
:10414000507A137A044201EA03011AD0937A03F0F9
:10415000030309B143F0040343F008039910082B4B
:1041600091722AD8072B22D2032B2ED011D9042BDF
:1041700013D0062B14D1D3685DF8044B023BD360F7
:104180007047937A03F003030029E7D043F0040358
:10419000E4E7012B0BD0022B02D1D368013BD360A3
:1041A0005DF8044B70470D2BF7D00E2BF8D1D36878
:1041B0005DF8044B0133D36070470C2B05D0F2D867
:1041C000092BD8D00B2BE8D0EAE7D3685DF8044B75
:1041D0000233D360704700BF4AF28853C2F2010332
:1041E00010B45A6F1368506819780478507A137AAB
:1041F000044201EA03011AD0937A03F0030309B1E0
:1042000043F0040343F008039910082B91722AD855
:10421000072B22D2032B2ED011D9042B13D0062B1F
:1042200014D1D3685DF8044B023BD3607047937A96
:1042300003F003030029E7D043F00403E4E7012B74
:104240000BD0022B02D1D368013BD3605DF8044B45
:1042500070470D2BF7D00E2BF8D1D3685DF8044BC7
:104260000133D36070470C2B05D0F2D8092BD8D07E
:104270000B2BE8D0EAE7D3685DF8044B0233D36038
:10428000704700BF4AF28853C2F2010310B49A6F1C
:104290001368506819780478507A137A044201EA56
:1042A00003011AD0937A03F0030309B143F0040326
:1042B00043F008039910082B91722AD8072B22D2B9
:1042C000032B2ED011D9042B13D0062B14D1D36875
:1042D0005DF8044B023BD3607047937A03F003030D
:1042E0000029E7D043F00403E4E7012B0BD0022BB5
:1042F00002D1D368013BD3605DF8044B70470D2BAE
:10430000F7D00E2BF8D1D3685DF8044B0133D3609E
:1043100070470C2B05D0F2D8092BD8D00B2BE8D046
:10432000EAE7D3685DF8044B0233D360704700BFFF
:104330004AF28853C2F2010310B4DA6F136850686E
:1043400019780478507A137A044201EA03011AD0EA
:10435000937A03F0030309B143F0040343F0080325
:104360009910082B91722AD8072B22D2032B2ED01A
:1043700011D9042B13D0062B14D1D3685DF8044B4C
:10438000023BD3607047937A03F003030029E7D020
:1043900043F00403E4E7012B0BD0022B02D1D368D6
:1043A000013BD3605DF8044B70470D2BF7D00E2B0B
:1043B000F8D1D3685DF8044B0133D36070470C2B00
:1043C00005D0F2D8092BD8D00B2BE8D0EAE7D36878
:1043D0005DF8044B0233D360704700BF4AF2885344
:1043E000C2F2010310B4D3F8802013685068197822
:1043F0000478507A137A044201EA03011AD0937ABE
:1044000003F0030309B143F0040343F008039910D8
:10441000082B91722AD8072B22D2032B2ED011D928
:10442000042B13D0062B14D1D3685DF8044B023B48
:10443000D3607047937A03F003030029E7D043F079
:104440000403E4E7012B0BD0022B02D1D368013B1C
:10445000D3605DF8044B70470D2BF7D00E2BF8D1CD
:10446000D3685DF8044B0133D36070470C2B05D043
:10447000F2D8092BD8D00B2BE8D0EAE7D3685DF847
:10448000044B0233D36070474AF28853C2F20103EF
:1044900010B4D3F884201368506819780478507ADF
:1044A000137A044201EA03011AD0937A03F003035A
:1044B00009B143F0040343F008039910082B9172EB
:1044C0002AD8072B22D2032B2ED011D9042B13D09C
:1044D000062B14D1D3685DF8044B023BD3607047C0
:1044E000937A03F003030029E7D043F00403E4E7E1
:1044F000012B0BD0022B02D1D368013BD3605DF8B6
:10450000044B70470D2BF7D00E2BF8D1D3685DF814
:10451000044B0133D36070470C2B05D0F2D8092B24
:10452000D8D00B2BE8D0EAE7D3685DF8044B023310
:10453000D36070474AF28853C2F2010310B4D3F833
:10454000E8201368506819780478507A137A044286
:1045500001EA03011AD0937A03F0030309B143F08F
:10456000040343F008039910082B91722AD8072BF3
:1045700022D2032B2ED011D9042B13D0062B14D109
:10458000D3685DF8044B023BD3607047937A03F025
:1045900003030029E7D043F00403E4E7012B0BD029
:1045A000022B02D1D368013BD3605DF8044B704706
:1045B0000D2BF7D00E2BF8D1D3685DF8044B0133E7
:1045C000D36070470C2B05D0F2D8092BD8D00B2B19
:1045D000E8D0EAE7D3685DF8044B0233D360704754
:1045E0004AF28853C2F2010310B4D3F8EC201368E6
:1045F000506819780478507A137A044201EA03016A
:104600001AD0937A03F0030309B143F0040343F093
:1046100008039910082B91722AD8072B22D2032B5A
:104620002ED011D9042B13D0062B14D1D3685DF8EA
:10463000044B023BD3607047937A03F003030029D5
:10464000E7D043F00403E4E7012B0BD0022B02D1A7
:10465000D368013BD3605DF8044B70470D2BF7D056
:104660000E2BF8D1D3685DF8044B0133D36070474B
:104670000C2B05D0F2D8092BD8D00B2BE8D0EAE7C9
:10468000D3685DF8044B0233D36070474AF2885315
:10469000C2F2010310B41A681368506819780478DC
:1046A000507A137A044201EA03011AD0937A03F094
:1046B000030309B143F0040343F008039910082BE6
:1046C00091722AD8072B22D2032B2ED011D9042B7A
:1046D00013D0062B14D1D3685DF8044B023BD36092
:1046E0007047937A03F003030029E7D043F00403F3
:1046F000E4E7012B0BD0022B02D1D368013BD3603E
:104700005DF8044B70470D2BF7D00E2BF8D1D36812
:104710005DF8044B0133D36070470C2B05D0F2D801
:10472000092BD8D00B2BE8D0EAE7D3685DF8044B0F
:104730000233D360704700BF4AF28853C2F20103CC
:1047400010B45A681368506819780478507A137A4C
:10475000044201EA03011AD0937A03F0030309B17A
:1047600043F0040343F008039910082B91722AD8F0
:10477000072B22D2032B2ED011D9042B13D0062BBA
:1047800014D1D3685DF8044B023BD3607047937A31
:1047900003F003030029E7D043F00403E4E7012B0F
:1047A0000BD0022B02D1D368013BD3605DF8044BE0
:1047B00070470D2BF7D00E2BF8D1D3685DF8044B62
:1047C0000133D36070470C2B05D0F2D8092BD8D019
:1047D0000B2BE8D0EAE7D3685DF8044B0233D360D3
:1047E000704700BF10B445F250240023C0F2020409
:1047F0004172026104600372C36041B1194600E076
:10480000026942F82310427A01339A42F8DC4AF6F0
:104810003003C2F201031A680AB90CE01A46536960
:10482000002BFBD15061002343618380C3808372DE
:104830005DF8044B70471860F5E700BFF8B541F626
:104840007864C2F2010447F61221A06C0368DB69A8
:10485000984741F6C947032041F6294346F249717A
:1048600044F6295641F6556284F86400C0F200030C
:10487000C0F20007C0F20001C0F20006C0F2000260
:1048800041F6CD0063602760E1606661A261C0F21D
:10489000000045F6594341F2850741F6511140F6B3
:1048A000194640F6DD122061C0F20003C0F2000795
:1048B000C0F20001C0F20006C0F2000241F2F15065
:1048C000E3612762A160A662E262C0F2000040F6E6
:1048D000794340F6CD4740F6215140F6755641F2F6
:1048E0000102C0F200022063C0F20003C0F2000720
:1048F000C0F20001C0F200064EF2402545F24470BD
:104900006264C2F200056363A76300234FF6FF777A
:10491000E16326641721C0F2020084F84C3084F869
:104920004E3084F84D30A365636584F8E93084F82F
:10493000663084F8653084F8673084F86830E7655D
:10494000276619F0E1FA28461AF0F2F913F0FEFF93
:1049500041F2C053C2F2010341F6F92141F6C917F1
:1049600046F2916644F6AD5441F6E562C0F20001AC
:10497000C0F20007C0F20006C0F20004C0F200025C
:1049800041F28D70C3F86811C3F86471C3F87061A7
:10499000C3F87841C3F87C21C0F2000045F6B94164
:1049A00041F6B93741F6250641F6892440F6E96219
:1049B000C3F87401C0F20001C0F20007C0F20006A3
:1049C000C0F20004C0F2000241F27560C3F8841125
:1049D000C3F88871C3F86C61C3F89041C3F894219F
:1049E000C0F2000040F6312140F6892740F6E1266A
:1049F00040F6393440F69132C0F20002C3F8980113
:104A0000C0F20001C0F20007C0F20006C0F20004CC
:104A100045F25C70C3F89C11C3F8A071C3F8A4619F
:104A2000C3F8A841C3F8AC211D21C0F2020019F05F
:104A30006BFA28461AF07CF94AF61801C2F2010115
:104A400041F2E13EC0F2000E4AF61004C1F800E067
:104A5000C2F2010441F2792EC0F2000E4AF61403AC
:104A6000C4F800E0C2F2010346F27D5EC0F2000E1F
:104A70004AF2E877C3F800E0C2F2010744F6456E57
:104A8000C0F2000E4AF2D870C7F800E0C2F201008E
:104A900041F2A94EC0F2000E4AF2D476C0F800E00E
:104AA000C2F2010641F2413EC0F2000E4AF2F87233
:104AB000C6F800E0C2F2010245F63D5EC0F2000E0B
:104AC0004AF2F071C2F800E0C2F2010141F6DD5E87
:104AD000C0F2000E4AF2E474C1F800E0C2F2010430
:104AE00041F2D91EC0F2000E4AF60C03C4F800E0F1
:104AF000C2F2010341F6655EC0F2000E4AF2F4779D
:104B0000C3F800E0C2F2010741F2E90EC0F2000E64
:104B10004AF2BC70C7F800E0C2F2010041F2FD6742
:104B2000C0F200074AF2EC760760C2F201064AF2D0
:104B3000CC7240F64177C2F20102C0F200074AF699
:104B4000040140F6A1703760C2F20101C0F200001A
:104B50004AF2C4744AF2C07340F68967C2F2010394
:104B60001060C2F20104C0F2000740F6296641F26B
:104B7000491245F27C700F60C0F20006C0F20002DC
:104B8000C0F20200182126601A6019F0BDF928460B
:104B9000BDE8F8401AF0CCB84DF20A73C3F62343CF
:104BA00006EE103A437EC17E07EE103A837CB8EEE3
:104BB000C77A07EE903A70B4F8EEE76A27EE067A05
:104BC00083B067EE267A0022FCEEE77A8273CDEDA1
:104BD000017A42739DF80430027301B10373827E3F
:104BE00002B14373027F02B1837390F8213090F8D1
:104BF000231007EE103A4DF20A73C3F6234306EE74
:104C0000103A037CB8EEC77A07EE903A27EE067AA0
:104C1000F8EEE76A67EE267AFCEEE77ACDED017AE8
:104C20009DF8043021B1017B994238BF19460173C8
:104C300090F8221021B1417B994238BF1946417347
:104C400090F8244024B1817B8B4238BF0B4683739C
:104C5000437FC17F07EE103A4DF20A73C3F6234338
:104C600006EE103A437CB8EEC77A07EE903A27EE8C
:104C7000067AF8EEE76A67EE267AFCEEE77ACDED83
:104C8000017A9DF8043021B1017B994238BF194661
:104C90000173817F21B1417B994238BF194641732D
:104CA00090F8201021B1857BAB4238BF2B4683732F
:104CB00090F8253090F8275007EE103A4DF20A731D
:104CC000C3F6234306EE103AC37BB8EEC77A07EE6D
:104CD000903A27EE067AF8EEE76A67EE267AFCEE5F
:104CE000E77ACDED017A9DF8043025B1057B9D4230
:104CF00038BF1D46057390F8265025B1457B9D426F
:104D000038BF1D46457390F8285025B1867BB342C5
:104D100038BF3346837322B919B914B90DB97F234B
:104D2000837303B070BC704738B541F29053C2F240
:104D300001030C461B680546240483F8CF1003F1D9
:104D4000C00004F4FE04013DFFF726FF44F4504484
:104D500045F298702D020D2105F47065C0F2020035
:104D600044F00D0419F0D0F82C4341F2C050214614
:104D7000C2F2010015F01CFC45F2E0201421C0F243
:104D8000020019F0C1F8204618F034FA45F2F82074
:104D9000C0F202000F2119F0B7F84EF24020C2F223
:104DA0000000BDE8384019F0C3BF00BF41F2905386
:104DB000C2F2010370B51B68054683F8CF1003F1FA
:104DC000C0000C46FFF7E8FE45F2A8701221013D35
:104DD000C0F2020019F098F8E9B20F290FD841F695
:104DE0007866C2F2010641F0D001B06C03681B681E
:104DF0009847B06C036804F07F011B68984745F240
:104E000020300F21C0F2020019F07EF8230403F4D1
:104E1000FE03280243F4504343F00D0300F4706096
:104E2000184318F0E7F945F2F820C0F202000F210C
:104E300019F06AF84EF24020C2F20000BDE870405E
:104E400019F076BF41F29053C2F2010370B51B68AE
:104E5000054683F8CF1003F1C0000C46FFF79CFE17
:104E600045F2BC700D21013DC0F2020019F04CF872
:104E7000E9B20F290FD841F67866C2F2010641F077
:104E8000D001B06C03681B689847B06C036804F0ED
:104E90007F011B68984745F220300F21C0F20200C5
:104EA00019F032F8230403F4FE03290243F45043BB
:104EB00043F00D0301F4706141F2C0501943C2F296
:104EC000010015F075FB45F2E020C0F2020014214C
:104ED00019F01AF84EF24020C2F20000BDE870400E
:104EE00019F026BF10B4036841681A780C78417A2B
:104EF000037A0C4202EA03021AD0837A03F0030316
:104F00000AB143F0040343F008039A10082B82729D
:104F10002AD8072B22D2032B2ED011D9042B13D041
:104F2000062B14D1C3685DF8044B023BC360704785
:104F3000837A03F00303002AE7D043F00403E4E795
:104F4000012B0BD0022B02D1C368013BC3605DF87B
:104F5000044B70470D2BF7D00E2BF8D1C3685DF8CA
:104F6000044B0133C36070470C2B05D0F2D8092BDA
:104F7000D8D00B2BE8D0EAE7C3685DF8044B0233C6
:104F8000C36070471D2810B50B4600F0E983024648
:104F900022D92C2800F064813FD8242800F0EE8329
:104FA00040F2A880282800F0748300F2D6802628DA
:104FB00000F0F58140F2D5824AF28854C2F2010431
:104FC00042F65101C0F2000104222720C4F89C30AF
:104FD00016F0FCFD012010BD0E2800F097833AD892
:104FE000062800F0A1836CD90A2800F0058300F29E
:104FF0000781082800F07E8140F275824AF28854C9
:10500000C2F2010443F26941C0F200010422092006
:10501000636216F0DBFD012010BD342800F0BD8373
:1050200036D8302800F0638300F2D6802E2800F0B6
:10503000528140F201824AF28854C2F2010442F6DF
:10504000B151C0F2000104222F20C4F8BC3016F088
:10505000BDFD012010BD152800F0748364D9192806
:1050600000F0FA8100F2A580172800F08A8140F252
:10507000D1824AF28854C2F2010443F67D61C0F243
:10508000000104221820236616F0A0FD012010BDA7
:10509000382800F0CE8275D8362800F0398140F2E9
:1050A0007F824AF28854C2F2010442F2F121C0F236
:1050B000000104223720C4F8DC3016F087FD0120FF
:1050C00010BD022800F0018240F27881042800F02F
:1050D0004B8140F2BD824AF28854C2F2010443F28D
:1050E000B911C0F2000104220520636116F06EFDC3
:1050F000012010BD202800F0448240F2898122283E
:1051000000F0238140F2D4824AF28854C2F20104B2
:1051100042F2A151C0F2000104222320C4F88C30D5
:1051200016F054FD012010BD112800F0B18140F2AD
:105130005A81132800F0FB8040F2B8814AF288546B
:10514000C2F2010443F6CD31C0F200010422142062
:10515000236516F03BFD012010BD2A2800F0AC802D
:1051600040F2E0814AF28854C2F2010442F6013171
:10517000C0F2000104222B20C4F8AC3016F026FD4A
:10518000012010BD3A2800F08880C0F072823B28D0
:1051900040F06D824AF28854C2F2010444F2E151B7
:1051A000C0F200010422C4F8EC3016F00FFD01201B
:1051B00010BD1B2863D040F28B824AF28854C2F2A1
:1051C000010444F22D11C0F2000104221C202367C7
:1051D00016F0FCFC012010BD322824D040F2928150
:1051E0004AF28854C2F2010442F24101C0F20001C5
:1051F00004223320C4F8CC3016F0E8FC012010BDA6
:105200000C281FD040F29E814AF28854C2F2010459
:1052100043F21971C0F2000104220D20636316F0FD
:10522000D5FC012010BD4AF28854C2F2010441F6B7
:105230009571C0F200010422C4F8C83016F0C6FC13
:10524000012010BD4AF28854C2F2010443F26D619C
:10525000C0F200010422236316F0B8FC012010BD47
:105260004AF28854C2F2010442F6AD31C0F20001A4
:105270000422C4F8B03016F0A9FC012010BD4AF297
:105280008854C2F2010444F28101C0F200010422F8
:10529000E36616F09BFC012010BD4AF28854C2F26E
:1052A000010444F23551C0F200010422C4F8E83090
:1052B00016F08CFC012010BD4AF28854C2F20104A1
:1052C00042F65521C0F200010422C4F8A83016F0BD
:1052D0007DFC012010BD4AF28854C2F2010442F65E
:1052E0000551C0F200010422C4F8B83016F06EFC7B
:1052F000012010BD4AF28854C2F2010443F2BD31CC
:10530000C0F200010422236216F060FC012010BDEF
:105310004AF28854C2F2010442F24521C0F200016F
:105320000422C4F8D83016F051FC012010BD4AF216
:105330008854C2F2010443F62131C0F20001042274
:10534000E36416F043FC012010BD4AF28854C2F217
:10535000010442F2F541C0F200010422C4F8883091
:1053600016F034FC012010BD4AF28854C2F2010448
:1053700043F20D11C0F20001236116F027FC012059
:1053800010BD4AF28854C2F2010443F6D151C0F272
:1053900000010422E36516F019FC012010BD4AF259
:1053A0008854C2F2010442F2A571C0F20001042245
:1053B000C4F8983016F00AFC012010BD002800F057
:1053C000FF80012840F053814AF28854C2F2010460
:1053D00044F23971C0F2000104220120636016F02A
:1053E000F5FB012010BD0F2800F0F880102840F0D8
:1053F0003E814AF28854C2F2010443F61D11C0F204
:10540000000104221020236416F0E0FB012010BDEF
:105410001E282FD01F2840F02A814AF28854C2F259
:10542000010444F23131C0F2000104221F20E3677D
:1054300016F0CCFB012010BD4AF28854C2F20104E0
:1054400042F65941C0F2000104222D20C4F8B430C4
:1054500016F0BCFB012010BD4AF28854C2F20104D0
:1054600043F62971C0F200010422636616F0AEFB18
:10547000012010BD4AF28854C2F2010444F2852191
:10548000C0F200010422A36716F0A0FB012010BDAA
:105490004AF28854C2F2010443F6C911C0F2000175
:1054A0000422636416F092FB012010BD4AF2885476
:1054B000C2F2010443F67521C0F200010422122059
:1054C000A36416F083FB012010BD4AF28854C2F297
:1054D000010442F6B571C0F200010422A36016F087
:1054E00075FB012010BD4AF28854C2F2010443F258
:1054F0001131C0F2000104220720E36116F066FBBF
:10550000012010BD4AF28854C2F2010442F609712A
:10551000C0F2000104223120C4F8C43016F056FB5A
:10552000012010BD4AF28854C2F2010442F6A911CA
:10553000C0F2000104222920C4F8A43016F046FB72
:10554000012010BD4AF28854C2F2010443F2C15155
:10555000C0F2000104220B20E36216F037FB0120A9
:1055600010BD4AF28854C2F2010442F2F961C0F25D
:10557000000104222520C4F8943016F027FB0120F6
:1055800010BD4AF28854C2F2010444F2DD31C0F287
:1055900000010422C4F8803016F018FB012010BD71
:1055A0004AF28854C2F2010442F29911C0F2000199
:1055B00004223520C4F8D43016F008FB012010BDB9
:1055C0004AF28854C2F2010444F28D61C0F2000133
:1055D0000422236016F0FAFA012010BD4AF2885422
:1055E000C2F2010443F67101C0F200010422E36338
:1055F00016F0ECFA012010BD4AF28854C2F2010400
:1056000043F21551C0F200010422A36216F0DEFA43
:10561000012010BD4AF28854C2F2010443F625511C
:10562000C0F2000104221620A36516F0CFFA012073
:1056300010BD4AF28854C2F2010442F29D31C0F218
:1056400000010422C4F8E03016F0C0FA012010BDB9
:105650004AF28854C2F2010443F26101C0F200012F
:1056600004220320E36016F0B1FA012010BD0020EF
:1056700010BD4AF28854C2F2010442F24941C0F21C
:10568000000104223920C4F8E43016F09FFA01200A
:1056900010BD4AF28854C2F2010442F6FD01C0F284
:1056A00000010422C4F8A03016F090FA012010BDC9
:1056B0004AF28854C2F2010444F28941C0F2000166
:1056C00004222120C4F8843016F080FA012010BD95
:1056D0004AF28854C2F2010443F6D571C0F20001C7
:1056E00004221A20A36616F071FA012010BD4AF2B6
:1056F0008854C2F2010442F65D61C0F20001042246
:10570000C4F8C03016F062FA012010BD4AF2885485
:10571000C2F2010443F2C571C0F200010422A36386
:1057200016F054FA012010BD4AF28854C2F2010466
:1057300043F26521C0F200010422A36116F046FA8B
:10574000012010BD4AF28854C2F2010443F67941A7
:10575000C0F200010422636516F038FA012010BD82
:105760004AF28854C2F2010444F2D911C0F2000195
:105770000422636716F02AFA012010BD4AF2885409
:10578000C2F2010442F24D61C0F200010422C4F8E9
:10579000903016F01BFA012010BD4AF28854C2F274
:1057A000010442F2ED01C0F200010422C4F8D0303D
:1057B00016F00CFA012010BDF8B5044615460E4649
:1057C0000846022116F07AFC2846022116F076FCE3
:1057D00046F68C23C0F20203012253F836002272EF
:1057E00000F50071216053F8351062724DF2C0432C
:1057F00001F5007762F31F4300226760E260013B1E
:10580000FDD190F8003291F8002203F00103D20795
:1058100044BF43F00203DBB2A37221463046FFF7D8
:10582000B1FB214620742846FFF7ACFB237C1844CB
:1058300020742046F8BD00BFF0B5074645F2CC7095
:10584000A9B00E46C0F202000B2118F05DFB4EF22B
:1058500040203146C2F2000000230A2219F07AFAF1
:1058600045F2D870C0F20200012118F04DFBB6B12C
:1058700000252C4645F6C8300121C0F2020018F080
:1058800043FB01344EF24020795DE4B2C2F20000E5
:1058900000230A2219F05EFAA6422546EAD84EF203
:1058A0004020C2F2000019F043FA4DF6C063C2F284
:1058B00000031B7C6BB1B87800F00F00013083420D
:1058C00007D0FBF781FA20B945F2DC70C0F2020084
:1058D00006E07B78432B0ED045F2F870C0F2020050
:1058E0001B2118F011FB4EF24020C2F2000019F00B
:1058F0001FFA29B0F0BD45F614000C21C0F20200D9
:1059000018F002FBB9784EF24020C1F30211C2F246
:10591000000019F0AFF945F2D8700121C0F2020081
:1059200018F0F2FA4EF24020C2F2000019F000FA2C
:10593000072E1DD0A32E07D045F67810C0F2020026
:10594000FBF73AF829B0F0BD45F6AC00C0F2020012
:1059500097F8A140FBF730F897F8A230F72B00F04A
:10596000F88045F6C000C0F20200FBF725F8C0E75A
:10597000FB78C3F38403002B69D1BB79F72B40F08C
:10598000F9803A797B7941F29054C2F2010402F035
:105990007F0203F07F0320683A717B710AF064F89C
:1059A000FA783B792068797902F0030203EBC2139D
:1059B000034483F86C1109F04BFFFC783B7903EB4F
:1059C000C41404F0FF0445F6C010C0F20200FAF758
:1059D000E9FFFB7813F07C0F05D145F68400C0F297
:1059E0000200FAF7DFFF45F69000C0F20200FAF776
:1059F000D9FF4EF24020397900230A22C2F200007A
:105A000019F0A8F945F6A800C0F20200FAF7CAFF9B
:105A10004EF24020797900230A22C2F2000019F0E8
:105A200099F945F69C00C0F20200FAF7BBFF4EF26E
:105A30004020214600230A22C2F2000019F08AF910
:105A40004EF24020C2F2000019F072F951E7022B29
:105A500040F09780BB79F72B40F08C8041F2905357
:105A6000C2F2010339791B687A794AF6AB2001F05A
:105A70007F01C3F6AA5007EE100A581802F07F0201
:105A800039717A7180F8C82193F80A4293F8075265
:105A900093F80C0293F80862C3F8C45093F80952C3
:105AA00093F80E2293F81012C3F8C86083F8D95007
:105AB00004F00106C4F34005C4F3800493F80BE23C
:105AC00083F8DA6083F8DB5000F0010683F8DC40ED
:105AD000C0F3400593F80D4283F8DDE0C0F3800089
:105AE00083F8DE6002F0010E83F8DF5083F8E000F7
:105AF00093F80F5283F8E140C1F3400001F0010434
:105B0000C2F34006C2F3800283F8E42083F8E64043
:105B100083F8E2E083F8E36083F8E55083F8E70078
:105B200093F81122520607EE902AF8EEE77AC1F3B5
:105B3000800167EE877A83F8E810FDEEE77A03F1DB
:105B4000C000C3ED357AFFF727F83C795C34E4B246
:105B500039E7FB7813F07F034ED139797A7942EA3D
:105B6000C1129B2A14D045F60410C0F20200FAF7C5
:105B700023FFBEE645F65C00C0F20200FAF71CFF08
:105B8000B7E645F62400C0F20200FAF715FFB0E6CA
:105B90001A4607F1A0007B1D13F8011F9842A2EBE3
:105BA0000102F9D165B202F07F04AC422BD045F678
:105BB0003C10C0F20200FAF7F5FE4EF240202946F2
:105BC00000231022C2F2000019F0C4F845F660105C
:105BD000C0F20200FAF7E6FE4EF240202146002312
:105BE0001022C2F2000019F0B5F845F2D870C0F2E8
:105BF0000200FAF7E1FE7CE645F6E000C0F20200A2
:105C0000FAF7DAFE75E6B91D01A89B2215F00EFC25
:105C100041F654600DF195010A22C2F201001FF015
:105C20001DF845F66410C0F20200FAF7BBFE41F61B
:105C30005460C2F20100FAF7B5FE45F66C10C0F2EE
:105C40000200FAF7AFFE41F29053C2F2010301A93C
:105C500018680AF089F84CE638B504460D46FFF797
:105C6000EBFD45F69C101021C0F2020018F04CF933
:105C700041F2C05000232A462146C2F2010014F02E
:105C8000D5FC45F2E0201421C0F2020018F03CF9E6
:105C900029462046002217F001FB45F2F820C0F209
:105CA00002000F2118F030F94EF24020C2F200003D
:105CB000BDE8384019F03CB82DE9F04141F678656F
:105CC0000F468046C2F20105FFF7B6FD45F6B0105B
:105CD0001521C0F2020018F017F9A86C0368F02132
:105CE000DB6C984757B1444608EB0706A86C14F8DC
:105CF000011B03681B689847A642F7D1A86C03688C
:105D0000F721DB6C984745F220300F21C0F20200EA
:105D100018F0FAF839464046002217F0BFFA45F26B
:105D2000F820C0F202000F2118F0EEF84EF24020E9
:105D3000C2F20000BDE8F04118F0FABF2DE9F041D1
:105D400041F678650F468046C2F20105FFF774FD03
:105D500045F6C8101021C0F2020018F0D5F8A86C62
:105D60000368F021DB6C984757B1444608EB0706FF
:105D7000A86C14F8011B03681B689847A642F7D16A
:105D8000A86C0368F721DB6C984745F220300F219F
:105D9000C0F2020018F0B8F841F2C0503A4641464D
:105DA000C2F20100002314F041FC45F2E020C0F2F1
:105DB0000200142118F0A8F84EF24020C2F20000B0
:105DC000BDE8F04118F0B4BF38B545F6DC1010EE70
:105DD000105A4DF6C0642DED048BC2F2000414215C
:105DE000C0F20200B0EE608AC4ED030A84ED020A3C
:105DF00018F08AF828461DF0A9FE41EC100B4EF26F
:105E000040200A21C2F2000018F0E4FF45F6F41029
:105E10000121C0F2020018F077F840F6DB73C4F2FB
:105E20004903A06809EE103A1DF090FE41EC100BFA
:105E30004EF240200A21C2F2000018F0CBFF45F6D6
:105E4000F8100621C0F2020018F05EF845F6F410D2
:105E50000121C0F2020018F057F8E0681DF076FE4C
:105E600041EC100B4EF240200A21C2F2000018F063
:105E7000B1FF45F600200221C0F2020018F044F8FC
:105E8000E36807EE903A27EE890AF6EE008A20EEE4
:105E9000280A1AF099FEA36807EE903A60EE277A76
:105EA00017EE900A1DF052FE9FED511B41EC100BB6
:105EB0001AF08AFF4EF240200321C2F2000018F0CF
:105EC00089FF45F604200121C0F2020018F01CF8F9
:105ED000E36807EE903A27EE890A20EE280A1AF0C6
:105EE00023FEA36807EE903A60EE277A17EE900A39
:105EF0001DF02CFE9FED3E1B41EC100B1AF064FFD1
:105F00004EF240200321C2F2000018F063FF4EF26F
:105F10004020C2F2000018F00BFF41F2905328EE2F
:105F2000098AC2F2010328EE288A1B68B0EE480AEB
:105F3000C3F868511AF048FE4FF47E43C4F2FF6381
:105F400007EE903AB4EEE70AF1EE10FA0EDC4FF4E9
:105F50007E43CCF2FF6307EE903AB4EEE70AF1EE2F
:105F600010FA30D50023C8F2010302E00023C7F67F
:105F7000FF7341F23452C2F20102B0EE480A93615B
:105F80001AF0D2FD4FF47E43C4F2FF6307EE903A5D
:105F9000B4EEE70AF1EE10FA23DC4FF47E43CCF2C4
:105FA000FF6307EE903AB4EEE70AF1EE10FA11D56E
:105FB0000023C8F20103BDEC048B41F26442C2F23B
:105FC0000102936138BDF0EE407AFEEEC87A17EE1A
:105FD000903ACEE7F0EE407AFEEEC87A17EE903AAD
:105FE000E9E70023C7F6FF73E5E700BFAFF30080E2
:105FF0000000002085EBB13F2DE9F041044645F655
:1060000008200D46C0F20200032117F07DFF4EF27A
:10601000402000230A222146C2F2000018F09AFE16
:1060200045F60C200121C0F2020017F06DFF4EF280
:106030004020294600230A22C2F2000018F08AFEFE
:106040004EF24020C2F2000018F072FE672C00F001
:10605000CF8150D9782C00F0A28000F28C80692C7E
:1060600000F0C080C0F09C816A2C00F05D816B2C38
:1060700040F06782002301EE903A05EB45050023CE
:10608000C4F2482305EB051501EE103AC5F3C7131A
:1060900007EE903A41F67462C2F20102B8EE670A66
:1060A000F0EE610AB7EE002A137003F091FE4FF490
:1060B0007E43C4F2FF6307EE903AB4EEE70AF1EED6
:1060C00010FA00F3D5814FF47E43CCF2FF6307EE64
:1060D000903AB4EEE70AF1EE10FA40F13482002370
:1060E000C8F2010341F2BC42C2F20102BDE8F04134
:1060F000D36106F00DBA042C00F0A28140F2C980F1
:106100000A2C5ED040F2E480202C00F00681402C66
:1061100040F0308241F29056C2F201063F2D94BF0A
:1061200000210121306809F09FFB306809F0A4FBD1
:106130000546002840F0AB803068374609F038FD4E
:10614000EBB203EB430498424FEA840440F29F8091
:10615000306803190135DA78002AEFD093F802800D
:10616000B8F1000FEAD198680BF06EF83868044473
:1061700084F80380E2E77B2C1AD040F29D807E2CCD
:1061800000F0C1807F2C40F0F78141F29053C2F2C1
:10619000010300211868BDE8F04109F05DBB41F240
:1061A0009053C2F20103BDE8F041186809F068BBE2
:1061B00041F29053C2F20103BDE8F041186809F0C2
:1061C00053BC4DF6C063C2F2000300EE905A9A68C9
:1061D000FBEEEC0A00EE102ABDE8F041C3ED030A25
:1061E000FFF7F2BD002301EE903A0023C4F296437C
:1061F00002EE103A05EB45050023C4F2482305EBF7
:10620000051501EE103AC5F3C71307EE903A40F2B8
:106210006C52C2F20102B8EE670AF0EE610A137026
:1062200003F0D6FDB5EEC00AF1EE10FA00F13181AF
:1062300047F67903C4F2302307EE103AF6EE007AFF
:10624000E0EE077A49F68073C0F20103FCEEE77ACC
:1062500017EE902A9A4240F284811A464FF4507009
:1062600040F22073C2F20103197ECC0700F11481C1
:10627000DC8B1A62844241F0010138BFD883197661
:10628000BDE8F04106F044B9632D40F2F980BDE865
:10629000F081012C00F0E080F6D3022C40F04F8119
:1062A00041F29053C2F20103186880F8D050C03018
:1062B000FEF772FCBDE8F081792C40F0598141F283
:1062C0009053C2F20103BDE8F041186809F0ECBA3E
:1062D000072C40F04B8107EE905A0023C4F2FE23B6
:1062E000B8EE677A07EE903A87EE270A4DF6C0635C
:1062F000C2F20003BDE8F041DA6800EE902A83EDB7
:10630000020AFFF761BD41F29053C2F2010301217D
:106310001868BDE8F04109F09FBA4DF6C063C2F2BB
:1063200000031D71BDE8F08105EBC5050022C5F332
:10633000471501EE902A07EE905A41F6F0430022ED
:10634000C2F20103C4F20C22B8EE670A01EE102A71
:10635000F0EE610AB7EE002A1D7003F039FD4FF42C
:106360007E43C4F2FF6307EE903AB4EEE70AF1EE23
:1063700010FA00F381804FF47E43CCF2FF6307EE06
:10638000903AB4EEE70AF1EE10FA40F1E380002310
:10639000C8F2010341F28442C2F20102D3616FE705
:1063A0002DB205EB850303EB830305EB8305C5F3F2
:1063B000C71507EE905A0023C4F2C823F8EE676AA7
:1063C00007EE903A86EEA77A41F29052C2F20102AD
:1063D00040F21C03C2F2010312681D70BDE8F041D7
:1063E000F7EE007A77EEC77AC2ED587A06F090B8E9
:1063F0002DB205EB850303EB830305EB8305C5F3A2
:10640000C71507EE905A0023C4F2C823F8EE676A56
:1064100007EE903A86EEA77A41F29052C2F201025C
:1064200041F6F143C2F2010312681D70BDE8F0416C
:10643000F7EE007A77EEC77AC2ED597A06F068B8BF
:1064400041F29053C2F20103186880F8D150C03075
:10645000FEF7A2FBBDE8F08141F29053C2F20103C6
:10646000186880F8D250C030FEF796FBBDE8F08186
:106470000023C7F6FF7335E60023C7F6FF7389E7ED
:106480004DF6C063C2F200031D71BDE8F04106F095
:106490003FB801200022E3E61C6AA24205D9D98B4D
:1064A0001A62884288BFD883EAE602F17F00C009F9
:1064B000013000281A62024638BF0022880706D53C
:1064C000586A7F30C0090130824238BF02464F0708
:1064D00006D5986A7F30C0090130824238BF024633
:1064E0000E0706D5D86A7F30C0090130824238BF16
:1064F0000246CD0606D5186B7F30C00901308242B6
:1065000038BF02468C0606D5586B7F30C009013073
:10651000824238BF0246480606D5986B7F30C009D4
:106520000130824238BF0246C90906D0D96B7F319B
:10653000C90901318A4238BF0A46DA83A0E6BDE8BC
:10654000F081BDE8F081F0EE407AFEEEC87A17EEF9
:10655000903AC7E5F0EE407AFEEEC87A17EE903A30
:1065600018E702F17F00C009013079E6BDE8F0814B
:10657000BDE8F081BDE8F081BDE8F081F8B54DF6E9
:10658000C067C2F2000704463B7C0E4615467BB34B
:1065900098422DD045F220401E21C0F2020017F093
:1065A000B3FC4EF2402000230A222146C2F2000032
:1065B00018F0D0FB45F240400E21C0F2020017F067
:1065C000A3FC4EF24020397C00230A22C2F20000D4
:1065D00018F0C0FB45F250400121C0F2020017F054
:1065E00093FC4EF24020C2F2000018F0A1FB03E041
:1065F00029463046FFF700FD45F610200D21013CED
:10660000C0F2020017F080FCE1B20F2915D841F664
:106610007867C2F2010741F0B001B86C03681B68EB
:106620009847B86C036806F07F011B689847B86C00
:10663000036805F07F011B68984745F220300F2161
:10664000C0F2020017F060FC2B0603F0FE43310499
:1066500043F4304343F00B0301F4FE0124021943D9
:1066600004F4706441F2C0502143C2F2010013F0FF
:106670009FFF45F2E020C0F20200142117F044FC15
:106680004EF24020C2F20000BDE8F84018F050BBC6
:10669000F8B54DF6C063C2F200030E461B7C1446EB
:1066A000054623B1984202D0FAF78EFB18B1214675
:1066B0003046FFF7A1FC45F620201221013DC0F233
:1066C000020017F021FCE9B20F2915D841F67867CE
:1066D000C2F2010741F0B001B86C03681B6898472B
:1066E000B86C036806F07F011B689847B86C0368B4
:1066F00004F07F011B68984745F220300F21C0F25B
:10670000020017F001FC230603F0FE43310443F4BA
:10671000304301F4FE01280243F00B030B4300F465
:106720007060184316F066FD45F2F820C0F20200D2
:106730000F2117F0E9FB4EF24020C2F20000BDE845
:10674000F84018F0F5BA00BF70B54DF6C063C2F25C
:1067500000030E461B7C1446054623B1984202D026
:10676000FAF732FB18B121463046FFF745FC45F6F3
:1067700034200D21C0F2020017F0C6FB230603F0FF
:10678000FE43340443F43043013D43F00B0304F46F
:10679000FE042D021C4305F470652C4341F2C050E9
:1067A0002146C2F2010013F003FF45F2E02014215C
:1067B000C0F2020017F0A8FB204616F01BFD45F2C0
:1067C000F820C0F202000F2117F09EFB4EF240208D
:1067D000C2F20000BDE8704018F0AABA4AF28C6319
:1067E000C2F2010382B01B68019341F67062C2F2EB
:1067F000010240F2CC53C2F201030199116001225F
:106800001A7002B0704700BF45F288232DE9F04F9F
:10681000C0F202031C460FCCB1B020AD0FC50FCCA7
:106820000FC50FCC0FC594E80F0010944DF6C0674C
:1068300040F2CC54C2F20007C2F201044FF0000E45
:1068400084F800E01F9585E80F00BD7A0395FD7A76
:106850003B7904953D7B05957D7B06956FEA0309A1
:10686000BD7B079509F00F0930AD05EB8909BA79B1
:1068700097F80580787A02901D1159F8403C1195DF
:106880001146FA79139183F070431446DB433A7A48
:10689000019283EA05020DF1C00E02F00F020EEB29
:1068A00082024FEA281E52F8402C82EA1313DB437F
:1068B00083EA0802754602F00F020DF1C00E0EEBDE
:1068C00082020DF1C00E52F8402C129582EA131389
:1068D00083EA050202F00F020EEB82020DF1C00EF8
:1068E00052F8402C82EA1313DB4383EA010202F0E0
:1068F0000F020EEB8202081152F8402C0199064655
:1069000082EA131383EA06020DF1C00E02F00F02B1
:106910000EEB8202081114960990029852F8402C4E
:10692000159482EA1313DB4383EA04020DF1C00ECF
:1069300002F00F020EEB8202251152F8402C039C4C
:10694000169582EA131383EA05020DF1C00E02F0D8
:106950000F020EEB82020DF1C00E52F8402C82EABB
:1069600013136FEA030C8CEA010202F00F0205997F
:106970000EEB82020B1152F8402C0C93099B82EA19
:106980001C1C8CEA03020DF1C00E02F00F020EEB8C
:106990008202069B52F8402C1B110D9382EA1C13B5
:1069A000DB4383EA0002061102F00F0207980A9601
:1069B0000DF1C00E0EEB820E02110E925EF8402C0D
:1069C00082EA13130A9A5A4002F00F020DF1C00E28
:1069D0000EEB820E109AA2F1300C5EF8402C82EA87
:1069E0001313DB4383EA04020DF1C00E02F00F0221
:1069F0000EEB820226110B9652F8402C0B9C049E43
:106A000082EA131383EA04020DF1C00A02F00F02B6
:106A10000AEB8202351152F8402C179582EA1313C3
:106A2000DB4383EA060202F00F020AEB82020DF159
:106A3000C00A52F8402C0C9E82EA131383EA050226
:106A400002F00F020AEB82020DF1C00A52F8402C4C
:106A500082EA1313DB4383EA010202F00F020AEB1E
:106A600082020DF1C00A52F8402C82EA131383EA25
:106A7000060202F00F020AEB82020DF1C00A52F880
:106A8000402C069E0E9D97F813B082EA1313DB4349
:106A900083EA060202F00F020AEB82020D9E52F810
:106AA000402C82EA131383EA06020DF1C00A02F0B9
:106AB0000F020AEB82020DF1C00A52F8402C82EA62
:106AC0001313DB4383EA000202F00F020AEB820297
:106AD0000DF1C00A52F8402C82EA131383EA050232
:106AE00002F00F020AEB820297F80FA052F8402C36
:106AF000564697F810A01896514697F811A01A918B
:106B000082EA13135046DB4397F812A083EA060289
:106B1000554602F00F020DF1C00A0AEB820236114F
:106B200052F8402C199682EA131383EA06020DF1FB
:106B3000C00A02F00F020AEB82020DF1C00A52F8FD
:106B4000402C1D9582EA1313DB4383EA010202F015
:106B50000F020AEB82020E1152F8402C0F9682EAC5
:106B600013130F9A5A400DF1C00A02F00F020AEBFC
:106B70008202064652F8402C1B9682EA1313DB432E
:106B800083EA06020DF1C00A02F00F020AEB82024C
:106B9000011152F8402C1C9182EA131383EA01027E
:106BA0004FEA2B1ACDF820A002F00F020DF1C00A17
:106BB0000AEB82020DF1C00A52F8402C82EA13134C
:106BC000DB4383EA050202F00F020AEB820228117E
:106BD00052F8402C1E9082EA131383EA00020DF152
:106BE000C00A02F00F020AEB820230AE52F8402CCB
:106BF00082EA1313DB438BEA030202F00F020AEB73
:106C000082020DF1800E52F8402C82EA131A089B82
:106C100055468AEA030ABCE80F000AF00F0A06EBA1
:106C20008A0A3C465AF840ACAEE80F00BCE80F00B8
:106C3000AEE80F00BCE80F00AEE80F0059F8402C9A
:106C40008AEA151A82F07042119DD24382EA050346
:106C500003F00F0306EB83030DF1C00E53F8403C25
:106C600083EA1212D24382EA080303F00F0306EB11
:106C700083036FEA0A0A53F8403CC7F800A083EA8E
:106C80001212129B534003F00F030EEB83030DF11E
:106C9000C00E53F8403C1398019983EA1212D24374
:106CA00082EA000303F00F030EEB8303149853F8FA
:106CB000403C83EA121282EA00030DF1C00E03F099
:106CC0000F030EEB8303159853F8403C83EA12122E
:106CD000D24382EA00030DF1C00E03F00F030EEB66
:106CE0008303169853F8403C83EA121282EA0003A9
:106CF0000DF1C00E03F00F030EEB83030DF1C00E78
:106D000053F8403C099883EA1212D24382EA010305
:106D100003F00F030EEB83030DF1C00E53F8403C5C
:106D2000059983EA121282EA000303F00F030EEBC7
:106D30008303029853F8403C83EA1212D24382EA5A
:106D400000030DF1C00E03F00F030EEB83030A984E
:106D500053F8403C83EA121282EA00030DF1C00EA0
:106D600003F00F030EEB83030DF1C00E53F8403C0C
:106D70000B9883EA1212039BD243534003F00F0394
:106D80000EEB83030DF1C00E53F8403C83EA121260
:106D900082EA000303F00F030EEB83030DF1C00E34
:106DA00053F8403C179883EA1212049BD243534095
:106DB00003F00F030EEB83030DF1C00E53F8403CBC
:106DC00083EA121282EA000303F00F030EEB83033F
:106DD0000DF1C00E53F8403C0C9883EA1212D243D6
:106DE00082EA010303F00F030EEB83030DF1C00EE3
:106DF00053F8403C83EA121282EA000303F00F03C7
:106E00000EEB83030DF1C00E53F8403C0D9883EA5E
:106E10001212069BD243534003F00F030EEB830381
:106E20000DF1C00E53F8403C83EA121282EA0003CF
:106E300003F00F030EEB83030DF1C00E53F8403C3B
:106E400007981A9983EA1212D24382EA000303F0E8
:106E50000F030EEB83030E9853F8403C83EA1212A3
:106E600082EA00030DF1C00E03F00F030EEB830363
:106E70000DF1C00E53F8403C199883EA1212189B8A
:106E8000D243534003F00F030EEB83030DF1C00E0A
:106E900053F8403C83EA121282EA000303F00F0326
:106EA0000EEB83030DF1C00E53F8403C1E9883EAAD
:106EB0001212D24382EA010303F00F030EEB8303A5
:106EC0000F9953F8403C83EA121282EA01030DF154
:106ED000C00E03F00F030EEB83030DF1C00E53F849
:106EE000403C1C9983EA12121B9BD243534003F08F
:106EF0000F030EEB830307F1140553F8403C83EABC
:106F0000121282EA010303F00F030EEB8303FE4328
:106F100053F8403C83EA12121D9BD243534003F0C6
:106F20000F030EEB830353F8403C83EA121282EA0C
:106F3000000303F00F030EEB830353F8403C83EA96
:106F40001212D2438BEA020303F00F030EEB83030A
:106F500053F8403C83EA1212089B534003F00F039E
:106F60000EEB830353F8403C83EA1213DB433B7080
:106F700014F8018BA719384614F0E0FB8045414610
:106F8000384601D014F0F4FBAC42F1D145F6442070
:106F90002721C0F2020016F0B7FF4EF24020C2F2E5
:106FA000000031B0BDE8F04F17F0C2BEF0B597B0A9
:106FB00001AD2C4606AE601B14F0C0FB04F8010BBB
:106FC000B442F8D145F28825C0F202050FCD0FC4B6
:106FD0000FCD0FC40FCD0FC495E80F0084E80F004C
:106FE0009DF808609DF809509DF80A409DF80B2017
:106FF0009DF80C309DF80D009DF80E10F7430DF133
:10700000580E07F00F070EEB870757F8407C87F004
:107010007047FF4387EA161606F00F060EEB86064A
:1070200056F8406C86EA1716F64385EA060707F01D
:107030000F070EEB870757F8407C87EA161787EA99
:10704000151606F00F060EEB86069DF80F5056F843
:10705000406C86EA1716F64384EA060707F00F0726
:107060000EEB870757F8407C87EA161787EA141655
:1070700006F00F060EEB86069DF8104056F8406CA1
:1070800086EA1716F64382EA060707F00F070EEBAB
:10709000870757F8407C87EA161787EA121606F02A
:1070A0000F060EEB86069DF8112056F8406C86EA16
:1070B0001716F64383EA060707F00F070EEB87075C
:1070C00057F8407C87EA161787EA131606F00F0672
:1070D0000EEB86069DF8123056F8406C86EA1716BD
:1070E000F64380EA060707F00F070EEB870757F80D
:1070F000407C87EA161787EA101606F00F060EEB9B
:10710000860645F66C2056F8406C86EA1716F6435C
:1071100081EA060707F00F070EEB8707C0F20200AF
:1071200057F8407C87EA161787EA111606F00F0613
:107130000EEB8606132156F8406C86EA1716F643C6
:1071400085EA060707F00F070EEB870757F8407C24
:1071500087EA161686EA151505F00F050EEB85056C
:1071600055F8405C85EA1615ED4384EA050606F0FD
:107170000F060EEB860656F8406C86EA151585EA72
:10718000141404F00F040EEB840454F8404C84EA09
:107190001514E44382EA040505F00F050EEB85059E
:1071A00055F8405C85EA141484EA121202F00F02CA
:1071B0000EEB820252F8402C82EA1412D24383EA88
:1071C000020404F00F040EEB840454F8406C86EAC9
:1071D000121787EA131303F00F030EEB830353F820
:1071E000406C9DF813309DF814509DF815409DF8A3
:1071F000162086EA1716F64383EA060707F00F07FC
:107200000EEB870757F8407C87EA161787EA1316B4
:1072100006F00F060EEB86069DF8173056F8406C08
:1072200086EA1716F64385EA060707F00F070EEB06
:10723000870757F8407C87EA161686EA151505F089
:107240000F050EEB850555F8405C85EA1615ED43F4
:1072500084EA050606F00F060EEB860656F8406C2B
:1072600086EA151585EA141404F00F040EEB840465
:1072700054F8404C84EA1514E44382EA040505F00E
:107280000F050EEB850555F8405C85EA141484EA79
:10729000121202F00F020EEB820252F8402C82EA28
:1072A0001412D24383EA020404F00F040EEB8404A8
:1072B00054F8404C84EA121484EA131303F00F03C9
:1072C0000EEB830353F8403C83EA141416F01CFEC3
:1072D000019D4EF24020002310222946C2F20000F8
:1072E00017F038FD45F680200521C0F2020016F0A7
:1072F0000BFEE4434EF240202146C2F20000002380
:10730000102217F027FDA5421DD14DF6C065C2F22F
:10731000000505F114062C46601B14F00FFA04F862
:10732000010BB442F8D145F6AC20C0F202000F21A7
:1073300016F0EAFD4EF24020C2F2000017B0BDE8A0
:10734000F04017F0F5BC45F688202321C0F202007A
:1073500016F0DAFDFFF758FAECE700BF2DE9F84325
:107360004AF6B609C2F2010945F6BC202DED028BA2
:107370000521C0F2020016F0C7FDB9F8003007EE93
:10738000103A43F23333C4F2233308EE903AB8EEA6
:10739000C77A43F23333C4F2A33308EE103A37EE20
:1073A000287A4EF24024C7EE087AC2F200044AF668
:1073B000B007C2F201074AF6B408C2F201084AF661
:1073C0003406C2F2010640F22C05C2F2010517EEA6
:1073D000900A1CF0BBFB41EC100B0221204617F079
:1073E000F9FC45F6C4200D21C0F2020016F08CFD18
:1073F0003B8807EE903AF8EEE77A77EEA87A87EEC8
:10740000887A17EE100A1CF0A1FB41EC100B022148
:10741000204617F0DFFC45F6D4200821C0F2020018
:1074200016F072FDB8F80010204617F023FC45F660
:10743000E0200C21C0F2020016F066FD31882046E3
:1074400017F018FC45F6F0201421C0F2020016F0E7
:107450005BFD2988204617F00DFC45F60830092110
:10746000C0F2020016F050FD41F23053C2F20103A7
:107470000A2219682046002317F06CFC45F61430E8
:107480000D21C0F2020016F03FFD40F22003C2F2CF
:1074900001030A2219682046002317F05BFC45F619
:1074A00024300921C0F2020016F02EFD41F6A0435F
:1074B000C2F201030A2219682046002317F04AFC91
:1074C00045F630300C21C0F2020016F01DFD80217F
:1074D000204617F0CFFB45F640301021C0F20200E5
:1074E00016F012FD41F6CD43C2F201030A221978CB
:1074F0002046002317F02EFC204617F019FCBDECA7
:10750000028BB9F80030B8F800203B8000233280AD
:107510002B80BDE8F88300BF70B584B0002441F231
:10752000905502940194CDF80B40C2F20105062655
:1075300045F654300221C0F2020016F0E5FC4EF28E
:1075400040203146C2F2000017F094FB45F6B440EB
:107550000221C0F2020016F0D7FC4EF24020C2F227
:10756000000017F0E5FB45F658305621C0F2020046
:1075700016F0CAFC4EF24020C2F2000017F0D8FB11
:107580002B6823444EF2402093F86C110A2200230A
:10759000C2F2000017F0DEFB45F6C8300121C0F250
:1075A000020016F0B1FC2B6823444EF2402093F801
:1075B0006D110A220023C2F2000017F0CBFB45F642
:1075C000C8300121C0F2020016F09EFC2B68234453
:1075D0004EF2402093F86E110A220023C2F20000FE
:1075E00017F0B8FB45F6C8300121C0F2020016F0D2
:1075F0008BFC2B6823444EF2402093F86F110A2233
:107600000023C2F2000017F0A5FB45F6C8300121A7
:10761000C0F2020016F078FC2B6823444EF24020A2
:1076200093F870110A220023C2F2000017F092FBB7
:1076300045F6C8300121C0F2020016F065FC2B6847
:1076400023444EF2402093F871110A220023C2F223
:10765000000017F07FFB45F6C8300121C0F20200A0
:1076600016F052FC2B6823444EF2402093F872111E
:107670000A220023C2F2000017F06CFB45F6C83066
:107680000121C0F2020016F03FFC2B6823444EF2A9
:10769000402093F873110A220023C2F2000017F071
:1076A00059FB45F6B0300821C0F2020016F02CFC60
:1076B0002B6823444EF2402093F874110A220023D1
:1076C000C2F2000017F046FB45F6BC300D21C0F2B7
:1076D000020016F019FC2B6823444EF2402093F868
:1076E00075110A220023C2F2000017F033FB45F6A1
:1076F000BC300D21C0F2020016F006FC2B682344BA
:107700004EF240200A2293F87611C2F200000023C4
:1077100017F020FB4EF24020C2F2000017F008FBE9
:1077200045F6CC305C21C0F2020016F0EDFB4EF2C3
:107730004020C2F2000017F0FBFA45F62C4006216B
:10774000C0F2020016F0E0FB2B6823444EF240200A
:1077500093F877110A220023C2F2000017F0FAFA18
:1077600045F6C0300921C0F2020016F0CDFB2B68AF
:1077700023444EF2402093F878110A220023C2F2EB
:10778000000017F0E7FA45F6C0300921C0F2020008
:1077900016F0BAFB2B6823444EF2402093F879117F
:1077A0000A220023C2F2000017F0D4FA45F6B030E6
:1077B0000821C0F2020016F0A7FB2B6823444EF20A
:1077C000402093F87A110A220023C2F2000017F039
:1077D000C1FA45F6C4300521C0F2020016F094FB50
:1077E0002B6823444EF2402093F87B110A22002399
:1077F000C2F2000017F0AEFA45F62C400621C0F2A6
:10780000020016F081FB2B6823444EF2402093F8CF
:107810007C110A220023C2F2000017F09BFA45F601
:107820002C400621C0F2020016F06EFB2B682344A8
:107830004EF2402093F87D110A220023C2F200008C
:1078400017F088FA45F6B4300421C0F2020016F0B1
:107850005BFB2B6823444EF2402093F87E110A22F2
:107860000023C2F2000017F075FA45F6C430052176
:10787000C0F2020016F048FB2B6823444EF2402071
:1078800093F87F110A220023C2F2000017F062FA77
:1078900045F6C4300521C0F2020016F035FB2B6816
:1078A00023444EF2402093F880110A220023C2F2B2
:1078B000000017F04FFA4EF240201534C2F20000DB
:1078C00017F036FA7E2C06F1FF367FF431AE45F61E
:1078D00034402D21C0F2020016F016FB4EF240207B
:1078E000C2F2000017F024FA45F6C830C0F20200D8
:1078F000012116F009FB2B6823444EF2402093F837
:107900006C110A220023C2F2000017F023FA45F698
:1079100030400134C0F20200022141F2905616F0CC
:10792000F3FA862CC2F20106E5D14EF24020C2F2F3
:10793000000017F0FDF945F664400521C0F2020091
:1079400016F0E2FA33684EF2402093F8F2110A2260
:107950000023C2F2000017F0FDF94EF24020C2F2FF
:10796000000017F0E5F945F66C400421C0F2020072
:1079700016F0CAFA33684EF2402093F8F3110A2247
:107980000023C2F2000017F0E5F94EF24020C2F2E7
:10799000000017F0CDF945F674400521C0F2020051
:1079A00016F0B2FA33684EF2402093F8F4110A222E
:1079B0000023C2F2000017F0CDF94EF24020C2F2CF
:1079C000000017F0B5F945F67C400921C0F202002D
:1079D00016F09AFA33684EF2402093F8F5110A2215
:1079E0000023C2F2000017F0B5F94EF24020C2F2B7
:1079F000000017F09DF945F688400921C0F2020009
:107A000016F082FA33684EF2402093F8F6110A22FB
:107A10000023C2F2000017F09DF94EF24020C2F29E
:107A2000000017F085F945F694400921C0F20200E4
:107A300016F06AFA33684EF2402093F8F7110A22E2
:107A40000023C2F2000017F085F94EF24020C2F286
:107A5000000017F06DF945F6A0400921C0F20200C0
:107A600016F052FA33684EF2402093F8F8110A22C9
:107A70000023C2F2000017F06DF94EF24020C2F26E
:107A8000000017F055F945F6AC400A21C0F202009B
:107A900016F03AFA33684EF2402093F8F9110A22B0
:107AA0000023C2F2000017F055F94EF24020C2F256
:107AB000000017F03DF945F6B8400D21C0F2020074
:107AC00016F022FA33684EF2402093F8FA110A2297
:107AD0000023C2F2000017F03DF94EF24020C2F23E
:107AE000000017F025F945F6C8400921C0F2020050
:107AF00016F00AFA33684EF2402093F8FB110A227E
:107B00000023C2F2000017F025F94EF24020C2F225
:107B1000000017F00DF945F6D4400921C0F202002B
:107B200016F0F2F933684EF2402093F8FC110A2265
:107B30000023C2F2000017F00DF94EF24020C2F20D
:107B4000000017F0F5F845F6E0400621C0F202000B
:107B500016F0DAF931680A2201F2FD1101A81DF0D0
:107B60007DF845F6F4100121C0F2020016F0CCF9C0
:107B700001A81DF005F8014601A816F0C5F945F267
:107B8000D8700121C0F2020016F0BEF94EF240207A
:107B9000C2F2000017F0CCF89B244EF240200023E4
:107BA0000A222146C2F2000017F0D4F845F6B4408C
:107BB0000221C0F2020016F0A7F92B6823444EF20E
:107BC000402093F86C110A220023C2F2000017F043
:107BD000C1F84EF240200134C2F2000017F0A8F8BC
:107BE000AD2CDAD14EF24020C2F2000017F0A0F81E
:107BF00004B070BD2DE9F0412DED028B41F66060BF
:107C000086B0C2F2010013F0FFFB41F66060C2F2E1
:107C1000010013F075FA41F66060C2F2010013F042
:107C200067FA41F66060C2F2010013F0FFF841F616
:107C30006060C2F2010013F06BFA41F66060C2F2BC
:107C4000010013F06DFA41F66060C2F2010013F01A
:107C500047FA45F6E843C0F2020393E80700002420
:107C60004FF020376B46029703940494CDF80B70C5
:107C70008DF8144003C341F660601A802146224605
:107C8000C2F2010013F008FA68461CF079FF0246C0
:107C900041F660606946C2F2010016F0D5FF4EF26F
:107CA000402023460A222146C2F2000017F052F873
:107CB00045F604200121C0F2020016F025F94EF22B
:107CC000402023460A222146C2F2000017F042F863
:107CD00045F6F4400321C0F2020016F015F968469B
:107CE0001CF04EFF0146684616F00EF945F2D870BA
:107CF0000121C0F2020016F007F945F6F8464EF2EF
:107D00004020C0F20206C2F2000017F011F896E817
:107D10000300009041F66060019722468DF8041040
:107D2000C2F201000B21029703940494CDF80B706A
:107D30008DF8144013F0B0F968461CF021FF02469C
:107D400041F660606946C2F2010016F07DFF4EF216
:107D5000402023460A222146C2F2000016F0FAFF14
:107D600045F604200121C0F2020016F0CDF84EF2D3
:107D7000402023460A220B21C2F2000016F0EAFF3F
:107D800045F6F4400321C0F2020016F0BDF8684643
:107D90001CF0F6FE0146684616F0B6F845F2D870BB
:107DA0000121C0F2020016F0AFF84EF24020C2F2FC
:107DB000000016F0BDFF45F60053C0F202030FCBE2
:107DC0008DE80F0041F6606021460122C2F20100F9
:107DD00004948DF8144013F05FF968461CF0D0FE4F
:107DE000024641F660606946C2F2010016F02CFFBF
:107DF0004EF2402023460A220121C2F2000016F072
:107E0000A9FF45F604200121C0F2020016F07CF81B
:107E10004EF240200A2223462146C2F2000016F00C
:107E200099FF45F6F4400321C0F2020016F06CF809
:107E300068461CF0A5FE0146684616F065F845F256
:107E4000D8700121C0F2020016F05EF84EF2402018
:107E5000C2F2000016F06CFF0221042014F02EF98B
:107E600002211E2014F02AF9DC2014F08BF945F6CB
:107E700014503421C0F2020016F046F84EF24020B1
:107E8000C2F2000016F054FF45F64C502E21C0F20D
:107E9000020016F039F84EF24020C2F2000016F04F
:107EA00047FF45F67C502921C0F2020016F02CF85D
:107EB0004EF24020C2F2000016F03AFF45F6A850FC
:107EC0000921C0F2020016F01FF80521304616F015
:107ED0001BF84EF24020C2F2000016F029FF45F6D2
:107EE000B4500D21C0F2020016F00EF84EF2402000
:107EF000C2F2000016F01CFFFFF758F8FCF79EFCDA
:107F00004EF28813CEF20003012740F2002040F227
:107F10009855C2F201051F604FF4E171C1F6FF7080
:107F200016F06AF928460BF0EFFA28460AF03CFEF4
:107F3000EA88242122F0100228460AF001FCEA888F
:107F4000242122F4807228460AF0FAFB28460AF01F
:107F5000ABFDF6EE000AB0EE600A28460BF0CEF854
:107F60004CF6CD461D2128460AF00EFFC3F64C56AE
:107F700028460BF021F901EE106A4DF20A76C3F69D
:107F8000234600EE906A46F26666C3F666763B4686
:107F900000EE106A3A46394628460BF055F9284655
:107FA0000AF07EFC28460AF0FDFC02220721284642
:107FB0000AF070FE28460AF0F1FB4CF6CD43C3F6FA
:107FC0004C63022200EE903AB7EE000A394628468A
:107FD0000AF05EFF45F6C4501B21C0F2020015F006
:107FE00093FF4EF24020C2F2000016F0A1FE4DF6C3
:107FF000D860C2F200000B210CF04CFC4DF6D860AA
:10800000C2F200000D210CF0ADFC49F21400C2F2E6
:108010000100FE210CF0E4FD002840F0A18045F6AF
:10802000E0501721C0F2020015F06EFF4EF2402022
:10803000C2F2000016F07CFE45F6F853C0F20203CF
:1080400093E8030041F6A44241F65463C2F20102F0
:10805000C2F2010382E8030083E803004DF6C06624
:10806000C2F2000641F6F044C2F20104002301EE20
:10807000903A237800EE103A0023C4F2964302EEC1
:10808000103A0023C4F2482301EE103AB8EE400A39
:10809000F0EE610A01F09CFEB5EEC00AF1EE10FAB6
:1080A00000F1348347F67903C4F2302307EE103A27
:1080B000F6EE007AE0EE077A49F68073C0F201032B
:1080C000FCEEE77A17EE902A9A4240F222831A4693
:1080D0004FF4507140F22073C2F20103187EC507BD
:1080E00000F12481DD8B1A62A94240F0010088BFB3
:1080F000D9831876237800EE103A002301EE903AE7
:1081000041F284440023C4F20C23C2F2010401EEC4
:10811000103AB8EE400A4FF48033F0EE610AB7EE41
:10812000002AA36101F054FE4FF47E43C4F2FF63C2
:1081300007EE903AB4EEE70AF1EE10FA00F3BC80D5
:108140004FF47E43CCF2FF6307EE903AB4EEE70AB9
:10815000F1EE10FA40F1D3820023C8F20103AEE041
:1081600045F600600E21C0F2020015F0CDFE4EF281
:108170004020C2F2000016F0DBFD4DF6C06641F271
:108180005C53C2F20103C2F200061F7008F0C0FA8D
:10819000327941F6CC4EC2F2010E02EB420340F2BC
:1081A000300802EB8302C2F2010841F6A4418EF8C6
:1081B0000000C2F2010108EB020008F037F9307943
:1081C00008F052F945F610600621C0F2020015F0E1
:1081D0009BFE337903EB430503EB850308EB0305B3
:1081E00028461CF0CDFC0146284615F08DFE45F6CC
:1081F00004203946C0F2020015F086FE41F6A44084
:10820000C2F201001CF0BCFC014641F6A440C2F2DF
:10821000010015F079FE45F2D8703946C0F202002F
:1082200015F072FE4EF24020C2F2000041F6F44515
:1082300016F07EFDC2F201052FE045F6186003211D
:10824000C0F2020015F060FE4EF2402000230A2228
:108250002146C2F2000016F07DFD45F6F410012122
:10826000C0F2020015F050FE28461CF089FC0146C1
:10827000284615F049FE45F2D8700121C0F20200EF
:1082800015F042FE4EF240200134C2F2000016F01A
:108290004FFD202C05F10B0509D0092CCDD845F652
:1082A000C8300121C0F2020015F02EFEC5E7717939
:1082B000307908F0C1FBD5E60023C7F6FF7341F61D
:1082C0007465C2F20105002201EE902A2A78E3616A
:1082D00000EE102A0022C4F2482201EE102AB8EE65
:1082E000400AF0EE610AB7EE002A01F071FD4FF48A
:1082F0007E43F7EE007AC4F2FF6337EEC00A07EE62
:10830000903AB4EEE70AF1EE10FA19DC4FF47E432E
:10831000CCF2FF6307EE903AB4EEE70AF1EE10FA02
:1083200040F1E6810023C8F201030CE01D6AAA4275
:1083300040F29481D88B1A62814288BFD983D9E6F2
:108340000023C7F6FF732A7800EE102A002201EE00
:10835000902A41F2BC440022C4F24822C2F2010435
:1083600001EE102AB8EE400AF0EE610AB7EE002ADC
:10837000A36101F02DFD4FF47E43C4F2FF6307EECD
:10838000903AB4EEE70AF1EE10FA0FDC4FF47E43B8
:10839000CCF2FF6307EE903AB4EEE70AF1EE10FA82
:1083A00040F155810023C8F2010302E00023C7F623
:1083B000FF732A78E36100EE102A002201EE902A72
:1083C0000022C4F2482201EE102AB8EE400AF0EE74
:1083D000610AB7EE002A01F0FBFC4FF47E43C4F2C1
:1083E000FF6307EE903AB4EEE70AF1EE10FA0FDC05
:1083F0004FF47E43CCF2FF6307EE903AB4EEE70A07
:10840000F1EE10FA40F11C810023C8F2010302E0F2
:108410000023C7F6FF7341F6F14140F21C02C2F29D
:108420000101C2F2010209781278236207EE901A64
:1084300007EE102A0022C4F2C82208EE102AF8EE35
:10844000677AB8EE477AC7EE886A41F29053F268CD
:10845000C2F201031B68C7EE087AB7EE007A77EE26
:10846000666A77EE677A00EE902AB268C3ED596AC1
:1084700083ED5A7AC3ED587A00EE102AFDF7A4FC7A
:108480000023C4F22C2307EE903A002306EE903A24
:10849000B36807EE103A27EE087A27EE277AC7EE80
:1084A000087A77EEA67AFDEEE77A17EE903A9B000F
:1084B00072B641F2F444C2F20104E36062B6237C76
:1084C000012B40F22B8172B6E36862B640F22402BF
:1084D000002BC2F20102B8BF03339B101360737903
:1084E00072B69B00236262B694F82430012B40F2EE
:1084F0001A8172B6236A62B640F22402002BB8BF1A
:108500000333C2F2010241F6D0409B10C2F20100D7
:10851000536012F02BFC41F6E040C2F2010012F071
:1085200025FC4AF6B6044AF6B401C2F20104C2F2CE
:1085300001014AF6B0024AF63403C2F20102C2F265
:10854000010345F61C6025880C8815801821C0F2AF
:1085500002001C8015F0D8FC4EF2402000230A22B5
:108560003179C2F2000016F0F5FB45F60420012136
:10857000C0F2020015F0C8FC4EF2402000230A228F
:108580007179C2F2000016F0E5FB45F2D8700121C6
:10859000C0F2020015F0B8FC4EF24020C2F200001A
:1085A00016F0C6FBFEF7B8FF45F638601421C0F29E
:1085B000020015F0A9FC4EF240208021C2F200001A
:1085C00016F058FB45F650601121C0F2020015F07C
:1085D0009BFC4EF2402040F65A31C2F2000016F0E9
:1085E00049FB45F664600321C0F2020015F08CFCE3
:1085F0004EF24020C2F2000016F09AFBFEF7AEFEEB
:1086000041F66060C2F2010012F08AFD01F020FE26
:108610004EF20813CEF20003012245F668601A609C
:108620000B21C0F2020015F06FFC4EF24020C2F2A6
:10863000000016F07DFB06B0BDEC028BBDE8F081BA
:10864000F0EE407AFEEEC87A17EE903AE3E6F0EEEE
:10865000407AFEEEC87A17EE903AAAE602F17F0160
:10866000C909013100291A620A4638BF002287076A
:1086700006D5596A7F31C90901318A4238BF0A4695
:10868000450706D5996A7F31C90901318A4238BF49
:108690000A46010706D5D96A7F31C90901318A42E4
:1086A00038BF0A46C70606D5196B7F31C9090131A3
:1086B0008A4238BF0A46850606D5596B7F31C909FB
:1086C00001318A4238BF0A46410606D5996B7F318F
:1086D000C90901318A4238BF0A46C10906D0D96B9F
:1086E0007F31C90901318A4238BF0A46DA8301E580
:1086F000F0EE407AFEEEC87A17EE903A23E6F0EEFE
:10870000407AFEEEC87A17EE903AD8E501210022B1
:10871000E0E402F17F01C9090131DBE472B62046D1
:10872000FCF7E0FBD0E672B641F20850C2F201005D
:10873000FCF7D8FBDEE600BF2DE9F0479DF82040AE
:10874000013CE4B20F2C03D84EB2002E0D4601DBE3
:10875000BDE8F087E0290FD9F729F9D90835EDB23E
:10876000012303FA05F515F0DD0FF1D0806C0368E5
:10877000BDE8F0471B6818478146806C1F460368B8
:1087800046EA0401C9B21B6890469847D9F84800E8
:10879000036808F07F011B6805F0EF059847C02DBE
:1087A000D6D0D9F84800036807F07F011B68BDE800
:1087B000F0471847F8B50446806C03681B69984772
:1087C00008B90020F8BDA06C03685B699847C3B284
:1087D00003F0FB01F929F4D0A26D82B994F84D2081
:1087E00084F84F30150600F19C8040B20028C0F29A
:1087F0005081002084F84D00A0656065F8BD010639
:1088000067D494F84F10F02904EB020140D081F8AE
:108810004F30616D4B1E9A4240D394F84F20F02A9E
:10882000E7D013063DD4002384F86630B02B4CD03B
:10883000A02B4AD0D02B48D0E02B46D0C02B44D020
:10884000002094F8505084F86750032908BF94F82A
:10885000515084F8650018BF002500210120B02B7D
:1088600084F86850A165616584F8E90000F0B5807E
:1088700000F2AC80902B00F0B080A02B00F0AD8017
:10888000802B00F0AA80002384F84D300120F8BD31
:1088900081F86930636D013B9A42AAD20132A26528
:1088A0008FE702F10C03DBB2012BBCD902F0FB0312
:1088B000F92BB8D0EF2A00F2DB8002F0F003802B16
:1088C00084F8663001D0902BB0D102F00F00013057
:1088D000B7E7A3F1F701082993D8012505FA01F0BC
:1088E00010F4DD7F40F0968000298AD194F8693039
:1088F000F02B7FF47EAF561C2244F720370A82F813
:10890000690084F8676084F8687084F8651084F8FA
:108910004D10284684F8663084F8E950A1656165F9
:10892000F8BD02F10C05EEB2012E7FF65EAF02F04B
:10893000FB0EBEF1F90F3FF458AFEF2A2DD802F02D
:10894000F007802F2AD140B20028FFF64FAF012157
:1089500084F84F2084F85030A165EDB2012D7FF6E8
:1089600048AFBEF1F90F3FF444AFEF2A5FD802F0F1
:10897000F003B02B26D01ED9D02B04D0E02B21D071
:10898000C02B7FF436AF022363650121A36D9942AA
:1089900027D90133A3650020F8BD174607F0DF068D
:1089A000902ED0D007F0BF06A02ECCD007F0EF0756
:1089B000C02FC8D019E7902B04D0A02B02D0802B59
:1089C0007FF417AF032363650221DFE7D02B04D0C8
:1089D000E02B02D0C02B7FF456AF84F84D2001204D
:1089E000F8BDEF2A94BF02F0F005154602F00F0221
:1089F0000023013294F8501084F86520012084F897
:108A0000671084F8683084F86650A365636584F85D
:108A1000E900F8BD002284F8672084F8682084F813
:108A2000652084F8663084F8E9502846F8BDF62AB7
:108A30000FD007D8F12AA6D01CD9F22AC2D0F32A27
:108A4000A1D0D6E6FC2A21D8FA2A02D2F82A7FF44D
:108A5000D0AE0023012084F8653084F8673084F8B4
:108A6000683084F86620A365636584F8E900F8BD82
:108A70001346D9E6F02A7FF4BCAE8021002361655D
:108A800084F8692084F84D307F217FE7FE2AE0D208
:108A9000AFE61A468E4603F10C055EE790F86630A5
:108AA000F12B7CD00ED9FA2B2BD01FD8F32B38D03A
:108AB000C0F08180F62B7AD0F82B40F08B80036BCE
:108AC000F3B11847B02B6ED031D9D02B21D03ED97D
:108AD000E02B42D0F02B7ED1C3698BB1B0F8671088
:108AE000802900F1690028BF80211847FC2B0CD099
:108AF00051D3FE2B4BD0FF2B6BD1436C002BE0D11D
:108B00007047436B002BDCD1FAE7C36B002BD8D145
:108B1000F6E74369002BF3D090F8671090F86500F2
:108B20001847836A002BEBD090F867001847902B0A
:108B300029D0A02B23D0802BE2D10368002BDFD0DB
:108B400090F8682090F8671090F865001847C02BDF
:108B500042D10369002BDFD1D2E78269002ACFD04E
:108B600090F8681090F8673090F86500C90101F43A
:108B70007E5103F07F031943A1F50051104783682C
:108B8000002BDDD1BCE74368002BD9D1B8E7036CDB
:108B9000002B96D1B4E7836B002B92D1B0E7036A28
:108BA000002BC1D1ACE7C368002BC9D1A8E7C36AC9
:108BB000002B86D1A4E7426A002AA1D090F8683041
:108BC00090F86700DB0103F47E5300F07F00184348
:108BD0001047704770477047704700BF90F8643087
:108BE000DA0725D513F0FE0F22D070B590F8665045
:108BF00085F08002602A82B004461AD9F62D6ED024
:108C000067D8F12D7ED04FD9F22D2DD0F32D1AD16A
:108C1000806C94F86760036829461B689847A06CCD
:108C20000368DB6C06F07F0102B0BDE870401847B6
:108C3000704790F865608E4207D031B15B08012B18
:108C400008D0032B27D002B070BD5B08012B01D0E8
:108C5000022BF8D194F8683094F8672000962946E2
:108C60002046FFF769FDEEE7806C94F867300268F4
:108C700094F868601268294643EAC6159047A06CCC
:108C8000036805F07F019B6C9847A06C0368C5F3EF
:108C9000C6119B6CC8E794F8683094F8672000967A
:108CA0002946FFF749FDCEE7F02DCCD1B0F867603B
:108CB000802E28BF802600F16905002EC3D02E44E7
:108CC000A06C15F8011B03681B689847AE42F7D1EA
:108CD000B9E7FC2D26D8FA2D01D2F82DB3D105F134
:108CE0000803DBB2072BAED8012202FA03F313F01C
:108CF000DD0FA8D0A06C03681B68294602B0BDE850
:108D000070401847806C94F8672094F868300668C3
:108D10001201294603F00F0302F0700532681D436B
:108D20009047E7E7FE2D8ED3D9E700BFF0B540F2BC
:108D3000D05087B0C2F201000BF07AFC002840F05E
:108D4000FE804AF28C64C2F2010441F6706223682C
:108D50000193C2F20102019B116841F287325B1A52
:108D6000934206D941F6CD43C2F201031B78002B92
:108D700043D041F67865C2F2010595F84C60102E9B
:108D80004CD9002014F0D8FC10F018FE41F2C0506D
:108D90000021C2F2010011F003FD41F25853226894
:108DA0000292C2F20103029A1868121A4AF28C6106
:108DB000322AC2F201014ED841F28C532268049249
:108DC000C2F20103049A1968521A632A00F2B280AF
:108DD00040F2B06322680592C2F20103059A196855
:108DE00041F28730521A824205D901F59C5108316F
:108DF0001960FEF7B3FA07B0F0BD40F2CC53C2F2EF
:108E000001031B78002BB4D041F67865C2F201054E
:108E1000FDF7FAFC95F84C60102EB2D82846FFF703
:108E2000C9FC0028ADD095F86630902B00F00B817E
:108E300083F08003602B40F2098141F67860C2F232
:108E40000100FFF72BFE41F678603146C2F20100C7
:108E5000FFF7C4FE95E741F290560A680392C2F20A
:108E6000010641F26055039A30681A60C2F20105AA
:108E700006F0A2FE41F6CD43C2F20103AA881870A3
:108E8000002A40F03D8140F24455C2F20105AB8812
:108E9000002B40F0ED8040F2F065C2F20105AB8896
:108EA000002B89D03268D2F8601107EE901A296839
:108EB00007EE101A77EE877A45F6EC60C2ED587A25
:108EC000013BC0F20200AB80F7F76CFD3368D3F8CA
:108ED00060011AF03BFE41EC100B4EF240200521E0
:108EE000C2F2000015F076FF45F6FC60C0F2020009
:108EF000F7F758FD4EF24020A988C2F2000015F0A5
:108F0000B9FE45F61470C0F20200F7F74BFD286871
:108F10001AF01CFE41EC100B4EF240200521C2F26B
:108F2000000015F057FF4EF24020C2F2000015F08D
:108F3000FFFE41E76431196003F0EAFA48E740F2C6
:108F4000A454C2F2010413F0F5F82368C01AB0F576
:108F5000356F7FF6F6AE13F0EDF8206040F2D0509A
:108F6000C2F201000BF074FB044613F0E3F841F287
:108F70009053C2F20103054622461868802106F08C
:108F80000FF813F0D7F840F65A33401B984252D8E6
:108F900040F22C0413F0CEF8C2F20104401B2388E7
:108FA000834260D372B640F2A853C2F201031A7F23
:108FB00002F0FF010AB100221A7762B6A1B372B6BD
:108FC00047F6FF744FF40040B3F91E50B3F9202068
:108FD000DC83188462B685EAE57182EAE273A3EB6A
:108FE000E273A1EBE5718B42B8BF0B4607EE903AF6
:108FF0004FF47E43C4F2FF6306EE103AF8EEE77AD0
:1090000047F2A403C7EE866AC3F67D7307EE103AF3
:10901000F4EEC76AF1EE10FA06DD41F6A043C2F2A3
:1090200001031A6801321A6040F2D050C2F2010006
:109030000BF020FB85E641F23053C2F201031A68BF
:1090400001321A60A4E795F8683043B195F86530AD
:109050009E423FF4F2AE002E3FF4EFAEF3E68023E3
:1090600085F86630F2E713F065F8401B208099E739
:109070003268D2F8641107EE901A296807EE101AC8
:1090800077EE877A45F6A060C2ED597A013BC0F2CF
:109090000200AB80F7F786FC3368D3F864011AF05E
:1090A00055FD41EC100B4EF240200521C2F20000AC
:1090B00015F090FE45F6B460C0F20200F7F772FCBE
:1090C0004EF24020A988C2F2000015F0D3FD45F60B
:1090D000D060C0F20200F7F765FC28681AF036FD90
:1090E00041EC100B4EF240200521C2F2000015F0B9
:1090F00071FE4EF24020C2F2000015F019FECAE6E1
:109100004DF6C067C2F20007013AFB68AA8000EE84
:10911000903ABB6807EE903A2B6807EE103A37EEAC
:10912000870AFCF751FE45F67460C0F20200F7F7BB
:1091300039FCB8681AF00AFD41EC100B4EF24020E1
:109140000521C2F2000015F045FE45F68060C0F230
:109150000200F7F727FC4EF24020A988C2F2000077
:1091600015F088FD45F69060C0F20200F7F71AFC92
:1091700028681AF0EBFC41EC100B4EF24020052160
:10918000C2F2000015F026FE4EF24020C2F20000AE
:1091900015F0CEFD77E600BF2DE9F04F41F678657A
:1091A000C2F201058DB012F077FA95F86430002410
:1091B00001264EF2202743F001034FF6FF7E66F3AF
:1091C0004703214685F8654085F8664085F8674085
:1091D00085F8684085F8E940C2F2000705F16900AA
:1091E0008022C5F85CE0C5F860E085F86430AF64C3
:1091F00085F84C4085F84D4085F84E406C65AC656F
:109200001BF08EFB4DF6A02240F695112846C2F2C7
:109210000002C0F2000141F2C057C2F201072C6007
:109220006C60AC60EC602C616C61AC61EC612C62D8
:109230006C62AC62EC622C636C63AC63EC632C64B8
:109240006C641BF01FF846F64022C0F2020207F5DC
:109250009B6307F5B36107F5A36007F5AB653A605B
:109260007B61402250237C60BC60B861FD61384660
:1092700079627A85BB8511F057F941F6606845F24D
:109280005C23C2F20108C0F202033B6010220223F9
:109290002721404611F0BAFD41F2F44045F278230F
:1092A000C0F2020302220321C2F20100C8F800301A
:1092B000FCF782FA41F208501D221C21C2F2010083
:1092C000FCF77AFA4AF28C6341F6D040C2F201030D
:1092D00014220421C2F201001D46029311F02EFD5A
:1092E00041F6E04014221E21C2F2010011F026FDD9
:1092F0002B68069341F28C53C2F2010340F2D0591D
:10930000C2F20109069A1A602146224640F2A85B81
:109310004846FBF767FAC2F2010B46F6D003C0F2EB
:1093200002030BF118023146584689F89C40C9F8EF
:10933000984089F89D40C9F8003040F22075FBF74D
:1093400051FA4FF40041C2F2010547F6FF7246F6AA
:109350007803ABF8201045F25021C0F20203ABF8BD
:109360001E20C0F2020105F55462CBF800302C72C9
:109370002346EC6020466E722A6129602C4600E08C
:10938000226942F82300697A013340F2207299423F
:10939000C2F20102F4DC4AF63003C2F20103039385
:1093A000196809B9A8E219464B69002BFBD14D6138
:1093B0004FF00004002141F2844846F6A00340F239
:1093C0006070C2F20108C0F2020369614FF450629A
:1093D000AC80EC80AC722C76C2F201004FF000043D
:1093E0002B606C83AC83EC831BF09AFA08F12802A3
:1093F00004214046FBF7F6F94FF4803341F2644410
:1094000041F2BC47C2F20107C8F81830C8F81C3056
:10941000C8F82030C8F82430059341F2345623466A
:1094200046F6B80AC2F20106C2F20103C0F2020A0D
:1094300007F12802042138461C46C8F800A004930E
:10944000FBF7D0F9059B019606F11C02304601217D
:10945000C7F800A0BB61FB613B627B62FBF7C2F90E
:10946000019B46F6AC0A9E462246059BCEF8183074
:10947000C0F2020A1C320121204640F24C56CEF8BE
:1094800000A0FBF7AFF9059BA361C2F2010645F20C
:109490005023C0F2020306F11801002202203360BB
:1094A0004FF000033372707231610B46C4F800A0B4
:1094B000F2601146304600E0036943F82210747AE6
:1094C000013240F24C539442C2F20103F4DC039A9D
:1094D00012684AF63001C2F201010AB90EE21A46D8
:1094E0005369002BFBD15661002440F24C5040F2EE
:1094F000746A46F60453C0F20203C2F2010A7461B0
:10950000B480F480B472C2F20100336015F06EFFD3
:1095100050468AE8000A8AF808408AF80940CAF8E2
:109520000C408AF8104040F2886B14F0C3FF4DF6EF
:10953000A02240F69911C2F2010BC2F20002C0F261
:10954000000150461AF09EFE5846CBF80090CBF82A
:1095500004808BF808408BF80940CBF80C408BF85E
:10956000104040F29C6A14F0A5FF4DF6A02240F690
:109570009911C2F2010AC2F20002C0F2000158467B
:109580001AF080FE5046CAF800908AF808408AF81F
:109590000940CAF80C408AF81040CAF8047041F239
:1095A0001C5914F087FF4DF6A02240F69911C2F223
:1095B0000109C2F20002C0F2000150461AF062FE38
:1095C0004FF0010B484689E8200189F80840C9F8A6
:1095D0000C4089F8104089F809B040F2B46A14F0E0
:1095E00069FF4DF6A02240F69911C2F2010AC2F2BB
:1095F0000002C0F2000148461AF044FE0223504621
:109600008AF8093005938AE8A0008AF80840CAF869
:109610000C408AF8104040F2C86914F04BFF4DF638
:10962000A02240F69911C2F20109C2F20002C0F272
:10963000000150461AF026FE4846C9F80080C9F8D5
:10964000045089F8084089F80940C9F80C4089F8A5
:10965000104040F2DC6514F02DFF4DF6A02240F6DC
:109660009911C2F20105C2F20002C0F2000148469F
:109670001AF008FE2846C5F800802C72EC602C74A5
:109680006F6085F809B041F2945814F013FF4DF65D
:10969000A02240F69911C2F20108C2F20002C0F203
:1096A000000128461AF0EEFD019BC8F80430404640
:1096B00088F8084088F80940C8F80C4088F810403D
:1096C000C8F8007040F2F86514F0F4FE4DF6A022E0
:1096D00040F69911C2F20105C2F20002C0F2000187
:1096E00040461AF0CFFD049B6B6028462C726C72CA
:1096F000EC602C742F6040F20C7814F0DBFE4DF619
:10970000A02240F69911C2F20108C2F20002C0F292
:10971000000128461AF0B6FD4046C8F8046088F8F3
:10972000084088F80940C8F80C4088F81040C8F88C
:10973000007040F2705514F0BDFE4DF6A02240F6C8
:109740009911C2F20105C2F20002C0F200014046C6
:109750001AF098FD28466E602C72EC602C7485F827
:1097600009B02F6041F2685614F0A4FE4DF6A02215
:1097700040F69911C2F20106C2F20002C0F20001E5
:1097800028461AF07FFD059B737245F2502306F1BF
:109790001801C0F20203224633603472F46020469E
:1097A00031610B46344600E0236943F82200717AA8
:1097B000013241F268539142C2F20103F4DC039A90
:1097C00012684AF63001C2F201010AB998E01A465D
:1097D0005369002BFBD15661002441F2685046F6D4
:1097E000C403C0F202037461B480F480B472C2F2A4
:1097F000010040F28457C2F2010733600AF096FD7F
:10980000019B3C72384687E848007C72FC603C74DF
:1098100014F050FE4DF6A02240F69911C0F200015E
:109820003846C2F2000241F6B8451AF02BFDC2F2EA
:109830000105049A2C720123284685E844006B72C6
:10984000EC602C7414F036FE4DF6A02240F699110F
:10985000C0F200012846C2F200021AF013FD40F2E5
:109860009853C2F2010346F68402C0F202021A6063
:109870004FF419700A221A7215F0C8FB4AF64441D7
:10988000064605F00FF9029F3B680793079D3B686A
:109890000893089C3B68099341F29050C2F2010082
:1098A00041F6706140F2706241F6B443C2F20101C8
:1098B000C2F20102C2F20103066009980D60146051
:1098C000186012F037FC029F3B680A930A9D3B68C0
:1098D0000B9340F2A45141F2585240F2B063C2F2ED
:1098E0000101C2F20102C2F201030B9C0860156083
:1098F0001C600DB0BDE8F08F1A6059E50B60F3E510
:109900000B6069E74FF07E52002141670267826772
:10991000704700BF70B507EE901A2DED048BB8EEBE
:10992000E79AB7EE008A88EE097A4FF46043C4F2F2
:109930002B73002500260446866305638561C56197
:10994000C56085604560056007EE903A80ED057A58
:1099500087EE897A0562456380ED049A17EE100A56
:109960001AF0F4F841EC100B17F0CAFB51EC100B95
:109970001AF038FC49F6AB03C3F6B44308EE900A7C
:1099800007EE903A68EEA77A40F6DB7388EE277A06
:10999000C4F2490306EE903A2369C4ED097A05EE54
:1099A000903AB6EE006ABAEE040AA5EE860A63693A
:1099B00007EE903A20EE260A84ED0A7A20EE270A76
:1099C00017F04CF94BF60B43C3F6324307EE103A4F
:1099D0000023C4F2FC2307EE903A68EE878A87EEF4
:1099E000897A012323660023CBF6807384F85460C0
:1099F0006566A566E364A364C8EE287A38EE478AF4
:109A0000C4ED168A84ED1B8ABDEC048B84ED0B0A31
:109A1000C4ED177A70BD00BFF8B50B6806EE903A3A
:109A2000436E07EE903AC36E07EE103A836E76EE01
:109A3000E77A06EE103AE7EE067A02F18047012A4D
:109A40002DED108B07F1FF37C1ED007AC0ED196ADB
:109A500019DD01EB87040B465D6807EE905A37EE7F
:109A6000E67A06EE905AC56E06EE105A1D6805EEAF
:109A7000905AA6EE257A17EE105A43F8045FA342D7
:109A8000C0ED197AE8D1846FBF0007EE904ACB1978
:109A9000B7EE007AF4EE477A1B688366F1EE10FAAF
:109AA00011D0002A0FDD3C1D0C440B4602E0856FEF
:109AB00007EE905A1D6807EE105A67EE277AE3EC1E
:109AC000017AA342F3D1036F07EE903AB7EE007A22
:109AD000F4EE477AF1EE10FA00F0FB80C36C07EE6B
:109AE000103A436FF4EE477AF1EE10FA16460D463F
:109AF000044600EE103A40F0EF80836C07EE903A97
:109B0000B4EE670AF1EE10FA40F0E680C36B0CEE9B
:109B1000903AF7EE00BA3CEEABDA002E8CEE8DBA3E
:109B200040F3D78040F6DB73C4F249030437A66BD9
:109B30002F440AEE103A2BEE0B8A46F26663C3F608
:109B4000E6630DEE903A28EE0B8A4CF67743C3F2AB
:109B50002B2309EE903A8BEE8D9AF2EE0E8A28EEC8
:109B60000B8A10E0022E00F02981032E40F02281A2
:109B7000F0EE6B7AECEE2D7A67EEAA7AE5EC017ADC
:109B8000AF4200F0A6802B6807EE903AE36905EE3D
:109B9000903AA36906EE103AE36A04EE103A23689D
:109BA0000AEE903A63680EEE103AA3680FEE103A90
:109BB000E3680EEE903A236A0CEE103A636907EE02
:109BC000103A27EE287A37EEE55A27EE0A7AF0EEB9
:109BD0004E3A25EE075A37EE2B7AEBEE2A3A636AB5
:109BE000C5EE076AB0EE4F7A75EEA65AABEE237A51
:109BF000E5EEED7A74EE2B4A77EEC67AB0EE6E5A49
:109C000067EE847AABEE075A87EEA47A29EE455ABE
:109C100036EE076AF0EE6B3AF0EE467AE5EE0C7A35
:109C2000ECEE083A76EEA55AC7EEA36A37EE066A5E
:109C300076EEA96A07EE903A76EEEA6AC4ED075A24
:109C4000EBEE26AA84ED066AB0EE6A0AABEE260AAF
:109C500020EE270A16F08CFE7AEECE7AA36A67EE23
:109C6000AC7A07EE103A27EE000A87EE8D7A012EC5
:109C700084ED000A77EE0E7A37EECF6A37EE277A58
:109C800026EE2C6A84ED017AC6EE0D6A36EE8F7AE6
:109C900077EE6E5A76EE876A65EEAC5AC4ED026ACC
:109CA00085EE8D6A76EE2E6A36EE266A84ED036ABC
:109CB00074D03FF757AF002E7CD1636B06EE103A9D
:109CC00066EE077A3BEEC66AE6EE267AF0EE67AA03
:109CD0004EE7BDEC108BF8BD4BF61423B7EE008AAF
:109CE000C4F23F0309EE103A38EE400AF3EE038A5D
:109CF00020EE090A17F064FA30EE480A4BF22D23E1
:109D000080EE286AC3F67D7307EE103A002307EE53
:109D1000903AE6EE077A236FF0EE0C6A77EE677AF8
:109D200006EE103A27EEA67A26EE090AC4ED107A5E
:109D300084ED087A17F044FA30EE480A4FF478437D
:109D400080EE286AC4F2936306EE903A0023C4F2D0
:109D5000702307EE903A40F6DB73C4F24903E6EE57
:109D6000267A07EE103A636906EE903A27EEA60AC5
:109D700020EE070A16F072FF216C226F636F84EDEC
:109D80000F0A07EE901A38EE678AF0EE40CABDEE71
:109D9000C88AE264A36484ED188ABAE6636B06EEAF
:109DA000903A66EEA77A7BEEE66AE6EE877AF0EE08
:109DB00067AADDE600230AEE903AD9E6636B06EE69
:109DC000903A6AEEA6AA7BEEE66AE6EEA7AACFE68E
:109DD00030EE600A32EE612A31EE601A20EE022A7D
:109DE00082EE010A30EE210A704700BF00B583B051
:109DF00011F052FC4AF28C62C2F2010241F6647325
:109E000012680192C2F20103019A1A6003B05DF870
:109E100004FB00BF2DE9F0434DF6C068C2F2000814
:109E20002DED028BD8ED027A9FED748A9FED746A56
:109E3000F6EE008AF0EE686AE7EE886A4AF28C6312
:109E4000C2F20103B2EE0E7A26EE877A40F21D07C7
:109E5000C7EE087A91B0C2F201071B6803933A7803
:109E6000039941F66473C2F20103012A196077EE87
:109E7000867AFCEEE77ACDED017A9DF8046000F079
:109E8000E08141F66060C2F2010011F049F945F647
:109E90002C73C0F2020393E803000AAC00254FF0D4
:109EA00020336360A360E5602561A38125750A9076
:109EB00041F660602A46ADF82C10C2F20100294636
:109EC00011F0EAF820461AF05BFE024641F66060A7
:109ED0002146C2F2010014F0B7FE4EF240202B469C
:109EE0000A222946C2F2000014F034FF45F604208D
:109EF0000121C0F2020014F007F84EF240202B4678
:109F00000A222946C2F2000014F024FF45F6F4406C
:109F10000321C0F2020013F0F7FF20461AF030FED2
:109F20000146204613F0F0FF45F2D8700121C0F23F
:109F3000020013F0E9FF4EF24020C2F2000014F0DC
:109F4000F7FE41F660602A2301223146C2F2010089
:109F50000A956560A560E560256125758DF8283056
:109F600011F09AF820461AF00BFE024641F66060A6
:109F70002146C2F2010014F067FE4EF240202B464B
:109F80000A220121C2F2000014F0E4FE45F604208A
:109F90000121C0F2020013F0B7FF4EF240202B4621
:109FA0000A223146C2F2000014F0D4FE45F6F44015
:109FB0000321C0F2020013F0A7FF20461AF0E0FDD3
:109FC0000146204613F0A0FF45F2D8700121C0F2EF
:109FD000020013F099FF4EF24020C2F2000014F08C
:109FE000A7FED8ED027AF0EE686A41F66878E7EEEF
:109FF000886AC2F2010888F8006003E00000C842E5
:10A0000000000000FDEEE67A0A2217EE900A04A98D
:10A010001AF08AF905461AF0B3FDC0B203280246C9
:10A0200028BF0322C2F1030043F23003C0F2300321
:10A030002946204400250A956560A560E5602561F4
:10A040002575ADF82830A3701AF008FE41F660605F
:10A050002A460D21C2F2010011F01EF820461AF026
:10A060008FFD024641F660602146C2F2010014F005
:10A07000EBFD4EF240202B460A222946C2F2000098
:10A0800014F068FE45F604200121C0F2020013F02E
:10A090003BFF4EF240202B460A220D21C2F2000067
:10A0A00014F058FE45F6F4400321C0F2020013F00C
:10A0B0002BFF20461AF064FD0146204613F024FFD2
:10A0C00045F2D8700121C0F2020013F01DFF4EF2DC
:10A0D0004020C2F2000014F02BFE98F8003041F648
:10A0E0006878B342C2F2010800F0A48041F66060D3
:10A0F0002A2301223146C2F201000A956560A5605B
:10A10000E560256125758DF8283010F0C5FF2046E3
:10A110001AF036FD024641F660602146C2F20100A7
:10A1200014F092FD4EF240202B460A220121C2F289
:10A13000000014F00FFE45F604200121C0F20200D9
:10A1400013F0E2FE4EF240202B460A223146C2F2C4
:10A15000000014F0FFFD45F6F4400321C0F20200B8
:10A1600013F0D2FE20461AF00BFD0146204613F0F4
:10A17000CBFE45F2D8700121C0F2020013F0C4FEFC
:10A180004EF24020C2F2000014F0D2FD98F8009088
:10A190000A9541F66060202349460122C2F201007F
:10A1A0006560A560E560256125758DF8283010F0A3
:10A1B00073FF20461AF0E4FC024641F66060214637
:10A1C000C2F2010014F040FD4EF240202B460A225C
:10A1D0000121C2F2000014F0BDFD45F6042001216A
:10A1E000C0F2020013F090FE4EF240202B460A22ED
:10A1F0004946C2F2000014F0ADFD45F6F4400321DB
:10A20000C0F2020013F080FE20461AF0B9FC0146AD
:10A21000204613F079FE45F2D8700121C0F2020009
:10A2200013F072FE4EF24020C2F2000014F080FDE6
:10A2300088F8006001233B7011B0BDEC028BBDE8D3
:10A24000F08341F66878C2F201080AACDAE600BF92
:10A250002DE9F04340F21D07C2F201078DB03B78B3
:10A26000002B40F094854DF6C066C2F200066946A8
:10A270000A2230791AF058F804461AF081FCC0B26C
:10A280000228024628BF0222C2F1020006AB214684
:10A290001844002443F2300306940794ADF81830B4
:10A2A000089409940A948DF82C401AF0D7FC41F6D2
:10A2B000606022462146C2F2010010F0EDFE06A8C1
:10A2C0001AF05EFC024641F6606006A9C2F2010087
:10A2D00014F0BAFC4EF2402023460A222146C2F274
:10A2E000000014F037FD45F604200121C0F2020001
:10A2F00013F00AFE4EF2402023460A222146C2F203
:10A30000000014F027FD45F6F4400321C0F20200DE
:10A3100013F0FAFD06A81AF033FC014606A813F064
:10A32000F3FD45F2D8700121C0F2020013F0ECFDFC
:10A330004EF24020C2F2000014F0FAFC41F66060D8
:10A3400022460221C2F201004FF020090694079430
:10A35000089409940A948DF82C408DF8189010F008
:10A360009BFE06A81AF00CFC024641F6606006A9A6
:10A37000C2F2010014F068FC4EF2402023460A228B
:10A380002146C2F2000014F0E5FC45F6042001214C
:10A39000C0F2020013F0B8FD4EF2402023460A221C
:10A3A0000221C2F2000014F0D5FC45F6F44003216E
:10A3B000C0F2020013F0A8FD06A81AF0E1FB014666
:10A3C00006A813F0A1FD45F2D8700121C0F20200E9
:10A3D00013F09AFD4EF24020C2F2000014F0A8FCE7
:10A3E000337940F2300003EB43024DF6BE6803EBD5
:10A3F0008203C2F2010041F6A441C2F200081844EF
:10A40000C2F2010106F012F898F8005041F66060BF
:10A4100015F0FD05C2F2010000F0D08222460221B3
:10A4200006940794089409940A948DF82C408DF8AA
:10A43000189010F031FE06A81AF0A2FB024641F671
:10A44000606006A9C2F2010014F0FEFB4EF240204B
:10A4500023460A222146C2F2000014F07BFC45F696
:10A4600004200121C0F2020013F04EFD4EF2402004
:10A4700023460A220221C2F2000014F06BFC45F6CA
:10A48000F4400321C0F2020013F03EFD06A81AF0CA
:10A4900077FB014606A813F037FD45F2D87001217D
:10A4A000C0F2020013F030FD4EF24020C2F2000074
:10A4B00014F03EFC41F6A440C2F201001AF060FB29
:10A4C000C2B2082A41F6A44128BF08224FF0203327
:10A4D000C2F2010106A8069307940894CDF81B3038
:10A4E00009940A948DF82C401AF0B8FB41F660608C
:10A4F00022460321C2F2010010F0CEFD06A81AF098
:10A500003FFB024641F6606006A9C2F2010014F06A
:10A510009BFB4EF2402023460A222146C2F2000055
:10A5200014F018FC45F604200121C0F2020013F0DB
:10A53000EBFC4EF2402023460A220321C2F2000027
:10A5400014F008FC45F6F4400321C0F2020013F0B9
:10A55000DBFC06A81AF014FB014606A813F0D4FC95
:10A5600045F2D8700121C0F2020013F0CDFC4EF28A
:10A570004020C2F2000014F0DBFB41F6606022468E
:10A580000B21C2F2010006940794089409940A94DE
:10A590008DF82C408DF8189010F07EFD06A81AF06A
:10A5A000EFFA024641F6606006A9C2F2010014F01B
:10A5B0004BFB4EF2402023460A222146C2F2000005
:10A5C00014F0C8FB45F60420C0F20200012113F08C
:10A5D0009BFC23464EF240200A220B21C2F20000CF
:10A5E00014F0B8FB45F6F4400321C0F2020013F06A
:10A5F0008BFC06A81AF0C4FA014606A813F084FCE6
:10A6000045F2D8700121C0F2020013F07DFC4EF239
:10A610004020C2F2000014F08BFB707969460A22D8
:10A62000013019F081FE04461AF0AAFAC0B20228DD
:10A63000024628BF0222C2F1020006AB214618449E
:10A64000002443F2300306940794ADF818300894C0
:10A6500009940A948DF82C401AF000FB41F66060D2
:10A6600021460122C2F2010010F016FD06A81AF0E0
:10A6700087FA024641F6606006A9C2F2010014F0B2
:10A68000E3FA4EF2402023460A220121C2F20000E2
:10A6900014F060FB45F604200121C0F2020013F023
:10A6A00033FC4EF2402023460A222146C2F200002B
:10A6B00014F050FB45F6F4400321C0F2020013F001
:10A6C00023FC06A81AF05CFA014606A813F01CFC4D
:10A6D00045F2D8700121C0F2020013F015FC4EF2D1
:10A6E0004020C2F2000014F023FB41F6606001221A
:10A6F0000221C2F2010020250694079408940994CF
:10A700000A948DF82C408DF8185010F0C5FC06A85E
:10A710001AF036FA024641F6606006A9C2F201005C
:10A7200014F092FA4EF2402023460A220121C2F28E
:10A73000000014F00FFB45F604200121C0F20200D6
:10A7400013F0E2FB4EF2402023460A220221C2F21D
:10A75000000014F0FFFA45F6F4400321C0F20200B5
:10A7600013F0D2FB06A81AF00BFA014606A813F064
:10A77000CBFB45F2D8700121C0F2020013F0C4FBFC
:10A780004EF24020C2F2000014F0D2FA98F8008095
:10A7900008F0FD084DF6C06641F66060B8F1010FA3
:10A7A000C2F20006C2F2010000F0E781012202219C
:10A7B00006940794089409940A948DF82C408DF817
:10A7C000185010F069FC06A81AF0DAF9024641F6B2
:10A7D000606006A9C2F2010014F036FA4EF2402081
:10A7E00023460A220121C2F2000014F0B3FA45F612
:10A7F00004200121C0F2020013F086FB4EF240203B
:10A8000023460A220221C2F2000014F0A3FA45F600
:10A81000F4400321C0F2020013F076FB06A81AF000
:10A82000AFF9014606A813F06FFB45F2D87001217D
:10A83000C0F2020013F068FB4EF24020C2F20000AA
:10A8400014F076FA727941F6F44302EB820602EBD9
:10A850004606C2F201031E4430461AF091F9C2B214
:10A860000A2A28BF0A224FF02033314606A8069351
:10A870000793089409940A948DF82C408DF8205081
:10A880001AF0ECF941F6606001220321C2F20100E6
:10A8900010F002FC06A81AF073F9024641F6606057
:10A8A00006A9C2F2010014F0CFF94EF2402023466F
:10A8B0000A220121C2F2000014F04CFA45F60420ED
:10A8C0000121C0F2020013F01FFB4EF2402023468C
:10A8D0000A220321C2F2000014F03CFA45F6F440CB
:10A8E0000321C0F2020013F00FFB06A81AF048F98A
:10A8F000014606A813F008FB45F2D8700121C0F20A
:10A90000020013F001FB4EF24020C2F2000014F0EE
:10A910000FFA41F6606001220E21C2F20100069496
:10A920000794089409940A948DF82C408DF81850D7
:10A9300010F0B2FB06A81AF023F9024641F6606057
:10A9400006A9C2F2010014F07FF94EF2402023461E
:10A950000A220121C2F2000014F0FCF945F604209D
:10A960000121C0F2020013F0CFFA4EF2402023463C
:10A970000A220E21C2F2000014F0ECF945F6F44070
:10A980000321C0F2020013F0BFFA06A81AF0F8F88B
:10A99000014606A813F0B8FA45F2D8700121C0F2BA
:10A9A000020013F0B1FA4EF24020C2F2000014F09F
:10A9B000BFF900233B700DB0BDE8F0835B232A464E
:10A9C0000221069507958DF81830089509950A9586
:10A9D0008DF82C5010F060FB06A81AF0D1F8024652
:10A9E00041F6606006A9C2F2010014F02DF94EF2A2
:10A9F00040202B460A222946C2F2000014F0AAF990
:10AA000045F604200121C0F2020013F07DFA4EF257
:10AA100040202B460A220221C2F2000014F09AF9CB
:10AA200045F6F4400321C0F2020013F06DFA06A8C7
:10AA30001AF0A6F8014606A813F066FA45F2D87097
:10AA40000121C0F2020013F05FFA4EF24020C2F280
:10AA5000000014F06DF941F6A440C2F201001AF0B2
:10AA60008FF8C2B2082A41F6A44128BF08224FF04D
:10AA70002033C2F2010106A8069307950895CDF888
:10AA80001B3009950A958DF82C501AF0E7F841F61D
:10AA900060602A460321C2F2010010F0FDFA06A808
:10AAA0001AF06EF8024641F6606006A9C2F2010093
:10AAB00014F0CAF84EF240202B460A222946C2F270
:10AAC000000014F047F945F604200121C0F202000D
:10AAD00013F01AFA4EF240202B460A220321C2F24A
:10AAE000000014F037F945F6F4400321C0F20200EB
:10AAF00013F00AFA06A81AF043F8014606A813F064
:10AB000003FA45F2D8700121C0F2020013F0FCF9FB
:10AB10004EF24020C2F2000014F00AF941F66060E3
:10AB20005D232A460B21C2F20100069507958DF898
:10AB30001830089509950A958DF82C5010F0ACFA4C
:10AB400006A81AF01DF8024641F6606006A9C2F296
:10AB5000010014F079F84EF240202B460A222946D3
:10AB6000C2F2000014F0F6F845F60420C0F202002C
:10AB7000012113F0C9F92B462CE55B234246022143
:10AB8000069407948DF81830089409940A948DF867
:10AB90002C4010F081FA06A819F0F2FF024641F6A7
:10ABA000606006A9C2F2010014F04EF84EF2402097
:10ABB00023460A224146C2F2000014F0CBF845F6C3
:10ABC00004204146C0F2020013F09EF94EF24020EC
:10ABD00023460A220221C2F2000014F0BBF845F617
:10ABE000F4400321C0F2020013F08EF906A819F018
:10ABF000C7FF014606A813F087F945F2D870414611
:10AC0000C0F2020013F080F94EF24020C2F20000C0
:10AC100014F08EF8727941F6F44302EB820602EBEF
:10AC20004606C2F201031E44304619F0A9FFC2B223
:10AC30000A2A28BF0A224FF02033314606A806937D
:10AC40000793089409940A948DF82C408DF82050AD
:10AC50001AF004F841F6606042460321C2F2010096
:10AC600010F01AFA06A819F08BFF024641F6606050
:10AC700006A9C2F2010013F0E7FF4EF2402023467E
:10AC80000A224146C2F2000014F064F845F604209E
:10AC90004146C0F2020013F037F94EF2402023463D
:10ACA0000A220321C2F2000014F054F845F6F440E1
:10ACB0000321C0F2020013F027F906A819F060FF83
:10ACC000014606A813F020F945F2D8704146C0F2BB
:10ACD000020013F019F94EF24020C2F2000014F005
:10ACE00027F841F660605D2342460E21C2F2010062
:10ACF000069407948DF81830089409940A948DF8F6
:10AD00002C4010F0C9F906A819F03AFF024641F6A6
:10AD1000606006A9C2F2010013F096FF4EF24020D7
:10AD200023460A224146C2F2000014F013F845F609
:10AD300004204146C0F2020013F0E6F84EF2402033
:10AD400023460A220E21C2F2000014F003F845F651
:10AD5000F4400321C0F2020013F0D6F806A819F05F
:10AD60000FFF014606A813F0CFF845F2D870414610
:10AD7000C0F2020013F0C8F84EF24020C2F2000008
:10AD800013F0D6FF00233B700DB0BDE8F08341F611
:10AD90006060C2F2010010F0C3F9FFF764BA00BFAF
:10ADA0002DE9F04140F21D06C2F201068CB0337865
:10ADB000032B00F03E8341F66060C2F2010010F008
:10ADC000AFF945F63473C0F2020393E8030006AC12
:10ADD00000254FF02033A3606360E5602561C4F86F
:10ADE0000B302575069041F660602A46ADF81C10C0
:10ADF000C2F20100294610F04FF9204619F0C0FEBA
:10AE0000024641F660602146C2F2010013F01CFFC9
:10AE10004EF240202B460A222946C2F2000013F0CF
:10AE200099FF45F604200121C0F2020013F06CF8EE
:10AE30004EF240202B460A222946C2F2000013F0AF
:10AE400089FF45F6F4400321C0F2020013F05CF8DC
:10AE5000204619F095FE0146204613F055F845F2BC
:10AE6000D8700121C0F2020013F04EF84EF24020DB
:10AE7000C2F2000013F05CFF46F2525341F66060EC
:10AE8000C3F6732329460122C2F201006560A56062
:10AE9000E56025612575069310F0FEF8204619F04F
:10AEA0006FFE024641F660602146C2F2010013F0D7
:10AEB000CBFE4EF240202B460A220121C2F20000B6
:10AEC00013F048FF45F604200121C0F2020013F000
:10AED0001BF84EF240202B460A222946C2F20000FF
:10AEE00013F038FF45F6F4400321C0F2020013F0DE
:10AEF0000BF8204619F044FE0146204613F004F8F2
:10AF000045F2D8700121C0F2020012F0FDFF4EF2AE
:10AF10004020C2F2000013F00BFF47F2435341F60A
:10AF20006060C3F6742301220821C2F2010065604B
:10AF3000A560E56025612575069310F0ADF8204603
:10AF400019F01EFE024641F660602146C2F2010081
:10AF500013F07AFE4EF240202B460A220121C2F263
:10AF6000000013F0F7FE45F604200121C0F20200B4
:10AF700012F0CAFF4EF240202B460A220821C2F2EC
:10AF8000000013F0E7FE45F6F4400321C0F2020092
:10AF900012F0BAFF204619F0F3FD0146204612F0E8
:10AFA000B3FF45F2D870C0F20200012112F0ACFFED
:10AFB0004EF24020C2F2000013F0BAFE41F6F14317
:10AFC000C2F201034FF2CB081B7803EB830303EBC0
:10AFD0008303C2F68D089B0088FB0320DB17C3EBBD
:10AFE000201069460A2219F09FF9054619F0C8FD9C
:10AFF000C0B20228024628BF0222C2F1020029463E
:10B0000043F230070025204406956560A560E560A1
:10B0100025612575ADF8187019F020FE41F66060C5
:10B0200001220521C2F2010010F036F8204619F085
:10B03000A7FD024641F660602146C2F2010013F00E
:10B0400003FE4EF240202B460A220121C2F20000EC
:10B0500013F080FE45F604200121C0F2020012F038
:10B0600053FF4EF240200A222B460521C2F2000077
:10B0700013F070FE45F6F4400321C0F2020012F016
:10B0800043FF204619F07CFD0146204612F03CFFAC
:10B0900045F2D8700121C0F2020012F035FF4EF2E5
:10B0A0004020C2F2000013F043FE40F21C03C2F243
:10B0B000010369461B7803EB830303EB83039B00C7
:10B0C00088FB0320DB17C3EB20100A2219F02CF9B0
:10B0D000804619F055FDC0B20228024628BF022260
:10B0E000C2F102004146204406956560A560E56016
:10B0F00025612575ADF8187019F0B0FD41F6606056
:10B1000001220D21C2F201000FF0C6FF204619F006
:10B1100037FD024641F660602146C2F2010013F09D
:10B1200093FD4EF240202B460A220121C2F200007C
:10B1300013F010FE45F604200121C0F2020012F0C7
:10B14000E3FE4EF240202B460A220D21C2F20000FF
:10B1500013F000FE45F6F4400321C0F2020012F0A5
:10B16000D3FE204619F00CFD0146204612F0CCFE1D
:10B1700045F2D8700121C0F202004DF6BE6712F010
:10B18000C3FEC2F200074EF24020C2F2000013F0EC
:10B19000CFFD97F8008041F66060B8F1040FC2F26D
:10B1A000010000F04881012204214FF0200806959B
:10B1B0006560A560E560256125758DF818800FF044
:10B1C0006BFF204619F0DCFC024641F66060214628
:10B1D000C2F2010013F038FD4EF240202B460A2245
:10B1E0000121C2F2000013F0B5FD45F60420012153
:10B1F000C0F2020012F088FE4EF240200A222B46D6
:10B200000421C2F2000013F0A5FD45F6F44003212D
:10B21000C0F2020012F078FE204619F0B1FC01469F
:10B22000204612F071FE45F2D8700121C0F20200F2
:10B2300012F06AFE4EF24020C2F2000013F078FDD8
:10B2400041F660600695C2F201006560A560E560A8
:10B2500025612575012207218DF818800FF01CFF4C
:10B26000204619F08DFC024641F660602146C2F28C
:10B27000010013F0E9FC4EF240202B460A22012186
:10B28000C2F2000013F066FD45F604200121C0F271
:10B29000020012F039FE4EF240202B460A2207210E
:10B2A000C2F2000013F056FD45F6F4400321C0F24F
:10B2B000020012F029FE204619F062FC01462046E9
:10B2C00012F022FE45F2D8700121C0F2020012F005
:10B2D0001BFE4EF24020C2F2000013F029FD3B7825
:10B2E00041F66060052B4FF00005C2F2010000F04E
:10B2F000FE8001220C21202706956560A560E5608F
:10B30000256125758DF818700FF0C6FE204619F0DE
:10B3100037FC024641F660602146C2F2010013F09C
:10B3200093FC4EF240202B460A220121C2F200007B
:10B3300013F010FD45F604200121C0F2020012F0C6
:10B34000E3FD4EF240200A222B460C21C2F20000FF
:10B3500013F000FD45F6F4400321C0F2020012F0A4
:10B36000D3FD204619F00CFC0146204612F0CCFD1E
:10B3700045F2D8700121C0F2020012F0C5FD4EF274
:10B380004020C2F2000013F0D3FC41F66060069545
:10B39000C2F201006560A560E560256125750122A6
:10B3A0000F218DF818700FF077FE204619F0E8FB9A
:10B3B000024641F660602146C2F2010013F044FCEF
:10B3C0004EF240202B460A220121C2F2000013F067
:10B3D000C1FC45F604200121C0F2020012F094FDE8
:10B3E0004EF240202B460A220F21C2F2000013F039
:10B3F000B1FC45F6F4400321C0F2020012F084FDD6
:10B40000204619F0BDFB0146204612F07DFD45F2B5
:10B41000D8700121C0F2020012F076FD4EF24020F9
:10B42000C2F2000013F084FC032333700CB0BDE8BB
:10B43000F08106ACC2E55B230122414606956560BA
:10B44000A560E560256125758DF818300FF024FEA4
:10B45000204619F095FB024641F660602146C2F293
:10B46000010013F0F1FB4EF240202B460A2201218D
:10B47000C2F2000013F06EFC45F604200121C0F278
:10B48000020012F041FD4EF240202B460A224146B6
:10B49000C2F2000013F05EFC45F6F4400321C0F256
:10B4A000020012F031FD204619F06AFB01462046E9
:10B4B00012F02AFD45F2D8700121C0F2020012F00C
:10B4C00023FD4EF24020C2F2000013F031FC41F6A1
:10B4D00060605D230695C2F201006560A560E560CD
:10B4E00025612575012207218DF81830B6E65B230A
:10B4F00001220C2106956560A560E5602561257532
:10B500008DF818300FF0C8FD204619F039FB0246BF
:10B5100041F660602146C2F2010013F095FB4EF245
:10B5200040202B460A220121C2F2000013F012FC37
:10B5300045F604200121C0F2020012F0E5FC4EF2B3
:10B5400040202B460A220C21C2F2000013F002FC1C
:10B5500045F6F4400321C0F2020012F0D5FC20466B
:10B5600019F00EFB0146204612F0CEFC45F2D870D1
:10B570000121C0F2020012F0C7FC4EF24020C2F2DC
:10B58000000013F0D5FB41F660605D230695C2F222
:10B5900001006560A560E5602561257501220F2128
:10B5A0008DF81830FFE600BFF0B54AF28C63C2F2A6
:10B5B000010340F21D068FB0C2F201061B68019321
:10B5C0003278019941F66473C2F20103022A1960CC
:10B5D00000F0D18041F66060C2F201000FF0A0FDE2
:10B5E00045F63C73C0F2020393E8070008AC00255F
:10B5F0004FF02033E560C4F80B3084E8070041F6D3
:10B6000060602A462946C2F20100256125750FF0C7
:10B6100043FD204619F0B4FA024641F66060214627
:10B62000C2F2010013F010FB4EF240202B462946D7
:10B630000A22C2F2000013F08DFB45F6042001211E
:10B64000C0F2020012F060FC4EF240202B460A22AB
:10B650002946C2F2000013F07DFB45F6F4400321B9
:10B66000C0F2020012F050FC204619F089FA01469F
:10B67000204612F049FC45F2D8700121C0F20200C8
:10B680004DF6C06712F040FCC2F200074EF24020B7
:10B69000C2F2000013F04CFB3D7C002D73D00A2257
:10B6A00002A9284618F040FE054619F069FAC0B212
:10B6B0000228024628BF0222C2F1020043F23003F0
:10B6C00029462044002508956560A560E560256150
:10B6D0002575ADF8203019F0C1FA41F660602946B1
:10B6E0000122C2F201000FF0D7FC204619F048FAFF
:10B6F000024641F660602146C2F2010013F0A4FA4E
:10B700004EF240202B460A220121C2F2000013F023
:10B7100021FB45F604200121C0F2020012F0F4FBE7
:10B720004EF240202B460A222946C2F2000013F0B6
:10B7300011FB45F6F4400321C0F2020012F0E4FBD5
:10B74000204619F01DFA0146204612F0DDFB45F2B5
:10B75000D8700121C0F2020012F0D6FB4EF2402058
:10B76000C2F2000013F0E4FA3F7C012F60D0022304
:10B7700033700FB0F0BD4DF6C067C2F2000708ACE1
:10B780003D7C002D8BD144F64F5341F66060C4F6EA
:10B790004E1329460122C2F201006560A560E560F2
:10B7A0002561257508930FF077FC204619F0E8F91C
:10B7B000024641F660602146C2F2010013F044FAED
:10B7C0004EF240202B460A220121C2F2000013F063
:10B7D000C1FA45F604200121C0F2020012F094FBE8
:10B7E0004EF240202B460A222946C2F2000013F0F6
:10B7F000B1FA45F6F4400321C0F2020012F084FBD6
:10B80000204619F0BDF90146204612F07DFB45F2B5
:10B81000D8700121C0F2020012F076FB4EF24020F7
:10B82000C2F2000013F084FA022333700FB0F0BDAF
:10B8300041F6606042F220033A460221C2F2010062
:10B8400008956560A560E56025612575ADF8203037
:10B850000FF022FC204619F093F9024641F6606091
:10B860002146C2F2010013F0EFF94EF240202B46C0
:10B870000A223946C2F2000013F06CFA45F60420A1
:10B880003946C0F2020012F03FFB4EF240202B4638
:10B890000A220221C2F2000013F05CFA45F6F440DD
:10B8A0000321C0F2020012F02FFB204619F068F9C4
:10B8B0000146204612F028FB45F2D8703946C0F206
:10B8C000020012F021FB4EF24020C2F2000013F001
:10B8D0002FFA022333700FB0F0BD00BF2DE9F04105
:10B8E00040F21D06C2F201068CB03378042B00F042
:10B8F000F88441F66060C2F201000FF011FC45F6D9
:10B900004C73C0F2020393E8030006AC00256560A7
:10B91000A560E56025612575069041F660602A46C0
:10B920008DF81C10C2F2010029460FF0B5FB20462D
:10B9300019F026F9024641F660602146C2F2010084
:10B9400013F082F94EF240202B460A222946C2F219
:10B95000000013F0FFF945F604200121C0F20200B7
:10B9600012F0D2FA4EF240202B460A222946C2F2A9
:10B97000000013F0EFF945F6F4400321C0F2020095
:10B9800012F0C2FA204619F0FBF80146204612F0E8
:10B99000BBFA45F2D8700121C0F2020012F0B4FAED
:10B9A0004EF24020C2F2000013F0C2F941F660608E
:10B9B00043F654232A460621C2F20100069565602B
:10B9C000A560E56025612575ADF818300FF064FBC2
:10B9D000204619F0D5F8024641F660602146C2F2D1
:10B9E000010013F031F94EF240202B460A2229467D
:10B9F000C2F2000013F0AEF945F604200121C0F2B6
:10BA0000020012F081FA4EF240202B460A22062153
:10BA1000C2F2000013F09EF945F6F4400321C0F293
:10BA2000020012F071FA204619F0AAF801462046E9
:10BA300012F06AFA45F2D8700121C0F2020012F049
:10BA400063FA4EF24020C2F2000013F071F941F6A1
:10BA5000606047F26D332A460E21C2F2010006955E
:10BA60006560A560E56025612575ADF818300FF0BB
:10BA700013FB204619F084F8024641F66060214627
:10BA8000C2F2010013F0E0F84EF240202B460A22E9
:10BA90002946C2F2000013F05DF945F604200121A9
:10BAA000C0F2020012F030FA4EF240202B460A2279
:10BAB0000E21C2F2000013F04DF945F6F4400321C7
:10BAC000C0F2020012F020FA204619F059F801469F
:10BAD000204612F019FA45F2D8700121C0F2020096
:10BAE00012F012FA4EF24020C2F2000013F020F9D8
:10BAF00045F65473C0F2020341F660601B68069578
:10BB00001F0C29460122C2F201006560A560E560B4
:10BB100025612575ADF818308DF81A700FF0BCFA54
:10BB2000204619F02DF8024641F660602146C2F227
:10BB3000010013F089F84EF240202B460A22012121
:10BB4000C2F2000013F006F945F604200121C0F20C
:10BB5000020012F0D9F94EF240202B460A22294663
:10BB6000C2F2000013F0F6F845F6F4400321C0F2EB
:10BB7000020012F0C9F9204619F002F801462046E9
:10BB800012F0C2F945F2D8700121C0F2020012F0A1
:10BB9000BBF94EF24020C2F2000013F0C9F846F69D
:10BBA000567341F66060C3F66C2301220821C2F28D
:10BBB00001006560A560E5602561257506930FF0BD
:10BBC0006BFA204618F0DCFF024641F66060214621
:10BBD000C2F2010013F038F84EF240202B460A2240
:10BBE0000121C2F2000013F0B5F845F6042001214E
:10BBF000C0F2020012F088F94EF240202B460A22D1
:10BC00000821C2F2000013F0A5F845F6F440032124
:10BC1000C0F2020012F078F9204618F0B1FF014698
:10BC2000204612F071F945F2D870C0F202000121ED
:10BC300012F06AF94EF24020C2F2000013F078F8D8
:10BC400040F26C52C2F201024FF49663107848F24F
:10BC50001F57C5F2EB1703FB00F387FB0320DB172D
:10BC6000C3EB201069460A2218F05EFB054618F067
:10BC700087FFC0B20428024628BF0422C2F1040094
:10BC80004FF030332946204400256560A560E5600B
:10BC900025612575069318F0E1FF41F660602A469C
:10BCA0000921C2F201000FF0F7F9204618F068FFF1
:10BCB000024641F660602146C2F2010012F0C4FF64
:10BCC0004EF240202B460A222946C2F2000013F011
:10BCD00041F845F604200121C0F2020012F014F9E7
:10BCE0004EF240200A222B460921C2F2000013F036
:10BCF00031F845F6F4400321C0F2020012F004F9D5
:10BD0000204618F03DFF0146204612F0FDF845F2AE
:10BD1000D8700121C0F2020012F0F6F84EF2402075
:10BD2000C2F2000013F004F841F6F043C2F201033E
:10BD30004AF2EB001B7803EB430303EB4313CEF60D
:10BD40000E2080FB03201844DB17C3EB601069460C
:10BD50000A2218F0E9FA804618F012FFC0B2022851
:10BD6000024628BF0222C2F102004146204443F2AB
:10BD7000300806956560A560E56025612575ADF81C
:10BD8000188018F06BFF41F6606001220421C2F2B6
:10BD900001000FF081F9204618F0F2FE024641F64C
:10BDA00060602146C2F2010012F04EFF4EF24020C8
:10BDB0002B460A220121C2F2000012F0CBFF45F609
:10BDC00004200121C0F2020012F09EF84EF2402041
:10BDD0000A222B460421C2F2000012F0BBFF45F6F6
:10BDE000F4400321C0F2020012F08EF8204618F051
:10BDF000C7FE0146204612F087F845F2D8700121AF
:10BE0000C0F2020012F080F84EF24020C2F20000B0
:10BE100012F08EFF41F67463C2F2010369461B788B
:10BE200003EB430303EB431387FB0320DB17C3EB55
:10BE300020100A2218F078FA074618F0A1FEC0B2C6
:10BE40000228024628BF0222C2F1020039462044DD
:10BE500006956560A560E56025612575ADF81880DB
:10BE600018F0FCFE41F6606001220D21C2F20100D3
:10BE70000FF012F9204618F083FE024641F660608A
:10BE80002146C2F2010012F0DFFE4EF240202B46A6
:10BE90000A220121C2F2000012F05CFF45F60420E4
:10BEA0000121C0F2020012F02FF84EF240202B4682
:10BEB0000A220D21C2F2000012F04CFF45F6F440B8
:10BEC0000321C0F2020012F01FF8204618F058FEBD
:10BED0000146204612F018F845F2D8700121C0F250
:10BEE00002004DF6BE6712F00FF8C2F200074EF2E4
:10BEF0004020C2F2000012F01BFF3B7841F6606068
:10BF0000062BC2F2010000F04A822A4608214FF0B7
:10BF1000200806956560A560E560256125758DF8AA
:10BF200018800FF0B9F8204618F02AFE024641F6B4
:10BF300060602146C2F2010012F086FE4EF24020FF
:10BF40002B460A222946C2F2000012F003FF45F6F2
:10BF500004200121C0F2020011F0D6FF4EF2402071
:10BF60000A222B460821C2F2000012F0F3FE45F629
:10BF7000F4400321C0F2020011F0C6FF204618F081
:10BF8000FFFD0146204611F0BFFF45F2D8700121A8
:10BF9000C0F2020011F0B8FF4EF24020C2F20000E1
:10BFA00012F0C6FE41F660600695C2F201006560BF
:10BFB000A560E560256125752A460D218DF818805C
:10BFC0000FF06AF8204618F0DBFD024641F660608B
:10BFD0002146C2F2010012F037FE4EF240202B46FD
:10BFE0000A222946C2F2000012F0B4FE45F60420EF
:10BFF0000121C0F2020011F087FF4EF240202B46D3
:10C000000A220D21C2F2000012F0A4FE45F6F4400F
:10C010000321C0F2020011F077FF204618F0B0FDB6
:10C020000146204611F070FF45F2D8700121C0F2A0
:10C03000020011F069FF4EF24020C2F2000012F03F
:10C0400077FE3B7841F66060072B4FF00005C2F2A7
:10C05000010000F04881012203214FF020080695DD
:10C060006560A560E560256125758DF818800FF085
:10C0700013F8204618F084FD024641F66060214620
:10C08000C2F2010012F0E0FD4EF240202B460A22DF
:10C090000121C2F2000012F05DFE45F604200121EC
:10C0A000C0F2020011F030FF4EF240200A222B466F
:10C0B0000321C2F2000012F04DFE45F6F4400321C8
:10C0C000C0F2020011F020FF204618F059FD014691
:10C0D000204611F019FF45F2D8700121C0F202008C
:10C0E00011F012FF4EF24020C2F2000012F020FECA
:10C0F00041F660600695C2F201006560A560E560EA
:10C1000025612575012206218DF818800EF0C4FFE7
:10C11000204618F035FD024641F660602146C2F225
:10C12000010012F091FD4EF240202B460A2201211F
:10C13000C2F2000012F00EFE45F604200121C0F20A
:10C14000020011F0E1FE4EF240202B460A220621A9
:10C15000C2F2000012F0FEFD45F6F4400321C0F2E9
:10C16000020011F0D1FE204618F00AFD01462046DB
:10C1700011F0CAFE45F2D8700121C0F2020011F0A0
:10C18000C3FE4EF24020C2F2000012F0D1FD3B7817
:10C1900041F66060082B4FF00005C2F2010000F08C
:10C1A0005A8101220C21202706956560A560E56073
:10C1B000256125758DF818700EF06EFF204618F079
:10C1C000DFFC024641F660602146C2F2010012F037
:10C1D0003BFD4EF240202B460A220121C2F2000014
:10C1E00012F0B8FD45F604200121C0F2020011F062
:10C1F0008BFE4EF240200A222B460C21C2F2000098
:10C2000012F0A8FD45F6F4400321C0F2020011F03F
:10C210007BFE204618F0B4FC0146204611F074FE67
:10C2200045F2D8700121C0F2020011F06DFE4EF20D
:10C230004020C2F2000012F07BFD41F660600695DE
:10C24000C2F201006560A560E560256125750122E7
:10C250000F218DF818700EF01FFF204618F090FC8B
:10C26000024641F660602146C2F2010012F0ECFC89
:10C270004EF240202B460A220121C2F2000012F0A9
:10C2800069FD45F604200121C0F2020011F03CFED8
:10C290004EF240202B460A220F21C2F2000012F07B
:10C2A00059FD45F6F4400321C0F2020011F02CFEC6
:10C2B000204618F065FC0146204611F025FE45F2A7
:10C2C000D8700121C0F2020011F01EFE4EF2402093
:10C2D000C2F2000012F02CFD042333700CB0BDE854
:10C2E000F08106ACACE45B23012203210695656076
:10C2F000A560E560256125758DF818300EF0CCFE3F
:10C30000204618F03DFC024641F660602146C2F22C
:10C31000010012F099FC4EF240202B460A22012126
:10C32000C2F2000012F016FD45F604200121C0F211
:10C33000020011F0E9FD4EF240202B460A220321B3
:10C34000C2F2000012F006FD45F6F4400321C0F2EF
:10C35000020011F0D9FD204618F012FC01462046DB
:10C3600011F0D2FD45F2D8700121C0F2020011F0A7
:10C37000CBFD4EF24020C2F2000012F0D9FC41F693
:10C3800060605D230695C2F201006560A560E5600E
:10C3900025612575012206218DF81830B6E65B234C
:10C3A0002A46082106956560A560E560256125752A
:10C3B0008DF818300EF070FE204618F0E1FB0246B2
:10C3C00041F660602146C2F2010012F03DFC4EF2DF
:10C3D00040202B460A222946C2F2000012F0BAFC85
:10C3E00045F604200121C0F2020011F08DFD4EF24D
:10C3F00040202B460A220821C2F2000012F0AAFCBB
:10C4000045F6F4400321C0F2020011F07DFD204604
:10C4100018F0B6FB0146204611F076FD45F2D870C3
:10C420000121C0F2020011F06FFD4EF24020C2F275
:10C43000000012F07DFC41F660605D230695C2F2BB
:10C4400001006560A560E560256125752A460D211E
:10C450008DF81830B4E55B2301220C210695656048
:10C46000A560E560256125758DF818300EF014FE85
:10C47000204618F085FB024641F660602146C2F274
:10C48000010012F0E1FB4EF240202B460A2201216E
:10C49000C2F2000012F05EFC45F604200121C0F259
:10C4A000020011F031FD4EF240202B460A220C21F1
:10C4B000C2F2000012F04EFC45F6F4400321C0F237
:10C4C000020011F021FD204618F05AFB01462046DB
:10C4D00011F01AFD45F2D8700121C0F2020011F0EE
:10C4E00013FD4EF24020C2F2000012F021FC41F692
:10C4F00060605D230695C2F201006560A560E5609D
:10C500002561257501220F218DF81830A3E600BFA3
:10C510002DE9F04F2DED068B4AF28C67C2F2010730
:10C5200089B041F664723B680493C2F20102049B35
:10C53000116840F6B7325B1A934207D940F21D03E7
:10C54000C2F201031B78002B40F0488141F2F4480D
:10C55000C2F2010841F670633A680592C2F2010323
:10C5600041F287321968059B5B1A934208D94DF650
:10C57000BE63C2F200031A78911E012940F2E280E4
:10C5800041F2F444C2F2010441F6D04340F22406E1
:10C590004BF6836A04F10C02C2F201039FEDD08ACC
:10C5A0009FEDD09ADFEDD08A9FEDD0AADFEDD09A33
:10C5B000CDF80480C2F201060093C2F6A07A0025ED
:10C5C000904603EB051B58460EF0D0FB58465FFA29
:10C5D00085F90EF011FC38B13B68069341F6B4437F
:10C5E000C2F20103069A1A6058460EF0FBFBA0B394
:10C5F00041F6B4433A680792C2F201031A68079BF6
:10C600009B1AB3F5FA7F00F2238140F21D03C2F2B8
:10C610000103B9F1010F1B7800F0D580012B00F068
:10C620007284C0F01183022B00F08784AB4645F67C
:10C6300084700721C0F2020011F066FC4EF2402027
:10C640005946C2F2000000230A2212F083FB4EF288
:10C650004020C2F2000012F06BFB237C012B40F261
:10C66000498172B6E36862B6002B56F8042BB8BF56
:10C670000333B2EBA30F5CD0B9F1010F6DD140F2DF
:10C680001D02C2F201021378012B00F0AE82C0F04D
:10C690006983032B00F0FA81042B0FD14DF6BE63A2
:10C6A000C2F200031B78072B00F0E986082B00F08C
:10C6B000CB84062B00F05387FFF710F946F2D00029
:10C6C0000821C0F2020011F01FFC4EF240200023AE
:10C6D0000A222946C2F2000012F03CFB45F6B440A3
:10C6E000C0F20200022111F00FFC237C012B40F26A
:10C6F000068372B6E16862B60029B8BF03314EF214
:10C7000040208910C2F2000012F0B4FA4EF240202C
:10C71000C2F2000012F00CFB237C012B40F2C48219
:10C7200072B6E36862B6002BB8BF03339B1046F8BD
:10C73000043C0135022D04F1140408F1140807D05B
:10C74000009B3EE7032A40F0008101221A7017E7A0
:10C7500009B0BDEC068BBDE8F08F40F21D03C2F2BC
:10C7600001031B78012B40F2F380022BA6D1237C1E
:10C77000012B40F2D28772B6E36862B6032B40F316
:10C780005185237C012B41F2508072B6E36862B67A
:10C790003F2B03DD72B64023E36062B6237C012B9E
:10C7A00040F28F8772B6E36862B64DF6C062002B26
:10C7B000C2F20002B8BF03339B101374FAF70EF8ED
:10C7C000FEF7F2FE7AE7002B00F02982033B012BF3
:10C7D0004FF0040140F23883CB4628E7033B012B9E
:10C7E0007FF6B4AE4DF6C063C2F2000393ED027A59
:10C7F000DFED3B6ADFED3B7A9FED3B6A27EE267A61
:10C8000027EE277AC7EE267A77EE867AFDEEE77A6C
:10C8100017EE903A9B0072B641F2F448C2F201085A
:10C82000C8F80C3062B698F81030012B40F238830B
:10C8300072B6D8F80C3062B640F22402002BC2F275
:10C840000102B8BF03339B101360FDF701FD81E6C1
:10C8500045F658702921C0F2020011F055FB4EF246
:10C86000402000230A222946C2F2000012F072FA88
:10C870004EF24020C2F2000012F05AFAB9F1010F54
:10C88000AB467FF4D4AE40F21D03C2F201031B7825
:10C89000032B00F0FC84042B00F0DA84002B7FF4DF
:10C8A000C6AE4DF6BE6241F6F143C2F20002C2F2DC
:10C8B0000103042111701B7872B69B00E36062B61D
:10C8C000237C012B41F2158372B6E36862B6002B1C
:10C8D000B8BF03339B103360FEF762FAA7E600BFD0
:10C8E0000000C84200002C420000000000000C4282
:10C8F00000FEFF4672B694E80C0010781978637A4F
:10C90000227A194202EA000200F0B780A37A03F00B
:10C9100003030AB143F0040343F008039A10082B01
:10C92000A27200F21482072B80F03483032B00F0F4
:10C93000368340F2AF81042B00F0B281062B7FF4E6
:10C9400091AEE368023BE3608DE600221A7017E6C1
:10C95000237C012B40F2898672B6E36862B6032B12
:10C9600040F36684237C012B40F28B8772B6E36828
:10C9700062B6AB2B03DD72B6AC23E36062B6237CF8
:10C98000012B40F2228772B6E36862B6002B227C4C
:10C99000B8BF03339B10012A46F8043C40F2E986F5
:10C9A00072B6E36862B6002BB8BF03339A106423F3
:10C9B00003FB02F38AFB0312DB17C3EBE20307EE70
:10C9C000903AF8EEE77A4DF6C06387EE887AC2F2C5
:10C9D000000341F26059C2F2010945F68C7014223D
:10C9E0001C21C0F20200A9F804200293D3ED027AC0
:10C9F00077EE677AF3EE046A87EEA67A89ED007A1D
:10CA000011F082FA029B986817F0A0F841EC100B25
:10CA10004EF240200521C2F2000012F0DBF945F68B
:10CA2000AC700E21C0F2020011F06EFA4EF24020FE
:10CA3000B9F80410C2F2000012F01CF945F6BC70FF
:10CA40000E21C0F2020011F05FFAD9F8000017F0D1
:10CA50007DF841EC100B4EF240200521C2F200009F
:10CA600012F0B8F94EF24020C2F2000012F060F964
:10CA7000F9F7B4FEFDF7CEF920E6A37A03F003033D
:10CA8000002A3FF44BAF43F0040347E74DF6BE6383
:10CA9000C2F200031B78042B00F02084052B40F029
:10CAA000A180237C012B41F2E68272B6E36862B674
:10CAB000032B40F3E887237C012B41F2AB8472B651
:10CAC000E36862B6B3F5C87F04DB72B64FF4C8738F
:10CAD000E36062B6237C012B41F2A18272B6E36867
:10CAE00062B6002B227CB8BF03339B10012A46F8A4
:10CAF000043C41F2688272B6E36862B640F21C02FE
:10CB0000002B217CB8BF0333C2F201029B10012924
:10CB1000137041F2528272B6E36862B6002BB8BF5E
:10CB200003339B1007EE903AB8EEE77A41F2905B40
:10CB3000C7EE087AC2F2010B40F2F069DBF8003070
:10CB4000C2F2010946F22C0014222321C0F2020095
:10CB5000A9F80420B7EE007A37EE677AD3ED587A59
:10CB600077EE677AF3EE046A87EEA67A89ED007AAB
:10CB700011F0CAF9DBF80030D3F8600116F0E6FFD7
:10CB800041EC100B4EF240200521C2F2000012F0E1
:10CB900021F946F250001521C0F2020011F0B4F95B
:10CBA0004EF24020B9F80410C2F2000012F062F810
:10CBB00046F26800C0F20200152111F0A5F9D9F87B
:10CBC000000016F0C3FF41EC100B4EF24020C2F201
:10CBD0000000052112F0FEF84EF24020C2F20000E3
:10CBE00012F0A6F8FEF7DCF868E54DF6C06341F6F2
:10CBF0006060C2F200030021C2F2010002930393BD
:10CC000011700EF08DFA029B5B7972B6019A9B004F
:10CC1000136262B6F9F7E2FDFDF71AFB4EE54DF639
:10CC2000BE62C2F200021378012B00F01484C0F03F
:10CC3000E182022B00F0DE82032B00F00C84FDF772
:10CC400007FB4FF0010BF2E44DF6C063C2F20003A4
:10CC500093ED027A27EE087A27EE097AC7EE087A72
:10CC600077EEA87AFDEEE77A17EE903A9B0072B65F
:10CC7000E36062B6237C012B40F2108772B6E36852
:10CC800062B6002BB8BF03339B103360AB46FDF791
:10CC9000C1F8CCE4012B00F07D81022B7FF4E2ACE3
:10CCA000E368013BE360DEE472B694E80C001078C0
:10CCB0001978637A227A194202EA000200F096801B
:10CCC000A37A03F003030AB143F0040343F008031B
:10CCD0009A10082BA27200F2A880072B80F0AF8177
:10CCE000032B00F0B08240F26681042B00F0A88094
:10CCF000062B7FF416ADE368023BE36012E572B6E3
:10CD000094E80C0010781978637A227A194202EAC2
:10CD1000000274D0A37A03F003030AB143F00403C2
:10CD200043F008039A10082BA27270D8072B80F0EA
:10CD30007B81032B00F0828240F23681042B70D07D
:10CD4000062B7FF4D7ACE1680239E160D3E40C2B09
:10CD500000F0258100F21881092B3FF4F2AD0B2B76
:10CD60009ED07FE44DF6BE63C2F200031A78012A1A
:10CD700000F05785C0F0FB81022A00F0FA81032AF7
:10CD800031D1237C012B40F2B18772B6E36862B6E1
:10CD9000032B40F31586237C012B41F2A38272B64C
:10CDA000E36862B67F2B4DF6C063C2F2000307DD75
:10CDB0001A79622A41F2A68172B67C22E26062B6DA
:10CDC000227C012A40F2BC8772B6E26862B6002A71
:10CDD000B8BF0332C2F38702114618795A7103F0C3
:10CDE0002BFEF9F7FBFCFDF733FA67E4A37A03F0B7
:10CDF0000303002A3FF46CAF43F0040368E7A37A0F
:10CE000003F00303002A8DD043F004038AE70C2BC0
:10CE100000F0148200F20281092B94D00B2B7FF4D6
:10CE200069ACE1680139E16065E40C2B00F00B822C
:10CE300000F2FF80092B3FF45EAF0B2B7FF471AC47
:10CE4000E368013BE3606DE44DF6BE63C2F20003AC
:10CE50001A78062A00F0558500F2BD80042A00F0F9
:10CE60005785052A40F0F38241F6F142C2F20102F1
:10CE70001970137872B69B00E36062B6237C012BB5
:10CE800041F25B8272B6E36862B6002BB8BF03332F
:10CE90009B1033604FF0010BFDF782FFFFF7C7BB1C
:10CEA00072B6D8F80030D8F804101A78087898F8D4
:10CEB000091098F80830084202EA030200F0828064
:10CEC00098F80A3003F003030AB143F0040343F077
:10CED00008039A10082B88F80A2000F28D82072B8D
:10CEE00080F00185032B00F0058540F23585042B89
:10CEF00000F08D82062B7FF49CACD8F80C30023BFE
:10CF0000C8F80C3097E44DF6C063C2F200031B7CF6
:10CF100072B69B00E36062B6237C012B40F221864F
:10CF200072B6E36862B6002BB8BF03339B10336060
:10CF3000AB46FEF739FBFFF77ABB4DF6C063C2F292
:10CF4000000393ED027A27EE087A27EE097AC7EEFE
:10CF5000087A77EEA87AFDEEE77A17EE903A9B0012
:10CF600072B6E36062B6237C012B40F2CD8572B6C7
:10CF7000E36862B6002BB8BF03339B103360AB4647
:10CF8000FDF766F9FFF753BB0D2B3FF489AE0E2B6F
:10CF90007FF468ABE3680133E360FFF764BBE368E9
:10CFA0000233E360FFF75FBB012B3DD0022B3FF460
:10CFB00038AFFFF79FBB012B41D0022B3FF440AFAE
:10CFC000FFF7AFBB98F80A3003F00303002A80D0C4
:10CFD00043F004037DE7072A00F02082082A40F08E
:10CFE000368240F26C52C2F20102062112781970A8
:10CFF00072B69300E36062B6237C012B41F280811C
:10D0000072B6E36862B6002BB8BF03339B1033607F
:10D010004FF0010BFEF762FCFFF709BB0D2B3FF44D
:10D0200000AF0E2B7FF466ABE1680131E160FFF7E2
:10D0300062BB0D2B3FF404AF0E2B7FF472ABE368A1
:10D040000133E360FFF76EBB237C012B41F2CC81FF
:10D0500072B6E36862B6032B40F3DE85237C012BB6
:10D0600041F2308272B6E36862B6CB2B03DD72B652
:10D07000C823E36062B6237C012B41F2AF8172B614
:10D08000E36862B6002BB8BF0333C3F3870307EE30
:10D09000903A9FED907AF8EE676A41F67469C6EEB1
:10D0A000877AC2F2010989F80030B7EE007A77EE8C
:10D0B000A87A37EE677AB4EEE97AF1EE10FA00F367
:10D0C0003B84DFED826AB4EEE67AF1EE10FA00F10D
:10D0D000F585F0EE476AFEEEC86A16EE903A41F228
:10D0E000BC42C2F20102F4EEE97AF1EE10FA936169
:10D0F00000F31D849FED757AF4EEC77AF1EE10FA15
:10D1000000F1EA85B0EE677ABEEEC87A17EE103A03
:10D11000F4EEE97AF1EE10FAD36101F39E849FED0B
:10D120006B7AF4EEC77AF1EE10FA00F1D085B0EE2A
:10D13000677ABEEEC87A17EE103A46F2B4001921AB
:10D14000C0F20200136210F0DFFE4EF2402099F8A8
:10D15000001000230A22C2F2000011F0FBFD4EF283
:10D160004020C2F2000011F0E3FDFFF7A5BA022251
:10D170001A70237C012B40F2388672B6E36862B6DF
:10D18000032B40F32A8441F6CC49237CC2F20109E7
:10D19000012B99F800B041F2F68072B6E36862B6EE
:10D1A000002BB8BF0333BBEBA30F06DC99F80030AC
:10D1B000013B9B0072B6E36062B6237C012B40F218
:10D1C000EA8572B6E36862B61A1EB8BF03324DF63E
:10D1D000C063C2F38702C2F2000310461A710293C1
:10D1E00003F042F9029B5979187903F025FCF9F70D
:10D1F000F5FAF8E54DF6C063C2F2000301215B7950
:10D20000117072B69B00E36062B6237C8B4240F2E1
:10D21000318172B6E36862B6002BB8BF03339B104E
:10D2200033600CE572B60023E36062B6FFF7B6BA6E
:10D2300072B60023E36062B6FFF7A1BBE16802317A
:10D24000E160FFF758BAE3680233E360FFF76ABAB8
:10D250004DF6BE624DF6C063C2F20002C2F2000398
:10D2600082F800905B7972B69B00E36062B6237C23
:10D27000012B40F2118672B6E36862B6002BB8BF8C
:10D2800003339B103360FCF7E3FFFFF7D0B94DF693
:10D29000BE6240F26C53C2F20002C2F201030621E8
:10D2A00011701B7872B69B00E36062B6237C012B81
:10D2B00040F2C58572B6E36862B6002BB8BF03338F
:10D2C0009B103360FEF70AFBFFF7B1B900FEFFC603
:10D2D000000096440000484279783042237C012BBC
:10D2E00040F23F8672B6E36862B6032B40F3D18307
:10D2F000237C012B41F24D8072B6E36862B6B3F530
:10D30000C87F04DB72B64FF4C873E36062B6237C57
:10D31000012B40F2788772B6E36862B6002B227C5C
:10D32000B8BF03339B10012A46F8043C40F2138730
:10D3300072B6E36862B641F6F142002B217CB8BFB9
:10D340000333C2F201029B100129137040F22F87B0
:10D3500072B6E36862B6002BB8BF03339B1007EECA
:10D36000903AF8EEE77A41F2905B87EE887AC2F263
:10D37000010B40F24459DBF80030C2F2010945F6D6
:10D38000CC7014222621C0F20200A9F80420F7EE86
:10D39000007A37EEC77AD3ED597A77EE677AF3EEF3
:10D3A000046A87EEA67A89ED007A10F0ADFDDBF80D
:10D3B0000030D3F8640116F0C9FB41EC100B4EF2BB
:10D3C00040200521C2F2000011F004FD45F6F47082
:10D3D0001821C0F2020010F097FD4EF24020B9F87B
:10D3E0000410C2F2000011F045FC46F21000C0F239
:10D3F00002001821FFF7E1BB0C2B00F07B8200F24A
:10D400006C82092B3FF479AD0B2B7FF412AAD8F86C
:10D410000C30013BC8F80C30FFF70DBA41F67462CE
:10D42000C2F2010208211278197072B69300E3600B
:10D4300062B6237C012B41F27F8172B6E36862B64B
:10D44000002BB8BF03339B103360FEF747FA4FF051
:10D45000010BFFF7ECB84DF6C063C2F200030021E8
:10D460001B79117072B69B00E36062B6237C012BBE
:10D470003FF6CFAE72B62046F7F734FDCAE6237CFE
:10D48000012B40F28C8772B6E36862B6032B40F33F
:10D49000CD83237C012B41F23D8072B6E36862B6F6
:10D4A0008F2B03DD72B68C23E36062B6237C012BE5
:10D4B00040F28E8772B6E36862B6002BB8BF0333C2
:10D4C000C3F3870307EE903AB8EE677A41F6F04966
:10D4D000C7EE0A7AC2F2010989F8003077EEA87A1D
:10D4E000F4EEE97AF1EE10FA00F31D821FED897A6D
:10D4F000F4EEC77AF1EE10FA00F1E583B0EE677A48
:10D50000BEEEC87A17EE103A41F28442C2F201022E
:10D5100046F298001B21C0F20200D36110F0F4FC27
:10D5200099F8003007EE903AF8EE677A87EE8A7A3B
:10D5300077EE287A17EE900A16F008FB41EC100BF4
:10D540004EF240200221C2F2000011F043FC4EF2E4
:10D550004020C2F2000011F0EBFBFFF7ADB8237CD6
:10D56000012B40F22F8772B6E36862B6032B40F3BB
:10D570004E83237C012B40F2DC8772B6E36862B6EF
:10D58000CB2B03DD72B6C823E36062B6237C012B8C
:10D5900040F2128772B6E36862B6002BB8BF03335D
:10D5A000C3F3870307EE903AB8EE677A5FEDB87A77
:10D5B0005FEDB86A67EE277A40F26C5987EEA67A7B
:10D5C000C2F2010989F8003077EE287AF5EEC07AC8
:10D5D000F1EE10FA00F126835FEDC16AB6EE007A33
:10D5E000A7EEA67A49F68073C0F20103FCEEC77A73
:10D5F00017EE90EA9E4540F274839E464FF45070B9
:10D6000040F22073C2F201031A7ED10700F1998122
:10D61000D98BC3F820E0814242F0010238BFD883A1
:10D620001A7646F280001721C0F2020010F06CFC5E
:10D6300099F800104FF4966348F21F5203FB01F370
:10D64000C5F2EB1282FB03124EF24020D917C1EB58
:10D650002211C2F2000011F00DFB4EF24020C2F286
:10D66000000011F065FBFFF727B872B694E80C00D4
:10D6700010781978637A227A194202EA000200F0DF
:10D680008481A37A03F003030AB143F0040343F057
:10D6900008039A10082BA27200F2A581072B80F0D4
:10D6A0002785032B00F0528540F21486042B00F0EE
:10D6B000A581062B7FF451A9E368023BE360FFF7E5
:10D6C0004DB972B694E80C0010781978637A227A12
:10D6D000194202EA000200F04F81A37A03F003032B
:10D6E0000AB143F0040343F008039A10082BA27216
:10D6F00000F29981072B80F0F084032B00F0BA85AB
:10D7000040F2F685042B00F09981062B7FF44BA89C
:10D71000E368023BE360FFF747B872B694E80C0099
:10D7200010781978637A227A194202EA000200F02E
:10D730003E81A37A03F003030AB143F0040343F0EC
:10D7400008039A10082BA27200F27D81072B80F04B
:10D75000F384032B00F0E58440F20586042B00F0EF
:10D760007D81062B7FF408A8E368023BE360FFF7A6
:10D7700004B872B694E80C0010781978637A227AAB
:10D78000194202EA000200F00981A37A03F00303C0
:10D790000AB143F0040343F008039A10082BA27265
:10D7A00000F23181072B80F06085032B00F0A58407
:10D7B00040F2AC85042B00F03181062B7FF4F1A8F8
:10D7C000E368023BE360FFF7EDB872B694E80C0043
:10D7D00010781978637A227A194202EA000200F07E
:10D7E000C280A37A03F00303002A41F03B8143F097
:10D7F00008039A10082BA27200F23581072B80F0E3
:10D80000AB83032B00F09D8440F2B585042B00F020
:10D810003581062B7FF4B8A8E368023BE360FFF78D
:10D82000B4B803221A70FFF7ACBA72B694E80C00D1
:10D8300010781978637A227A194202EA000200F01D
:10D84000BD81A37A03F003030AB143F0040343F05C
:10D8500008039A10082BA27200F2B981072B80F0FE
:10D86000E585032B00F0E78540F2FC85042B00F0F2
:10D87000B981062B7EF48AAFE368023BE360FEF7D2
:10D8800086BF72B694E80C0010781978637A227A11
:10D89000194202EA000200F02E81A37A03F003038A
:10D8A0000AB143F0040343F008039A10082BA27254
:10D8B00000F29D81072B80F0A385032B00F0A58546
:10D8C00040F2D785042B00F09D81062B7FF44FA8F2
:10D8D000E368023BE360FFF74BB80D2B3FF497ADD5
:10D8E0000E2B7EF4A6AFD8F80C300133C8F80C30FC
:10D8F000FEF7A1BFD8F80C300233C8F80C30FEF7A1
:10D900009ABF41F6F042C2F201020721FFF76EBB57
:10D9100040F21C02C2F2010205211278197072B69F
:10D920009300FFF7A9BA0023C7F6FF73ECE50023C5
:10D93000C7F6FF73D36100E40023C7F6FF73FFF758
:10D94000CEBB196A8E4540F27681DA8BC3F820E0AF
:10D95000824238BFD88364E6012BC4D0022B3FF447
:10D9600056ADFEF766BFA37A03F00303002A3FF427
:10D9700040AF43F004033CE7A37A03F00303002A1B
:10D980003FF4B3AE43F00403AFE6A37A03F003031E
:10D99000002A3FF47EAE43F004037AE6A37A03F054
:10D9A0000303002A3FF4F9AE43F00403F5E6A37A3B
:10D9B00003F00303002A3FF4C4AE43F00403C0E6BF
:10D9C0004DF6C063C2F200031A79002A40F0ED84DC
:10D9D00072B6E26062B6FFF7F3B972B60023E36095
:10D9E00062B6FFF7EABB0C2B00F0B08300F27A833B
:10D9F000092B3FF461AE0B2B7EF4AFAFE368013B24
:10DA0000E360FEF7ABBF0C2B00F0778300F22784B6
:10DA1000092B3FF4D5AE0B2B7EF4C3AFE368013B7B
:10DA2000E360FEF7BFBF0C2B00F0248400F24F83AD
:10DA3000092B3FF46DAE0B2B7EF4B5AEE368013BD2
:10DA4000E360FEF7B1BE0C2B00F06B8300F26E8337
:10DA5000092B3FF489AE0B2B7EF48EAEE368013BBD
:10DA6000E360FEF78ABE0C2B00F06B8300F26E823F
:10DA7000092B3FF4D1AE0B2B7EF486AFE368013B5C
:10DA8000E360FEF782BF72B60023E36062B6FFF781
:10DA900021B872B60023E36062B638E472B658F873
:10DAA0000C2C636810781978637A227A194202EA9A
:10DAB000000200F0ED83A37A03F00303002A40F094
:10DAC000E58743F008039A10082BA27200F2F28354
:10DAD000072B80F05586032B00F03B8640F2328600
:10DAE000042B00F0F283062B7FF4C9A8E368023B05
:10DAF000E360FFF7C5B8A37A03F00303002A3FF4FD
:10DB0000D4AE43F00403D0E672B658F80C2C636828
:10DB100010781978637A227A194202EA000200F03A
:10DB2000AE83A37A03F003030AB143F0040343F086
:10DB300008039A10082BA27200F20584072B80F0CC
:10DB40004186032B00F0338640F22A86042B00F036
:10DB50000584062B7FF40CAAE368023BE360FFF721
:10DB600008BA72B658F80C2C636810781978637A82
:10DB7000227A194202EA000200F09383A37A03F0AA
:10DB800003030AB143F0040343F008039A10082B7F
:10DB9000A27200F2C283072B80F0FD85032B00F0F8
:10DBA000E48540F2DB85042B00F0C283062B7FF472
:10DBB000B8A9E368023BE360FFF7B4B9A37A03F0C6
:10DBC0000303002A3FF445AE43F0040341E60C2B67
:10DBD00000F0318400F22484092B3FF44DAE0B2B6E
:10DBE0007EF4D4ADE368013BE360FEF7D0BD0C2BBF
:10DBF00000F00B8400F2FE83092B3FF469AE0B2B7F
:10DC00007EF4B5AEE368013BE360FEF7B1BE72B6E9
:10DC10000023E36062B6B9E472B60023E36062B643
:10DC2000FFF729BA01204FF0000EE9E472B6002395
:10DC3000E36062B63AE49107C3F820E006D5596A7A
:10DC40007F31C9090131884238BF0846510706D5DE
:10DC5000996A7F31C9090131884238BF08461107E6
:10DC600006D5D96A7F31C9090131884238BF0846D3
:10DC7000D10606D5196B7F31C9090131884238BFF9
:10DC80000846910606D5596B7F31C9090131884292
:10DC900038BF0846510606D5996B7F31C909013155
:10DCA000884238BF0846D20906D0DA6B7F32D209E3
:10DCB0000132904238BF1046D883B2E40023C8F244
:10DCC0000103FFF70CBA0023C8F201031CE4002390
:10DCD000C8F20103FFF731BA0023C8F20103FFF7CE
:10DCE00017BA0EF17F00C009013089E472B694E8DA
:10DCF0000C0010781978637A227A194202EA00023D
:10DD000040F0BE83A37A03F00303002A40F0C286EA
:10DD10009A10082BA27200F21284072B80F0108652
:10DD2000032B00F0DC8540F2D385042B00F0128435
:10DD3000062B7FF42BA8E368023BE360FFF727B8CC
:10DD400072B694E8060091F800E01078627A217AC1
:10DD500010420EEA010140F07383A27A02F003023E
:10DD6000002940F083869110082AA17200F2F783FF
:10DD7000072A80F0CF85032A00F0358640F22C86F2
:10DD8000042A00F0F783062A7FF41FA8E268023A0B
:10DD9000E260FFF71BB872B694E80C0010781978AF
:10DDA000637A227A194202EA000240F05283A37A8F
:10DDB00003F00303002A40F05D869A10082BA2723C
:10DDC00000F27083072B80F07285032B00F07B85B7
:10DDD00040F27285042B00F07083062B7FF4F2A9C9
:10DDE000E368023BE360FFF7EEB972B694E80C001B
:10DDF00010781978637A227A194202EA000240F018
:10DE00004883A37A03F00303002A40F047869A1060
:10DE1000082BA27200F26E83072B80F0B185032BD2
:10DE200000F0238540F21985042B00F06E83062B49
:10DE30007FF4A4A9E368023BE360FFF7A0B972B6E0
:10DE400058F80C2C636810781978637A227A194292
:10DE500002EA000200F04583A37A03F003030AB14B
:10DE600043F0040343F008039A10082BA27200F257
:10DE70002384072B80F0C084032B00F0C98440F278
:10DE8000C084042B00F02384062B7FF414AAE368DB
:10DE9000023BE360FFF710BA72B658F80C2C6368C7
:10DEA00010781978637A227A194202EA000200F0A7
:10DEB0000F83A37A03F003030AB143F0040343F092
:10DEC00008039A10082BA27200F2CD83072B80F072
:10DED0007385032B00F0658540F25C85042B00F010
:10DEE000CD83062B7FF4C8A9E368023BE360FFF70C
:10DEF000C4B972B658F80C2C636810781978637A34
:10DF0000227A194202EA000200F00A83A37A03F09F
:10DF100003030AB143F0040343F008039A10082BEB
:10DF2000A27200F24583072B80F0AA84032B00F035
:10DF3000B38440F2AA84042B00F04583062B7EF4C0
:10DF4000C4ACE368023BE360FEF7C0BC0D2B3FF4BA
:10DF500095AD0E2B7EF418ADE3680133E360FEF758
:10DF600014BD72B694E80C0010781978637A227A9E
:10DF7000194202EA000200F0BF83A37A03F0030310
:10DF8000002A40F07B8543F008039A10082BA27208
:10DF900000F2A283072B80F04684032B00F0F58467
:10DFA00040F22685042B00F0A283062B7FF49BA968
:10DFB000E368023BE360FFF797B972B62046F6F7D5
:10DFC00091FFFEF7A9BD72B694E80C00107819789D
:10DFD000637A227A194202EA000200F0D082A37A20
:10DFE00003F00303002A40F04D8543F008039A1024
:10DFF000082BA27200F2CC82072B80F07B84032BCB
:10E0000000F07D8440F20A85042B00F0CC82062BC0
:10E010007EF472ADE368023BE360FEF76EBD72B65C
:10E0200094E80C0010781978637A227A194202EA8F
:10E03000000200F03883A37A03F003030AB143F02F
:10E04000040343F008039A10082BA27200F21B830A
:10E05000072B80F08584032B00F0878440F2D08466
:10E06000042B00F01B83062B7EF439ADE368023BE2
:10E07000E360FEF735BD72B694E80C0010781978AD
:10E08000637A227A194202EA000200F0E382A37A5C
:10E0900003F003030AB143F0040343F008039A10AA
:10E0A000082BA27200F2C682072B80F03E84032B5D
:10E0B00000F04B8440F2AB84042B00F0C682062BA8
:10E0C0007EF4F4ACE368023BE360FEF7F0BC0D2B9A
:10E0D0003FF4B4AC0E2B7EF466ABE3680133E3602F
:10E0E000FEF762BB0D2B3FF489AC0E2B7EF435ACF2
:10E0F000E3680133E360FEF731BCE3680233E360B9
:10E10000FEF750BC72B60022E26062B61A790132A4
:10E11000D2B210461A71029302F0A6F9029BFEF7E2
:10E120004FBEE3680233E360FEF727BB0D2B3FF4DD
:10E1300095AC0E2B7EF420ABE3680133E360FEF771
:10E140001CBBE3680233E360FEF71FBCE3680233E5
:10E15000E360FEF703BC72B694E80C0010781978FF
:10E16000637A227A194202EA000200F0CE82A37A90
:10E1700003F003030AB143F0040343F008039A10C9
:10E18000082BA27200F22482072B80F05783032B06
:10E1900000F0598340F25184042B00F02482062BB6
:10E1A0007FF4C7A8E368023BE360FFF7C3B872B629
:10E1B00094E80C0010781978637A227A194202EAFE
:10E1C000000200F02E82A37A03F003030AB143F0A9
:10E1D000040343F008039A10082BA27200F29E82F7
:10E1E000072B80F0FE82032B00F0F18240F22D8499
:10E1F000042B00F09C82062B7FF4ABA8E368023B63
:10E20000E360FFF7A7B872B694E80C0010781978AD
:10E21000637A227A194202EA000200F0F981A37AB5
:10E2200003F003030AB143F0040343F008039A1018
:10E23000082BA27200F2DC81072B80F0C883032B2D
:10E2400000F0068340F2F283042B00F0DC81062B01
:10E250007FF462A8E368023BE360FFF75EB80D2B32
:10E260003FF4DCAB0E2B7EF49CABE3680133E36040
:10E27000FEF798BBE3680233E360FEF795BAA37A32
:10E2800003F00303002A3FF454AC43F0040350E4CA
:10E29000A37A03F00303002A3FF415AC43F0040310
:10E2A00011E4A37A03F00303002A3FF46FAC43F0B8
:10E2B00004036BE40C2B00F04C8200F25B82092B10
:10E2C0003FF414AC0B2B7EF4DAACE368013BE36063
:10E2D000FEF7D6BC012B3FF40BAF022B3FF48EAB05
:10E2E000FEF73BBB72B62046F6F7FCFDFEF758BDC5
:10E2F000012B3FF4F2AE022B3FF4A0ABFEF753BA72
:10E3000072B62046F6F7EEFDFEF77BBE012BACD0D1
:10E31000022B3FF483ABFEF744BB0C2B00F02582AD
:10E3200000F23382092B3FF444AC0B2B7EF4F9ADA1
:10E33000E368013BE360FEF7F5BD72B62046F6F7F1
:10E34000D1FDFEF7A0BD0C2B00F0318200F234822B
:10E35000092B3FF401AC0B2B7EF40AAEE368013BC2
:10E36000E360FEF706BE012B3FF4E6AE022B3FF45E
:10E3700075ABFEF701BA012B3FF4EEAD022B3FF473
:10E380007DABFEF701BB72B62046F6F7ABFDFEF79C
:10E3900005BF72B62046F6F7A5FDFEF7AEBF72B612
:10E3A0002046F6F79FFDFFF76FB872B67C22E26059
:10E3B00062B61A79013AABE672B62046F6F792FDDC
:10E3C000FFF7E9B872B62046F6F78CFDFFF7CCB838
:10E3D00072B62046F6F786FDFFF76DB872B6204696
:10E3E000F6F780FDFEF74CBE72B62046F6F77AFDD2
:10E3F000FEF72FBE0D2B3FF405AC0E2B7EF4B7AA13
:10E40000E3680133E360FEF7B3BAE3680233E36025
:10E41000FEF7AEBA72B62046F6F764FDFEF750BBC3
:10E420000D2B3FF4DFAB0E2B7EF4B0A9E368013374
:10E43000E360FEF7ACB9E3680233E360FEF7A7B927
:10E44000A27A02F0030209B142F0040242F008028B
:10E4500089E4A37A03F003030AB143F0040343F011
:10E460000803AAE4012BE1D0022B3FF4BBABFEF77B
:10E470008DB9012BC4D0022B3FF4C4ABFEF777BAA1
:10E48000A37A03F003030AB143F0040343F0080343
:10E490003EE4A37A03F003030AB143F0040343F01C
:10E4A0000803B4E40C2B00F00E8200F2FA81092B71
:10E4B0003FF496AC0B2B7EF485AEE368013BE36042
:10E4C000FEF781BE72B62046F6F70CFDFEF7CBBD17
:10E4D000A37A03F00303002A3FF4F3AC43F00403F0
:10E4E000EFE4A37A03F00303002A3FF4BDAC43F04A
:10E4F0000403B9E40C2B00F0B88100F23B82092B35
:10E500003FF498AC0B2B7EF439AEE368013BE3603B
:10E51000FEF735BE72B62046F6F7E4FCFEF7BEBF46
:10E52000A37A03F00303002A3FF4F8AC43F004039A
:10E53000F4E472B62046F6F7D5FCFFF71FB80C2BB3
:10E5400000F0CD8100F2F681092B3FF4F4AB0B2BE8
:10E550007EF41CACE368013BE360FEF718BC0C2AB8
:10E5600000F0418200F2D081092A3FF40FAC0B2A5F
:10E570007EF42BACE268013AE260FEF727BCA37A96
:10E5800003F00303002A3FF432AD43F004032EE509
:10E590000C2B00F0B48100F2A781092B3FF43AADB7
:10E5A0000B2B7EF4A9AAE368013BE360FEF7A5BA52
:10E5B0000C2B00F0718100F25D81092B3FF4C1AC9E
:10E5C0000B2B7EF482A9E368013BE360FEF77EB982
:10E5D0000C2B00F0388100F22B81092B3FF4E2ADC7
:10E5E0000B2B7EF4A6AEE368013BE360FEF7A2BE10
:10E5F0000C2B00F02D8100F2E481092B3FF42AAEB0
:10E600000B2B7EF489AEE368013BE360FEF785BE29
:10E61000A37A03F00303002A3FF409AE43F0040396
:10E6200005E6A37A03F00303002A3FF4D4AD43F0D8
:10E630000403D0E50C2B00F0888100F27081092BD7
:10E640003FF440AD0B2B7EF431AAE368013BE3605D
:10E65000FEF72DBAA37A03F00303002A3FF41FAD9F
:10E6600043F004031BE50C2B00F09B8100F29E811C
:10E67000092B3FF439AC0B2B7EF4FEADE368013B74
:10E68000E360FEF7FABD0C2B00F06F8100F26281AF
:10E69000092B3FF4EBAC0B2B7EF421AAE368013B82
:10E6A000E360FEF71DBAA37A03F00303002A3FF4E8
:10E6B000CAAC43F00403C6E40C2B00F0A98000F2BE
:10E6C0009580092B3FF4E3AB0B2B7EF4F4ADE368AC
:10E6D000013BE360FEF7F0BD0C2B00F0568100F229
:10E6E0009C80092B3FF464AC0B2B7EF4FCADE368FB
:10E6F000013BE360FEF7F8BDA37A03F00303002AB1
:10E700003FF443AC43F004033FE4A37A03F0030374
:10E71000002A3FF434AD43F0040330E50C2B56D00F
:10E720005AD8092B3FF46AAD0B2B7EF412AEE36886
:10E73000013BE360FEF70EBE72B62046F6F7D2FB51
:10E74000FEF77CBE012B1BD0022B3FF4BEADFEF7C3
:10E7500096BAE3680233E360FEF792BA012B1AD04F
:10E76000022B3FF4E5ADFEF7DCBBE3680233E36068
:10E77000FEF7D8BB0D2B3FF4A8AD0E2B7EF47FAA7D
:10E78000E3680133E360FEF77BBA0D2B3FF4D0ADB5
:10E790000E2B7EF4C6ABE3680133E360FEF7C2BB29
:10E7A000012B0FD0022B3FF4D9ADFEF7E1BBE3689C
:10E7B0000233E360FEF7DDBB0D2B3FF4CFAD0E2B34
:10E7C0007EF4D6ABE3680133E360FEF7D2BBE368C7
:10E7D0000233E360FEF7BEBD0D2BA8D00E2B7EF4F6
:10E7E000B8ADE3680133E360FEF7B4BD0D2B3FF431
:10E7F0006EAF0E2B7EF45FADE3680133E360FEF78E
:10E800005BBD012BF8D0022B3FF461AFFEF753BD87
:10E81000E3680233E360FEF74FBD0D2B3FF467AFB3
:10E820000E2B7EF460ADE3680133E360FEF75CBD60
:10E830000D2B3FF4D8AE0E2B7EF47BADE368013395
:10E84000E360FEF777BDE3680233E360FEF772BD75
:10E85000E3680233E360FEF760BD012B00F09080B7
:10E86000022B3FF452AEFEF789BCE3680233E3604B
:10E87000FEF785BC0D2B3FF4A6AE0E2B7EF425A82B
:10E88000E3680133E360FEF721B8012BF8D0022BD7
:10E890003FF499AEFEF719B8E3680233E360FEF780
:10E8A00015B80D2B3FF409AE0E2B7EF48BACE3684C
:10E8B0000133E360FEF787BC012BF8D0022B3FF455
:10E8C000FCADFEF77FBCE3680233E360FEF77BBC80
:10E8D000012B35D0022B3FF43DAEFEF757BAE3686B
:10E8E0000233E360FEF753BA0D2B3FF45CAE0E2B00
:10E8F0007EF402A9E3680133E360FEF7FEB8E36843
:10E900000233E360FEF7F9B80D2A3FF433AE0E2A66
:10E910007EF45BAAE2680132E260FEF757BA0D2B83
:10E920003FF493AE0E2B7EF4C1A8E3680133E3609D
:10E93000FEF7BDB80D2B3FF40DAE0E2B7EF426AACC
:10E94000E3680133E360FEF722BAE3680233E36071
:10E95000FEF7ADB80D2B3FF4A1AE0E2B7EF4BFA891
:10E96000E3680133E360FEF7BBB8E3680233E360BA
:10E97000FEF7B6B80D2B3FF4C8AD0E2B7EF4FEAB00
:10E98000E3680133E360FEF7FABBE3680233E36058
:10E99000FEF7AABC012B0FD0022B3FF46FAEFEF79F
:10E9A0006BBCE3680233E360FEF767BC0D2B3FF4FA
:10E9B00065AE0E2B7EF460ACE3680133E360FEF7D6
:10E9C0005CBC0D2B3FF41FAE0E2B7EF4A5ACE368B0
:10E9D0000133E360FEF7A1BC012A9BD0022A3FF479
:10E9E000C9ADFEF7F2B9E2680232E260FEF7EEB9B5
:10E9F000012B3FF418AF022B3FF479AEFEF773BC46
:10EA0000012BADD0022B3FF449AEFEF768B8012BC5
:10EA10008BD0022B3FF419AEFEF748B8012B3FF420
:10EA200069AF022B3FF4BFADFEF766B8012BCED025
:10EA3000022B3FF4E8ADFEF76FBC012B3FF4FEAEB6
:10EA4000022B3FF4D0ADFEF774BC012B3FF4C9AEEE
:10EA5000022B3FF46CAEFEF77CBC0023C7F6FF73BD
:10EA6000FEF76BBB43F00403FEF7C1BE42F00402A5
:10EA7000FFF779B943F00403FFF79FB943F00403AC
:10EA8000FFF781BA43F00403FFF7AFBA43F0040382
:10EA9000FFF717B843F00403FFF73AB943F0040354
:10EAA000FFF7B5B92DE9F0432DED028B05460027A0
:10EAB00083B000F1F004204685F8D97085F8DA704B
:10EAC00085F8DB7085F8DC7085F8DD7085F8DE7020
:10EAD00085F8DF7085F8E07085F8E17085F8E27000
:10EAE00085F8E37085F8E47085F8E57085F8E670E0
:10EAF00085F8E77085F8E87085F8CC7085F8CD70FA
:10EB000085F8CE700191FAF7FDFE46F2DC01AD22E8
:10EB1000C0F2020105F5B6700CF088FC102385F8F0
:10EB2000193202F0F7FF03F045F803F00BFDDDEDBD
:10EB3000017AB8EEE78A2E46B0EE480A03F002FBEF
:10EB4000B0EE480A03F04AFBB0EE480A03F026FC98
:10EB5000B0EE480A02F0E0FD01992046FAF7DAFE2D
:10EB60004FF4097010F052FA0446F1F789FCC5F829
:10EB70005C424FF4097010F049FA45F23823C0F2B4
:10EB800002030360C5F860024FF4097010F03EFA0A
:10EB900046F29C43C0F20203C5F85802036005F137
:10EBA000C0092C464FF4257010F030FA80460C3422
:10EBB00002F03EF844F8048C04F80A7C04F8097C5E
:10EBC00004F8087CA1454FF00003EBD195F8D9205B
:10EBD0009FEDD06ADFEDCE6A85F81A3207EE902AF3
:10EBE000B8EEE77A95F8DB20C5F8C43067EE067A10
:10EBF000102067EEA67A4FF40051FCEEE77AC5F8D4
:10EC0000C830CDED017A85F8D23085F8D13085F85D
:10EC1000D03085F8CF3085F8CE3085F8CD3085F806
:10EC2000CC3085F819029DF80430C5F8C0100AB13F
:10EC300085F8CC3095F8DA200AB185F8CD3095F812
:10EC4000DC200AB185F8CE3095F8E1309FEDB16A4D
:10EC5000DFEDAF6A95F8E31007EE903AB8EEE77A89
:10EC600067EE067A67EEA67AFCEEE77ACDED017ADA
:10EC70009DF8043031B195F8CC10994238BF19464F
:10EC800085F8CC1095F8E21031B195F8CD10994285
:10EC900038BF194685F8CD1095F8E40030B195F8E5
:10ECA000CE108B4238BF0B4685F8CE3095F8DD305C
:10ECB0009FED986ADFED966A95F8DF1007EE903ABF
:10ECC000B8EEE77A67EE067A67EEA67AFCEEE77AA8
:10ECD000CDED017A9DF8043031B195F8CC10994210
:10ECE00038BF194685F8CC1095F8DE1031B195F88B
:10ECF000CD10994238BF194685F8CD1095F8E0102F
:10ED000031B195F8CE40A34238BF234685F8CE30C6
:10ED100095F8E5309FED7F6ADFED7D6A95F8E74075
:10ED200007EE903AB8EEE77A67EE067A67EEA67AD3
:10ED3000FCEEE77ACDED017A9DF8043034B195F818
:10ED4000CC409C4238BF1C4685F8CC4095F8E64044
:10ED500034B195F8CD409C4238BF1C4685F8CD4073
:10ED600095F8E84034B195F8CE70BB4238BF3B46C9
:10ED700085F8CE302AB921B918B914B97F2385F89E
:10ED8000CE303F23002485F8D830C5F8D44005F2B2
:10ED9000F51105F5107003F037FA95F81C320BB138
:10EDA00085F81C4295F81E32002485F81B42002B82
:10EDB00000F0EF80D5F8583285F81E42C5F8EC30E7
:10EDC00033793BB1B368B47018463471F4700BB149
:10EDD00002F088FC0C36B145F2D195F8D9309FEDA0
:10EDE0004D6A95F8DB1007EE903A95F8D230B8EE00
:10EDF000E77A06EE903A67EE067AF8EEE66A0022C7
:10EE000067EEA67A85F8CE20FCEEE77A85F8CD206D
:10EE1000CDED017A9DF8043085F8CC2009B185F854
:10EE2000CC3095F8DA200AB185F8CD3095F8DC20A1
:10EE30000AB185F8CE3095F8E1309FED366A95F845
:10EE4000E31007EE903A95F8D030B8EEE77A06EE88
:10EE5000903A67EE067AF8EEE66A67EEA67AFCEE7E
:10EE6000E77ACDED017A9DF8043031B195F8CC10F8
:10EE7000994238BF194685F8CC1095F8E21031B1A7
:10EE800095F8CD10994238BF194685F8CD1095F800
:10EE9000E40030B195F8CE108B4238BF0B4685F8B0
:10EEA000CE3095F8DD309FED1B6A95F8DF1007EE48
:10EEB000903A95F8D130B8EEE77A06EE903A67EEE0
:10EEC000067AF8EEE66A67EEA67AFCEEE77ACDED12
:10EED000017A9DF8043031B195F8CC10994238BFD1
:10EEE000194685F8CC1095F8DE1031B195F8CD10A3
:10EEF000994238BF194685F8CD1095F8E01059B100
:10EF000095F8CE40A34238BF234685F8CE3003E0C3
:10EF1000000000000AD7233C95F8E5301FED036A96
:10EF200095F8E74007EE903A95F8CF30B8EEE77ADB
:10EF300006EE903A67EE067AF8EEE66A67EEA67A93
:10EF4000FCEEE77ACDED017A9DF8043034B195F806
:10EF5000CC409C4238BF1C4685F8CC4095F8E64032
:10EF600034B195F8CD409C4238BF1C4685F8CD4061
:10EF700095F8E84034B195F8CE60B34238BF3346D7
:10EF800085F8CE302AB921B918B914B97F2385F88C
:10EF9000CE30284603B0BDEC028BBDE8F08300BF45
:10EFA0002DE9F04F2DED028B8B00CDB00A3302AF6F
:10EFB00023F007037961ADEB030D90F81D127A6021
:10EFC00002AB06463B6139B390F81932DBB100243D
:10EFD00000F5B67503E00134A4B2A34213D904EBE3
:10EFE000440206EB820108790028F4D04B78886847
:10EFF00016F82220294602F03BF9013496F819321E
:10F00000A4B2A342EBD806F2F51106F5107003F096
:10F01000FBF8002386F81D327B69002B00F0AB80E3
:10F0200007F1270840F2200406F510739FED588A77
:10F03000BB6028F00F08C2F201044FF0000A3B69E0
:10F040004FF4807203EB8A090021404615F068FCFA
:10F0500000214FF48072484615F062FCBD682846D6
:10F0600003F014F98346284603F06AF996F819125A
:10F07000002955D0C7F80CA00025824603E00135D1
:10F08000EDB28D424AD205EB450306EB83031A79B4
:10F09000002AF4D0986806F1C00300935A465346FC
:10F0A000414601F09DFFA8F1040308F1FC0E4A4619
:10F0B000F7EE006ABFEE006A00200DE02168013122
:10F0C0002160B7EE007AD2ED007A186037EE877AC9
:10F0D0007345A2EC017A1BD053F8041F091121F3E8
:10F0E0005721491007EE901AF8EEE77A87EE887AF2
:10F0F000B4EEE67AF1EE10FAE0DCB4EEC67AF1EEA8
:10F1000010FAE0D5216801312160BFEE007ADAE71C
:10F1100096F819120135EDB28D42B4D3D7F80CA090
:10F120007B690AF1400A1FFA8AFA534587D83C697D
:10F130001D4606F1F0001A462146FAF76DFC7A6882
:10F140009FED137A681E80B202EB40002146023A1E
:10F15000F1EC017A67EE877AFDEEE77A17EE903AE6
:10F1600022F8023F8242F3D107F59677BD46BDEC07
:10F17000028BBDE8F08F39691A4606F1F000FAF704
:10F180004BFC07F59677BD46BDEC028BBDE8F08FD2
:10F1900000FEFF462DE9F843054690F8FC3190F853
:10F1A0001962002A00F0D680183BCF1890F81A8216
:10F1B000FFB2002E00F0C5804FEA480909EB0803B2
:10F1C00000EB830341469C78CE46002C00F09380F0
:10F1D000002403E08378002B00F08D80013101349E
:10F1E00091FBF6F306FB1311E4B24FEA410E0EEB6E
:10F1F0000100B44205EB80005FFA81F8EAD195F88E
:10F200001C32002B6ED095F81932002B6AD02A7967
:10F21000002A40F0CF81012B64D92A7C002A40F0DB
:10F22000D781022B5ED02A7F002A40F0CD81032BAC
:10F2300058D095F82820002A40F0C881042B51D0DE
:10F2400095F83420002A40F0B781052B4AD095F874
:10F250004020002A40F0B281062B43D095F84C2084
:10F26000002A40F0AD81072B3CD095F85820002AA9
:10F2700040F0A881082B35D095F86420002A40F092
:10F28000AB81092B2ED095F87020002A40F0A68182
:10F290000A2B27D095F87C20002A40F0A1810B2B67
:10F2A00020D095F88820002A40F09C810C2B19D0A2
:10F2B00095F89420002A40F097810D2B12D095F8F4
:10F2C000A020002A40F092810E2B0BD095F8AC20A4
:10F2D000002A40F07F810F2B04D095F8B830002B26
:10F2E00040F032814FEA4809C84405EB8805012304
:10F2F0002B71BDE8F8838E444FEA8E0E013105EB89
:10F300000E0991FBF6F306FB131685F81A6205F851
:10F310000E7089F8012095F81B3289F8033001211D
:10F32000134689F80210D9F808003A4605F5B67177
:10F3300001F098FC95F8F431002B78D1002C7FF483
:10F340005EAF05F5107003F021F895F81C32002B24
:10F35000C8D058E7183BCF18FBB2002E65D0017813
:10F36000994200F0BB80012E5FD92A7B9A4200F0BF
:10F37000AF80022E59D02A7E9A4200F0A380032E3D
:10F3800053D095F824209A4200F09580042E4CD05A
:10F3900095F830209A4200F08780052E45D095F8E8
:10F3A0003C209A427AD0062E3FD095F848209A42C7
:10F3B0006ED0072E39D095F854209A4262D0082E8C
:10F3C00033D095F860209A4256D0092E2DD095F86A
:10F3D0006C209A424AD00A2E27D095F878209A427B
:10F3E0003ED00B2E21D095F884209A4232D00C2E9C
:10F3F0001BD095F890209A4226D00D2E15D095F866
:10F400009C209A421AD00E2E0FD095F8A8209A422E
:10F4100000F093800F2E08D095F8B4209A4204D1C2
:10F4200095F8B630002B40F0A780BDE8F883D9F8F6
:10F43000080002F057F9002C83D0E0E695F89E20F2
:10F44000002AE0D00D2798E095F89220002AD4D029
:10F450000C2792E095F88620002AC8D00B278CE074
:10F4600095F87A20002ABCD00A2786E095F86E200D
:10F47000002AB0D0092780E095F86220002AA4D0A5
:10F4800008277AE095F85620002A98D0072774E0DC
:10F4900095F84A20002A8CD006276EE095F83E2089
:10F4A000002A80D0052768E095F83220002A3FF432
:10F4B00074AF042761E095F82620002A3FF466AF78
:10F4C00003275AE0AA7E002A3FF459AF022754E0EE
:10F4D000AA7B002A3FF44DAF01274EE08178002936
:10F4E0003FF441AF82701746804695F81C32E3B175
:10F4F0004FF0000E734671464FF0FF3203EB4303AB
:10F5000005EB8304481CA4782CB115F823309342F2
:10F51000C4BF5AB28E4641B2B1420B46EEDB013255
:10F5200003D098F80430002B62D195F81B32C3B396
:10F53000012388F80330BDE8F88395F8AA20002A53
:10F540003FF468AF0E2718E00F2303EB43039B0043
:10F55000EA189178C9B1EB5CBB42BFF466AF4FEAE1
:10F56000480909EB080305EB830300211171986832
:10F57000916802F063F8B7E60F2707EB470805EB41
:10F580008808002388F80230AFE74FEA480909EB02
:10F59000080305EB830311719868916802F06EF817
:10F5A000A2E607EB470205EB8205A868BDE8F84331
:10F5B00001F04ABE0023C8E70423C6E70523C4E7D9
:10F5C0000623C2E70723C0E70223BEE70323BCE705
:10F5D0000123BAE70E23B8E70823B6E70923B4E707
:10F5E0000A23B2E70B23B0E70C23AEE70D23ACE709
:10F5F0000EEB4E0E07EB470205EB8E03002105EBE9
:10F60000820288F80410012119719868916802F04B
:10F6100015F88AE7F8B590F8FC3190F81972183BA4
:10F620001944002F63D00378C9B28B4260D0012FF8
:10F630005DD9037B8B4200F0EA80022F57D0037E16
:10F640008B4200F0DE80032F51D090F824308B42A3
:10F6500000F0D080042F4AD090F830308B4200F078
:10F66000C280052F43D090F83C308B4200F0B4802C
:10F67000062F3CD090F848308B4200F0A680072F30
:10F6800035D090F854308B4200F09880082F2ED05F
:10F6900090F860308B4200F08A80092F27D090F8D4
:10F6A0006C308B427CD00A2F21D090F878308B427E
:10F6B00070D00B2F1BD090F884308B4264D00C2F6D
:10F6C00015D090F890308B4258D00D2F0FD090F875
:10F6D0009C308B424CD00E2F09D090F8A8308B4232
:10F6E00040D00F2F03D090F8B4308B422ED0F8BD0D
:10F6F0008378002B9BD000258570064690F81C323D
:10F700000446E3B100231A469C464FF0FF3E03EB4C
:10F71000430304EB8300511C807830B114F823308C
:10F720007345C4BF4FFA83FE94464AB2BA421346A9
:10F73000EDDBBEF1FF3F02D03379002B76D194F898
:10F740001B32002B69D00123F370F8BD90F8B6305E
:10F75000002BCCD00F2505EB450600EB86060023D9
:10F76000B370CBE790F8AA30002BBAD00E25F2E7A1
:10F7700090F89E30002BAED00D25ECE790F892303B
:10F78000002BA2D00C25E6E790F88630002B96D00F
:10F790000B25E0E790F87A30002B8AD00A25DAE7CB
:10F7A00090F86E30002B3FF47EAF0925D3E790F838
:10F7B0006230002B3FF471AF0825CCE790F856304B
:10F7C000002B3FF463AF0725C5E790F84A30002BC4
:10F7D0003FF455AF0625BEE790F83E30002B3FF4CE
:10F7E00047AF0525B7E790F83230002B3FF439AF2B
:10F7F0000425B0E790F82630002B3FF42BAF03250B
:10F80000A9E7837E002B3FF41EAF0225A3E7837B8D
:10F81000002B3FF412AF01259DE705EB450504EBF6
:10F820008500BDE8F840806801F00EBD0CEB4C0C83
:10F8300005EB450204EB8C03002104EB82023171DD
:10F84000012119719868916801F0F8FE77E700BF0F
:10F85000012380F81D32704790F81C328B4218BF8C
:10F8600080F81C12704700BF90F81B328B4218BF03
:10F8700080F81B12704700BF90F81B02704700BF52
:10F8800070B5044600F1C006002523793BB1A3689A
:10F89000A57018462571E5700BB101F023FF0C34FB
:10F8A000B442F2D170BD00BF90F8D9309FED6C6AC0
:10F8B000DFED6C6A90F8DB1007EE903AB8EEE77A6D
:10F8C00070B467EE067A83B067EEA67A0023FCEE8A
:10F8D000E77A4FF40052CDED017AC0F8C020C0F8AD
:10F8E000C4309DF80420C0F8C83080F8D23080F8C9
:10F8F000D13080F8D03080F8CF3080F8CE3080F82A
:10F90000CD3080F8CC3009B180F8CC2090F8DA30D6
:10F910000BB180F8CD2090F8DC1009B180F8CE2032
:10F9200090F8E1309FED4E6ADFED4E6A90F8E320EB
:10F9300007EE903AB8EEE77A67EE067A67EEA67AB7
:10F94000FCEEE77ACDED017A9DF8043032B190F803
:10F95000CC209A4238BF1A4680F8CC2090F8E2209A
:10F9600032B190F8CD209A4238BF1A4680F8CD20A7
:10F9700090F8E44034B190F8CE20934238BF13465B
:10F9800080F8CE3090F8DD309FED356ADFED356AD6
:10F9900090F8DF2007EE903AB8EEE77A67EE067A45
:10F9A00067EEA67AFCEEE77ACDED017A9DF8043099
:10F9B00032B190F8CC209A4238BF1A4680F8CC2059
:10F9C00090F8DE2032B190F8CD209A4238BF1A4626
:10F9D00080F8CD2090F8E02032B190F8CE50AB42C4
:10F9E00038BF2B4680F8CE3090F8E5309FED1C6A8A
:10F9F000DFED1C6A90F8E75007EE903AB8EEE77A30
:10FA000067EE067A67EEA67AFCEEE77ACDED017A2C
:10FA10009DF8043035B190F8CC509D4238BF1D465A
:10FA200080F8CC5090F8E65035B190F8CD509D421A
:10FA300038BF1D4680F8CD5090F8E85035B190F8A9
:10FA4000CE60B34238BF334680F8CE3029B922B9F0
:10FA50001CB915B97F2380F8CE3003B070BC704755
:10FA60000AD7233C0000000003791BB18378002BE8
:10FA700040F09A80037C1BB1837B002B40F0918087
:10FA8000037F1BB1837E002B40F0888090F82830E4
:10FA90001BB190F82630002B7CD190F834301BB18C
:10FAA00090F83230002B71D190F840301BB190F8B3
:10FAB0003E30002B66D190F84C301BB190F84A30A4
:10FAC000002B5BD190F858301BB190F85630002BCA
:10FAD00050D190F864301BB190F86230002B45D1C2
:10FAE00090F8703013B190F86E30DBBB90F87C303A
:10FAF00013B190F87A308BBB90F8883013B190F83E
:10FB000086303BBB90F8943013B190F89230EBB94B
:10FB100090F8A03013B190F89E309BB990F8AC30BB
:10FB200013B190F8AA304BB990F8B8302BB190F8D7
:10FB3000B63013B1002380F8B6307047002380F848
:10FB4000AA30F1E7002380F89E30E7E7002380F831
:10FB50009230DDE7002380F88630D3E7002380F879
:10FB60007A30C9E7002380F86E30BFE7002380F8C1
:10FB70006230B5E7002380F85630AAE7002380F80A
:10FB80004A309FE7002380F83E3094E7002380F856
:10FB9000323089E7002380F826307EE70023837621
:10FBA00074E7002383736BE70023837062E700BF71
:10FBB00090F81902704700BF2DE9F04F054690F804
:10FBC000F211D0F8EC0085B002F030F995F8191276
:10FBD000002900F0C780C0F3C0030093C0F30013F6
:10FBE00000260193C0F34013344600F00108C0F32F
:10FBF000400BC0F3800A029305F5087703E0013457
:10FC0000E4B2A1427CD904EB440305EB830999F8E3
:10FC10000420002AF3D000212022384614F080FE70
:10FC20003946D9F8080001F0CBFCB8F1000F6BD0D1
:10FC3000D5F8201240F22D42914269D895F8381239
:10FC4000A1F10401B1FA81F1022049090122BBF1BD
:10FC5000000F0AD0D5F8242240F22D4E724503D869
:10FC600095F83922042A57D00246BAF1000F0DD078
:10FC7000D5F8280240F22D4E01327045D2B205D897
:10FC800095F83A02042804BF0131C9B2009B6BB158
:10FC9000D5F82C0240F22D4E01327045D2B205D873
:10FCA00095F83B02042804BF0131C9B2019B6BB136
:10FCB000D5F8300240F22D4E01327045D2B205D84F
:10FCC00095F83C02042804BF0131C9B2029B6BB114
:10FCD000D5F8340240F22D4E01327045D2B205D82B
:10FCE00095F83D02042804BF0131C9B2914217D0F2
:10FCF00095F819120134E4B20136A142F6B282D865
:10FD0000304605B0BDE8F08F0120424641469EE7EF
:10FD10000220012200219AE70131C9B20246A4E77C
:10FD2000002246F28C1089F8042089F8032089F813
:10FD300002201021C0F2020003920EF0E5F8039AAF
:10FD40004EF24020134621460A22C2F200000FF074
:10FD500001F84EF24020C2F200000EF0E9FF95F8E3
:10FD600019124CE70E46CBE72DE9F04100F5B673CA
:10FD700084B004460A4600F5F575106856685E6062
:10FD800018601089967A9E721881D07A00F0030666
:10FD9000C0F38100DE721873107BC0F3C30600F05D
:10FDA00007001E755873507BC0F3820600F00300F5
:10FDB000DE739873907B1874D07BC0F3440600F018
:10FDC00001009E745874107CD87415339D4202F162
:10FDD0001102D2D10B460A4653F8660FDFEDD25A14
:10FDE0005B68C4F8EA016B6091F86E3003F01F03A2
:10FDF00084F8F23191F86F30C3F3C00003F00703C9
:10FE000084F8F40184F8F3310B6FC4F8F53191F8FC
:10FE10007430C3F30115C3F3420003F0010384F807
:10FE2000FB5184F8FA0184F8F93191F8753084F8BF
:10FE3000FC3152F8761F04F2FD175368C4F8FD1127
:10FE40007B6013893B8163220123072184F80732F9
:10FE500084F8083284F8092284F80B2284F80D22F1
:10FE600084F80F2284F80A1284F80C1284F80E1217
:10FE700084F8101294F8D01084F8123206EE101A9A
:10FE800094F8D21084F8133206EE901A94F8D11038
:10FE900084F81432B8EEC66AF8EEE66A07EE101A75
:10FEA00026EE256A94F8CF1084F8153266EEA56A1E
:10FEB000B8EEC77A07EE901ABCEEC66AFCEEE66AA8
:10FEC00027EE257A8DED016ACDED026AF8EEE77A2C
:10FED0009DF804009DF8081084F81632BCEEC77A2D
:10FEE00067EEA57A88428DED037A38BF0846FCEEAE
:10FEF000E77A9DF80C10CDED017A884238BF0846AC
:10FF00009DF8041084F817328842C4F8C430C4F84D
:10FF1000C83084F8D92084F8DA3084F8DB3084F8EB
:10FF2000DC3084F8DD2084F8DE3084F8DF3084F8BB
:10FF3000E03084F8E12084F8E23084F8E33084F89B
:10FF4000E43084F8E52084F8E63084F8E73084F87B
:10FF5000E830237938BF0846102500213F2284F875
:10FF6000CC0084F81112C4F8D41084F8185284F824
:10FF7000CD0084F8CE0084F8D8201BB1A378002BE4
:10FF800040F0A381237C1BB1A37B002B40F09A811E
:10FF9000237F1BB1A37E002B40F0918194F8283081
:10FFA00023B194F82630002B40F0858194F834304A
:10FFB00023B194F83230002B40F0798194F840302E
:10FFC00023B194F83E30002B40F06D8194F84C3012
:10FFD00023B194F84A30002B40F0618194F85830F6
:10FFE00023B194F85630002B40F0558194F86430DA
:10FFF00023B194F86230002B40F0758194F8703092
:020000021000EC
:1000000023B194F86E30002B40F0698194F87C3075
:1000100023B194F87A30002B40F05D8194F8883059
:1000200023B194F88630002B40F0518194F894303D
:1000300023B194F89230002B40F05D8194F8A03009
:1000400023B194F89E30002B40F0518194F8AC30ED
:1000500023B194F8AA30002B40F0518194F8B830C5
:1000600023B194F8B630002B40F01181102384F8AE
:100070001932254604F1C00800262B793BB1AB6844
:10008000AE7018462E71EE700BB101F02BFB0C35E3
:100090004545F2D194F8D9309FED246A94F8DB10ED
:1000A00007EE903A94F8D230B8EEE77A06EE903A3E
:1000B00067EE067AF8EEE66A002267EEA67A84F822
:1000C000CE20FCEEE77A84F8CD20CDED017A9DF8C4
:1000D000043084F8CC2009B184F8CC3094F8DA20CC
:1000E000002A40F0288194F8DC200AB184F8CE3050
:1000F00094F8E1309FED0D6A94F8E31007EE903A22
:1001000094F8D030B8EEE77A06EE903A67EE067AC9
:10011000F8EEE66A67EEA67AFCEEE77ACDED017AB4
:100120009DF8043004E000BFA3707D3F0AD7233C54
:1001300031B194F8CC10994238BF194684F8CC10EC
:1001400094F8E210002940F0EE8094F8E41031B108
:1001500094F8CE00834238BF034684F8CE3094F83A
:10016000DD301FED0E6A94F8DF0007EE903A94F848
:10017000D130B8EEE77A06EE903A67EE067AF8EEFE
:10018000E66A67EEA67AFCEEE77ACDED017A9DF895
:10019000043030B194F8CC00984238BF184684F847
:1001A000CC0094F8DE00002840F0B58094F8E00020
:1001B00030B194F8CE50AB4238BF2B4684F8CE30E5
:1001C00094F8E5301FED276A94F8E75007EE903A6F
:1001D00094F8CF30B8EEE77A06EE903A67EE067AFA
:1001E000F8EEE66A67EEA67AFCEEE77ACDED017AE4
:1001F0009DF8043035B194F8CC509D4238BF1D466F
:1002000084F8CC5094F8E650002D7CD194F8E85056
:1002100035B194F8CE60B34238BF334684F8CE305F
:100220002AB920B919B915B97F2384F8CE30012530
:1002300041F654600A22394684F81D52C2F2010088
:1002400014F00CFD45F664100721C0F202000DF019
:100250005BFE41F65460C2F2010014F091FC0146CD
:1002600041F65460C2F201000DF04EFE45F66C10EE
:100270000921C0F202000DF047FE4EF24020C2F20A
:1002800000000EF055FD284604B0BDE8F0810023C3
:1002900084F8B630EAE6002384F85630A6E6002358
:1002A00084F84A309AE6002384F83E308EE6002334
:1002B00084F8323082E6002384F8263076E6002384
:1002C000A3766BE60023A37362E6A1705AE60023CF
:1002D00084F88630AAE6002384F87A309EE600236C
:1002E00084F86E3092E6002384F8623086E60023BC
:1002F00084F89E30AAE6002384F892309EE600231C
:1003000084F8AA30AAE694F8CD509D4238BF1D4625
:1003100084F8CD507AE794F8CD00984238BF18465B
:1003200084F8CD0042E794F8CD10994238BF1946C1
:1003300084F8CD1009E784F8CD30D4E610B5044632
:1003400014F01EFC01462046BDE810400DF0DCBD57
:1003500010B5044614F014FC014620460DF0D4FDFF
:1003600004464EF24020C2F200000EF0E1FC2044B0
:1003700010BD00BF2DE9F04100262F270C468E60EE
:100380000E604E60C1F80B600A2201F8017B8046C6
:1003900013F0CAFF204614F0F3FB08EB480540F2C7
:1003A0003002C2F2010208EB85051544431C2754B4
:1003B0002946E01814F080FB4EF2402746F2A010C8
:1003C000C2F200072121C0F202000DF09DFD33466C
:1003D0000A22414638460EF0BDFC46F2C4100A21FE
:1003E000C0F202000DF090FD284614F0C9FB014652
:1003F00028460DF089FD45F6F4400321C0F20200C5
:100400000DF082FD204614F0BBFB014620460DF0A6
:100410007BFD45F2D870C0F2020001210DF074FDA1
:100420003846BDE8F0410EF083BC00BF10B584B083
:100430000C460146684614F03FFB45F6001168463D
:10044000C0F2020114F03EFC28B10146204614F02F
:1004500033FB04B010BD46F2D013C0F2020303CB4D
:100460002060616004B010BD2DE9F04194B00446F5
:1004700004A804F085FB41F6F440C2F201004FF4F9
:10048000B072002114F04CFA41F25C53C2F2010345
:100490001B7833B904A804F081FB002014B0BDE838
:1004A000F08148F21F53C5F2EB13A3FB04235B0951
:1004B000642000FB1340C0B26946FFF75BFF46F2C1
:1004C000D8101E21C0F202000DF01EFD684614F087
:1004D00057FB014668460DF017FD45F2D870012123
:1004E000C0F202000DF010FD4EF24020C2F20000FA
:1004F0000EF01EFC49F2140101236A460CA8C2F258
:10050000010104F019FC14AB9DF8344053F8131D9D
:10051000CDF81D105A689E681D7B0E99CDF82120DC
:10052000139B9DF83C20CDF825600CA88DF8295030
:100530008DF8144006918DF81C200B9304F02EFBCF
:1005400004A804F045FB0028A4D004A804F03CFB58
:1005500041F2080398420DD046F2F8101A21C0F279
:1005600002000DF0D1FC4EF24020C2F200000EF06D
:10057000DFFB8FE704A804F073FAF0280DD046F2F1
:1005800014201F21C0F202000DF0BEFC4EF24020EC
:10059000C2F200000EF0CCFB7CE704A804F060FA85
:1005A00043280DD046F234201C21C0F202000DF089
:1005B000ABFC4EF24020C2F200000EF0B9FB69E73E
:1005C00041F2070104A804F0F5FA04A804F048FA7F
:1005D000F72806D046F25420C0F20200FFF7B8FE1A
:1005E00058E7032104A804F0E5FA04A804F038FA57
:1005F000092806D046F27420C0F20200FFF7A8FED8
:1006000048E741F2060104A804F0D4FA04A804F073
:1006100027FA062146B204A804F0CCFA04A804F094
:100620001FFA002741F6F44502463C46B846C2F29E
:10063000010516E004F014FA04F07F0108EB8803CA
:1006400008EB43030246A1F1760009282B449CBF26
:100650005B1803F8762C7F2904BF08F101085FFAC4
:1006600088F80134A4B2D2B2B4F5805F04A8A7EB35
:100670000207DFD146F29420C0F20200FFF75EFECF
:1006800007F07F074EF24020394600231022C2F2C5
:1006900000000EF05FFB46F2A820C0F20200FFF758
:1006A0004DFE4EF24020002310223146C2F20000DF
:1006B0000EF050FB45F2D870C0F20200FFF748FE82
:1006C000B7423FF4E7AE46F2B020C0F20200FFF7B7
:1006D00035FE4EF24020394600231022C2F20000BF
:1006E0000EF038FB46F2D020C0F20200FFF726FEE3
:1006F0004EF24020314600231022C2F200000EF0DC
:1007000029FB4EF24020C2F200000EF011FBC1E6C0
:100710002DE9F04192B002A804F032FA40F2300024
:10072000C2F2010040F21452002114F0F9F841F233
:100730005C53C2F201031C78002C00F09E8040F252
:100740003006C2F20106002408E00AA804F026FAE6
:1007500002A804F03DFA002800F08F802F23002526
:100760000A220DF10501204601958DF8043013F0A1
:10077000DBFD49F21401C2F20101012301AA0AA81A
:1007800004F0DAFA9DF82CE00C9D9DF834709DF889
:1007900036009DF837109DF838209DF839309DF8C7
:1007A0003AC09DF835808DF80CE004959DF83BE04B
:1007B0008DF814709DF83D509DF83C708DF8160032
:1007C0008DF817109DF83E009DF83F108DF8182009
:1007D0008DF819309DF840209DF841308DF81F109C
:1007E0008DF820208DF81AC08DF81BE08DF81E00C2
:1007F0008DF815808DF81C708DF81D508DF8213006
:100800000AA8119B099304F0C9F902A804F0E0F9C1
:10081000012202A988B30AA804F006FB0AA804F082
:10082000C1F9002891D10AA804F0BAF904EB4405F3
:1008300004EB850535440146284614F03DF946F29F
:10084000D8200C21C0F202000DF05EFB284614F007
:1008500097F9014628460DF057FB45F2D870012163
:10086000C0F202000DF050FB4EF24020C2F2000038
:1008700001340EF05DFAE4B267E702A804F08EF9E5
:10088000204612B0BDE8F0812DE9F0470E469046B3
:10089000054604F099F941F2080398420FD046F258
:1008A000F810C0F202001A210DF02EFB4EF240208B
:1008B000C2F200000EF03CFA0020BDE8F0872846A6
:1008C00004F0CEF8F02805D046F21420C0F2020061
:1008D0001F21E9E7284604F0C3F8432805D046F273
:1008E0003420C0F202001C21DEE741F20701284655
:1008F00004F060F9284604F0B3F8F72805D046F272
:100900005420C0F202001D21CEE70321284604F046
:1009100051F9284604F0A4F8092804D046F27420BE
:10092000C0F20200EFE741F20601284604F042F966
:10093000284604F095F806214FFA80F9284604F07D
:1009400039F906F1010A00244FEACA1AF6012746CE
:10095000284604F085F8B442C3B2A7EB030704DBD2
:10096000A31B5445B8BF08F803000134B4F5805FF9
:10097000EED146F294201221C0F202000DF0C4FA2A
:1009800007F07F074EF24020002310223946C2F2C2
:1009900000000EF0DFF946F2A8200421C0F20200A8
:1009A0000DF0B2FA4EF24020002310224946C2F266
:1009B00000000EF0CFF945F2D8700121C0F202001C
:1009C0000DF0A2FA4EF24020C2F200000EF0B0F993
:1009D0004F4508D140F22C03C2F2010300221A80D5
:1009E0000120BDE8F08746F2B0201F21C0F20200CE
:1009F0000DF08AFA4EF24020394600231022C2F24E
:100A000000000EF0A7F946F2D0200621C0F2020045
:100A10000DF07AFA4EF24020494600231022C2F22D
:100A200000000EF097F94EF24020C2F200000EF0E6
:100A30007FF90020BDE8F08730B541F25C52C2F288
:100A40000102B5B01378002B00F09C80044604A886
:100A50000D4604F095F848F21F53C5F2EB13A3FBC3
:100A600004235B09642000FB1340C0B26946FFF712
:100A700081FC49F2140101236A4614A8C2F2010163
:100A800004F05AF934AB9DF8544053F8732DCDF867
:100A90001D2059689A681B7BCDF82110CDF82520C0
:100AA00016999DF85C208DF8293014A81B9B8DF8B1
:100AB000144006918DF81C200B9304F06FF804A8E5
:100AC00004F086F8044600BB46F2E8201021C0F28C
:100AD00002000DF019FA684614F052F80146684613
:100AE0000DF012FA46F2FC20C0F2020008210DF0CF
:100AF0000BFA4EF24020C2F200000EF019F904A8E1
:100B000004F04CF8204635B030BDDDF82130DDF87A
:100B10001D20CDF84130DDF82530CDF84530CDF839
:100B20003D209DF82930069A8DF849300E929DF8A7
:100B300014308DF8343046F670129DF81C308DF864
:100B40003C30C0F2020205F01F050B9B0C922946B7
:100B50000CA814AA1393FFF797FE04460CA804F000
:100B60001DF804BB46F218301A21C0F202000DF045
:100B7000CBF94EF24020C2F200000EF0D9F804A8E2
:100B800004F00CF846F234301321C0F202000DF0EC
:100B9000BBF94EF24020C2F200000EF0C9F800246A
:100BA000204635B030BD0A220DF1C6010CA814F064
:100BB00055F846F208300E21C0F202000DF0A4F9FB
:100BC000684613F0DDFF014668460DF09DF945F6D5
:100BD00014600221C0F202000DF096F905EB8503C6
:100BE00041F6F44005EB4305C2F2010005442846F6
:100BF00013F0C6FF014628460DF086F945F2D8707D
:100C00000121C0F202000DF07FF94EF24020C2F245
:100C100000000EF08DF841F29053C2F2010314A9C6
:100C20001868FFF7A1F8044669E700BF0AF034BD71
:100C30000022C0F8A421C0F89C21C0F8B421C0F85B
:100C4000AC21C0F8C421C0F8BC21C0F8D421C0F840
:100C5000CC21C0F8E421C0F8DC21C0F8F421C0F8B0
:100C6000EC2170472DE9F04F45F255541646C0F27D
:100C7000150404FB06F49A4604F142732DED088B2B
:100C800008EE903A4FF04E530AEE103A4CF28303BE
:100C9000CBF6CA6309EE903A43F27A63C3F6AB43EC
:100CA00009EE103A4DF20A73C3F623430BEE103AE5
:100CB0004AF63B23C4F6B83345F256550AEE903A4D
:100CC00018EE903AC5F2555593B085FB022703F212
:100CD00031733246A7EBE67746F2903B08EE903A46
:100CE0004FEA6A0303958146073F08930C46054681
:100CF000C0F2020B0026099190464EE0BAF1000FB7
:100D000000F30F816FF0EE0101FB02F20732D21007
:100D100000EB0213002F23EAE373627B40F3FF80B2
:100D20001F2FCCBFC2EB42127A43D21000920AA905
:100D30000EAA09EB060000F007FD627CA37CE17CB3
:100D4000207D002A7AD003F0030C4FF0640E40F6A9
:100D500078031EFB0C11C0F2440303FB01F30728C8
:100D60004FEAE301C3BF073843F2914343430023F3
:100D70000B44C5F86C22C5F83032A37B03F00303A3
:100D800044365BF82330C5F85432B6F5CC7F04F115
:100D9000150405F1040500F0D480207821796278EB
:100DA00063790A90A0780E910B92A179E2780F9363
:100DB0000C90E379207C0D921193109100F01EFEAF
:100DC000237AC3EB0803B3F1110200F18680039A82
:100DD000217B94F80AE0103B82FB03C2A2EBE37391
:100DE00001B303291ED01F2BDBBF46F22042C0F205
:100DF0000202FA23D35C03FB0EFE40F2491303FB0D
:100E00000EF301294FEAE33316DD18447F28A8BF0B
:100E10007F20BAF17F0F4FEA4010E27B7FF76EAF81
:100E20000F2171E703FB0EF340F2491202FB03F3BB
:100E300001294FEA2333E8DC5B42E6E7B8EEE88AB3
:100E4000079028EE0A0A069120EE290A05930492DB
:100E500010F0B6F920EE090AF1EE0C7A80EE277A4E
:100E60000798059B0699073846F2A03E03F01F033A
:100E7000C0F2020E5EF8233007EE900A27EE087AE1
:100E8000F8EEE77AA7EE278ABDEEC88A18EE102A98
:100E90001A441346049A00293FF46BAF07EE901AE8
:100EA000F8EEE77AB7EE000AA7EE8B0A059310F08A
:100EB00009FAF6EE007AE0EE2A7A17EE900A12F0BE
:100EC00045FE41EC100B0FF057FC51EC100B13F0EA
:100ED00041F9059B049A03444BE7039B94F809C02E
:100EE000C2F10101E27A83FB013EAEEBE17102B394
:100EF000032A1ED01F29DBBF46F2204EC0F2020E8D
:100F0000FA211EF8011040F2491301FB0CF103FB1A
:100F100001F3DB13012A3FF778AF5B4275E700224C
:100F200004E746F24833C0F202030899595CEF39EE
:100F3000EAE601FB0CF140F2491303FB01F31B133A
:100F4000E8E7DDF8248098F87E5098F8824098F819
:100F50007F3098F8830098F880600A950E9498F88E
:100F6000845098F881400B930F9098F88530119336
:100F70000EAA0AA909F5FC700C9610950D9401F0C3
:100F800029FA98F88630C9F8883298F887302BB358
:100F9000C3F10803C9F8503298F88B3003EB830390
:100FA00003EB43139B11C9F88C3298F88F3046F24B
:100FB0008832C0F2020203F00703D35CC9F8903212
:100FC00098F88C3003EB830303EB43139B11C9F8B0
:100FD000843213B0BDEC088BBDE8F08F1023D9E745
:100FE0002DE9F04F2DED048B89B0D0F89052DDF84B
:100FF000588007918146D0F88C0298F80DE09B4606
:10100000A2F5000305FB03F500FB0BF0A0FB056751
:10101000EB1700FB037714468EFB0523900B40EA89
:101020008340FE1186EAE67380EAE072A2EBE0728A
:10103000A3EBE6739342B8BF134609F5FC701E4656
:1010400001F000FAD8F80030002DB4BF4FF0FF32A5
:101050000122B3F5005A06FB02001AD0D8F8082086
:10106000002A40F0D980D8F804304FEACA2A07EEA7
:1010700090AA07EE103AF8EEE77AB8EEC77AF2EEE9
:10108000086A67EE877A87EEA67AFDEEC77A17EED2
:1010900090AA4FF05A5309EE103A45F62943C3F689
:1010A0008F53D9F8842298F80C1008EE903A43F246
:1010B0003333C4F2431308EE103A82FB0B23C4F11E
:1010C00080744FEA122B4BEA036BE3170BFB03F21E
:1010D00098F80E30002704FB07225B04ABFB046783
:1010E00081FB0445C3F57E0BE30943EA45635B4599
:1010F00017444FEA166138BF5B4641EA0721D8F82A
:1011000014208B4238BF0B4692449B4600EB0A03E7
:1011100005934E4609F50C744F46002514E05044E3
:1011200001F040F8C6F8A001384600F065FB626A9D
:1011300002BBC6F898010135062D07F1440706F1F8
:10114000100604F1040452D098F818302B4113F023
:10115000010344D0E36B2068002BE0D1059B1844C9
:1011600001F020F8C6F8A001384600F045FB626A9D
:10117000002ADED0D117ABFB0223CDE90223039A6C
:1011800006900BFB01230393DDE90201020E42EA04
:10119000012207EE902AF8EE677AB0EE480A67EE71
:1011A000897AA7EEA80A10F00BF8FCEEC07A069830
:1011B00017EE901AC3174FEA011E0EFB03F3090F37
:1011C00000FB0131AEFB0023CDE902230B44039366
:1011D000029B1A0F039B42EA0312801AA9E73846C2
:1011E000029300F009FB029BC6F89831A3E7D8F8F8
:1011F0002C00D9F850120268D9F88832019109F50B
:10120000127100919468079909F5CC72A04709B052
:10121000BDEC048BBDE8F08F21230C21C8F2040340
:1012200091FBF2F202FB0AFA83FB0A1353444FEAE2
:10123000EA7ACAEB233A41F6FF7393FBF2F303FB1E
:101240000AFA4FEACA2A24E770B50646044600F5B2
:10125000CC7520460021443400F080FBAC42F8D12C
:1012600006F5FC700021BDE8704001F039B900BFFF
:101270002DE9F04F45F255549246C0F2150404FB97
:101280000AF4994604F142732DED088B08EE903A6A
:101290004FF04E530AEE103A4CF28303CBF6CA637A
:1012A00009EE903A43F27A63C3F6AB4309EE103A83
:1012B0004DF20A73C3F623430BEE103A4AF63B2372
:1012C000C4F6B83345F256550AEE903A18EE903A05
:1012D000C5F2555593B085FB0A2803F23173A8EB8C
:1012E000EA7846F2903B08EE903A4FEA690302959D
:1012F000074607900891A8F1070809930C46054690
:10130000C0F2020B00262AE0B9F1000F00F31281AF
:101310006FF0EE0101FB02F20732D21000EB021374
:10132000B8F1000F23EAE373627B40F30181B8F167
:101330001F0FCCBFC2EB421208FB02F2D210009288
:10134000384601360EAA0AA900F062FB062E04F107
:10135000150405F1040507F1440700F0FB80627CE9
:10136000A37CE17C207D002A71D003F0030C4FF0B8
:10137000640E40F678031EFB0C11C0F2440303FB1D
:1013800001F307284FEAE301C3BF073843F2914353
:10139000434300230B44C5F83032A37BC5F86C22CD
:1013A00003F003035BF82330C5F854322078217929
:1013B000627863790A90A0780E910B92A179E27815
:1013C0000F930C90E379207C0D921193109100F013
:1013D00015FB237AC3EB0A03B3F1110200F18680F7
:1013E000029A217B94F80AE0103B82FB03C2A2EB35
:1013F000E37301B303291ED01F2BDBBF46F220424B
:10140000C0F20202FA23D35C03FB0EFE40F2491342
:1014100003FB0EF301294FEAE33316DD18447F285E
:10142000A8BF7F20B9F17F0F4FEA4010E27B7FF722
:101430006BAF0F216EE703FB0EF340F2491202FB84
:1014400003F301294FEA2333E8DC5B42E6E7B8EE19
:10145000E88A069028EE0A0A059120EE290A0493EC
:1014600003920FF0ADFE20EE090AF1EE0C7A80EE49
:10147000277A0698049B0599073846F2A03E03F0A8
:101480001F03C0F2020E5EF8233007EE900A27EE2B
:10149000087AF8EEE77AA7EE278ABDEEC88A18EE3A
:1014A000102A1A441346039A00293FF474AF07EE3A
:1014B000901AF8EEE77AB7EE000AA7EE8B0A0493CB
:1014C0000FF000FFF6EE007AE0EE2A7A17EE900AAF
:1014D00012F03CFB41EC100B0FF04EF951EC100BED
:1014E00012F038FE049B039A034454E7029B94F8DD
:1014F00009C0C2F10101E27A83FB013EAEEBE1716A
:1015000002B3032A1ED01F29DBBF46F2204EC0F2D1
:10151000020EFA211EF8011040F2491301FB0CF1F2
:1015200003FB01F3DB13012A3FF778AF5B4275E75A
:10153000002204E746F24833C0F202030999595CDD
:10154000EF39E7E601FB0CF140F2491303FB01F32D
:101550001B13E8E7089A079992F88630C1F8883299
:1015600092F887303BB3C3F1080308461446C0F82D
:10157000503294F88B3003EB830303EB43139B113E
:10158000C0F88C3294F88F3046F28832C0F20202F2
:1015900003F00703D35CC0F8903294F88C3003EB6F
:1015A000830303EB43139B11C0F8843213B0BDECEB
:1015B000088BBDE8F08F102308461446D7E700BF1C
:1015C0002DE9F84F43F66C7A804689460646A1F12C
:1015D000040B01F1180500F160070446C2F2010A8C
:1015E000D4F8981101F172414A1340F2FE7313408E
:1015F000581C5AF823205AF82000C1F30D0382FB2F
:101600000323920B42EA83420916C1F10601024408
:101610000A413046294610344BF8042F00F050FAA6
:10162000A74205F1010506F14406D9D109F11E01D1
:1016300008F5FC70BDE8F84F00F080BF2DE9F041DF
:1016400004460F4600F5CC7806460D46394620463E
:1016500000F03AFAD5F89C31C6F89C314434D5F8FC
:10166000A431C6F8A431444507F1440705F110053B
:1016700006F11006EAD1BDE8F08100BFD1F8AC3127
:10168000D1F8A42110B4D1F89C41C0F89C41C0F815
:10169000A421C0F8AC31D1F8B431C0F8B431D1F8DC
:1016A000BC31C0F8BC31D1F8C431C0F8C431D1F874
:1016B000CC31C0F8CC31D1F8D431C0F8D431D1F824
:1016C000DC31C0F8DC31D1F8E431C0F8E431D1F8D4
:1016D000EC31C0F8EC31D1F8F431C0F8F4315DF8F8
:1016E000044B70470023C0F89C31C0F8A431C0F807
:1016F000AC31C0F8B431C0F8BC31C0F8C431C0F866
:10170000CC31C0F8D431C0F8DC31C0F8E431C0F8D5
:10171000EC31C0F8F43170474FF48843C4F22C73B5
:1017200007EE103A87EE000A4FF0974307EE903A23
:1017300020EE270A4DF6D463BCEEC00AC2F20003C5
:1017400083ED000A704700BF30B40C680460146871
:1017500004614D684560556845618D688560956890
:101760008561C968C160D268C261132C4FF0000264
:1017700082624263DBBF46F24442C0F202021C3482
:1017800052F824400362641003EB8413A3F58553DD
:10179000026802994162102B02EB8204B8BF102349
:1017A00002EBC4021B04002B01EBA212D4BF0024E5
:1017B000012401253E2A80F84050C36280F8304061
:1017C00016DC02F0030392100433083203FA02F22B
:1017D000D3174DF6D461C2F200010968A1FB02459E
:1017E00001FB0355230E43EA0523836330BC704796
:1017F0004FF060720023ECE7426B022AF0B403461C
:1018000005DD032A66D190F84010002962D193F8D3
:10181000301071B9986A996BDC6A401AA0429862DC
:1018200059DC511C03299C6259635BDD2046F0BCE6
:1018300070474FF6FF70996AC0F2B36081424CDD89
:10184000C1F1885000169D6BDC6A05FB0010A042B8
:10185000986240DB511C03299C625963E6DC03EB70
:10186000820251691329DBBF46F24440C0F20200F4
:1018700001F11C0550F82150196A586A6D1001EBEE
:101880008511A1F585511029B8BF102109048C429A
:10189000ACBF00250125D96283F83050526802EBB5
:1018A000820102EBC10200EBA2123E2A4CDD4FF096
:1018B000607600274DF6D462C2F20002204612681C
:1018C000A2FB064502FB0755220E42EA05229A6357
:1018D000F0BC7047986AF0BC70470021C0F2B46158
:1018E0000A20B0E703EB820251691329DBBF46F2FD
:1018F0004440C0F2020001F11C0550F82150196A61
:10190000586A6D1001EB8511A1F585511029B8BFFA
:10191000102109048C42ACBF00250125D96283F84F
:101920003050526802EB820102EBC10200EBA210C0
:101930003E28BCDC00F0030680100436083006FAAE
:1019400000F00646C717B5E702F00306921004360A
:10195000083206FA02F21646D717ABE790F8403085
:101960008B4241D000290CBF0323002330B49D00DB
:10197000421980F8401043631369816A132BDBBF5F
:1019800046F24442C0F2020203F11C0452F8234022
:10199000036A426A641003EB8413A3F58553102B8A
:1019A000B8BF10231B048B42D4BF0021012180F853
:1019B0003010C362435903EB830103EBC10302EB15
:1019C000A3123E2A11DD4FF0607200234DF6D46160
:1019D000C2F200010968A1FB024501FB0355230E79
:1019E00043EA052330BC8363704702F0030392107F
:1019F0000433083203FA02F2D317E7E71328DBBFF8
:101A000046F24443C0F202031C3053F820007047F2
:101A100030B40C680460146804614C684460546815
:101A200044618C68846094688461C968C16090F87E
:101A30004010D568029AC56103624262002934D021
:101A4000132CDBBF46F24441C0F202011C3451F8B2
:101A500024408568816A641003EB8413A3F58553E1
:101A6000102BB8BF102305EB85041B0405EBC40540
:101A70008B4202EBA512D4BF0021012102243E2A91
:101A8000C36280F83010446311DD4FF060720023B0
:101A90004DF6D461C2F200010968A1FB024501FBC9
:101AA0000355230E43EA0523836330BC704702F0DD
:101AB000030322410433083203FA02F2D317E7E7A3
:101AC000436B0B70704700BF0A680B6903610260CB
:101AD0004B6843604B6943618B6883608B698361AA
:101AE000CB68C360F0B5CB69C3610B6A4F6A8E6A7D
:101AF000CD6A91F830E04C6B8A6B036291F840300C
:101B000047628662C56280F830E04463826380F891
:101B10004030F0BD70B54FF09D432DED048B08EEC5
:101B2000103A41F23063002143F66C74C3F68073BF
:101B30000020C4F2D01108EE903AC2F20104002550
:101B4000B6EE009A0BE078EE097A17EE900A11F0E3
:101B5000FDFF41EC100B0EF00FFE51EC100B6E0070
:101B600012F0F8FA01360135B5F5806F28EE288AB3
:101B700044F82600E7D1002340F2FF355A00D11C7B
:101B8000501C54F8211054F820000133091AAB42BC
:101B900043F66C7044F82210C2F20100EED141F617
:101BA000FC73BDEC048BC35841F6F872C3F10043DB
:101BB000835070BD002207EE902A4FF0974202EE4C
:101BC000102A4FF06C5204EE902A4FF06E5202EE43
:101BD000902A4AF6AB22C3F62A2241F66C7303EE32
:101BE000102AC2F201030022F6EE003AB7EE006AB4
:101BF000B0EE004AF0EE465AE7EEE75A03EBC201B8
:101C00000132B0EE677AA5EEA47AB2F5806FB0EE3D
:101C1000465AA7EE475AF0EE636AE7EE826AB0EEE4
:101C2000677AA5EE247AFDEEE66AC1ED016AF0EE70
:101C3000466AE7EE476AB0EE677AA6EEA27A76EEDB
:101C4000856AB0EE465AA7EE475A35EE257AA6EEDB
:101C5000847AE7EE037ACDD130B4002240F2FF352A
:101C60005100C81C4C1C53F8200053F8244001328A
:101C7000001BAA4241F66C7443F82100C2F2010431
:101C8000EED14FF0974306EE903AB6EE007AA7EE0B
:101C9000A67A41F6FC7341F6F872E358FDEEC77A76
:101CA00017EE901ACB1AA35030BC7047704700BF94
:101CB0002DE9F04F46F2A84491B003EB4303C0F284
:101CC000020404EBC3041546069007910FCC0AAE3C
:101CD0000FC694E80300002386E803004FF00108D4
:101CE00043F66C760AAF05F160098DF824808DF813
:101CF00025308DF82630C2F2010605973BE00AF147
:101D0000FF30069B00EB001003EB0010133020F0B7
:101D10000F0095E8084003F1724B4FEA6B3340F235
:101D2000FE721A40531C56F8222056F82340CBF37B
:101D30000D0382FB0323920B4FEA2B6B42EA834293
:101D4000CBF1060B144444FA0BF4BEF58C6F6C60B7
:101D50001CDAB4F58C6F19DABCF1000F03D110ABAB
:101D60009A440AF81CCCEB68AA6803EB8213EB6078
:101D70001035A9452FD0059B53F8041B059311F08E
:101D8000030A01F0040CBAD10798C2E710AB9A44D9
:101D90001AF81C3C1BB11CF1000318BF0123C1F34E
:101DA00001123AB110AF07EB020C1CF81CCCBCF1CD
:101DB000000F13D101F0C001C02902D11B9A0F2AD4
:101DC00020DDAA68E96801930094734600F0D6F814
:101DD0000AF81C8CC7E711B0BDE8F08F0699D5F85A
:101DE00008C0013A02EB021201EB02111331EA685A
:101DF000029321F00F0163460194CDF800E000F05A
:101E000051F8E5E71746E968AA6802971A9F039315
:101E10008DE89000734600F00FF9D9E710B54FF444
:101E2000097104460DF0F4F8204610BD46F2A843AF
